 sw_utilityG

 Timestamp is 548ff4fc (Tue Dec 16 17:01:48 2014)

 Preferred load address is 00100000

 Start         Length     Name                   Class
 0001:00000000 0002a760H .text                   CODE
 0001:0002a760 00000758H .text$yc                CODE
 0001:0002aeb8 000001ccH .text$yd                CODE
 0002:00000000 00015b2cH .rdata                  DATA
 0002:00015b2c 00000078H .rdata$debug            DATA
 0002:00015ba4 00000148H .xdata                  DATA
 0002:00015cec 00000034H .xdata$x                DATA
 0002:00015d20 00000004H ATL$__a                 DATA
 0002:00015d24 00000004H ATL$__z                 DATA
 0002:00015d28 00000050H .idata$2                DATA
 0002:00015d78 00000014H .idata$3                DATA
 0002:00015d8c 000002a8H .idata$4                DATA
 0002:00016034 0000007aH .idata$6                DATA
 0002:000160b0 00001ca2H .edata                  DATA
 0003:00000000 000002a8H .idata$5                DATA
 0003:000002a8 00000004H .CRT$XCA                DATA
 0003:000002ac 00000004H .CRT$XCAA               DATA
 0003:000002b0 0000000cH .CRT$XCC                DATA
 0003:000002bc 0000005cH .CRT$XCL                DATA
 0003:00000318 00000014H .CRT$XCU                DATA
 0003:0000032c 00000004H .CRT$XCZ                DATA
 0003:00000330 00000004H .CRT$XIA                DATA
 0003:00000334 00000004H .CRT$XIZ                DATA
 0003:00000338 00000004H .CRT$XPA                DATA
 0003:0000033c 00000004H .CRT$XPZ                DATA
 0003:00000340 00000004H .CRT$XTA                DATA
 0003:00000344 00000004H .CRT$XTZ                DATA
 0003:00000348 000001d8H .data                   DATA
 0003:00000520 00002b60H .bss                    DATA
 0004:00000000 00001490H .pdata                  DATA
 0005:00000000 000000a0H .rsrc$01                DATA
 0005:000000a0 000003dcH .rsrc$02                DATA

  Address         Publics by Value              Rva+Base       Lib:Object

 0000:00000000       ___safe_se_handler_count   00000000     <absolute>
 0000:00000000       ___safe_se_handler_table   00000000     <absolute>
 0001:00000000       ??4CVerInfo@@QAAAAV0@ABV0@@Z 00101000 f i CVERINFO.obj
 0001:00000038       ?ValueAvailable@@YAHI@Z    00101038 f   CVERINFO.obj
 0001:00000084       ??0CVerInfo@@QAA@XZ        00101084 f   CVERINFO.obj
 0001:000000e8       ??0CVerInfo@@QAA@PAG@Z     001010e8 f   CVERINFO.obj
 0001:0000012c       ??0CVerInfo@@QAA@PAUHINSTANCE__@@@Z 0010112c f   CVERINFO.obj
 0001:00000190       ??1CVerInfo@@QAA@XZ        00101190 f   CVERINFO.obj
 0001:000001d8       ?Init@CVerInfo@@AAAHPAG@Z  001011d8 f   CVERINFO.obj
 0001:00000228       ?InitVerInfoStruct@CVerInfo@@AAAHPAG@Z 00101228 f   CVERINFO.obj
 0001:0000038c       ?GetVerResourceStr@CVerInfo@@QAAPAGPAG@Z 0010138c f   CVERINFO.obj
 0001:000003f0       ?GetProductVersionStr@CVerInfo@@QAAPAGXZ 001013f0 f   CVERINFO.obj
 0001:0000041c       ?GetFileVersionStr@CVerInfo@@QAAPAGXZ 0010141c f   CVERINFO.obj
 0001:00000444       ?GetProductNameStr@CVerInfo@@QAAPAGXZ 00101444 f   CVERINFO.obj
 0001:00000474       ?GetVerResourceString@CVerInfo@@AAAPAGPAG@Z 00101474 f   CVERINFO.obj
 0001:0000053c       ?SetProductNameStr@CVerInfo@@AAAXXZ 0010153c f   CVERINFO.obj
 0001:000005dc       ?SetFileVersionStr@CVerInfo@@AAAXXZ 001015dc f   CVERINFO.obj
 0001:0000067c       ?SetProductVersionStr@CVerInfo@@AAAXXZ 0010167c f   CVERINFO.obj
 0001:00000724       ??0SW_RegistryKey@@QAA@ABV0@@Z 00101724 f i ModemStat.obj
 0001:00000788       ??4SW_RegistryKey@@QAAAAV0@ABV0@@Z 00101788 f i ModemStat.obj
 0001:000007dc       ?HKey@SW_RegistryKey@@IBAQAUHKEY__@@XZ 001017dc f i ModemStat.obj
 0001:00000808       ?HKey@SW_RegistryKey@@IAAQAUHKEY__@@QAU2@@Z 00101808 f i ModemStat.obj
 0001:00000850       ?Buffer@SW_RegistryKey@@IBAPAXXZ 00101850 f i ModemStat.obj
 0001:0000087c       ?Buffer@SW_RegistryKey@@IAAXPAX@Z 0010187c f i ModemStat.obj
 0001:0000089c       ?IsOpen@SW_RegistryKey@@UAAHXZ 0010189c f i ModemStat.obj
 0001:000008f4       ??0CModemStatus@@QAA@XZ    001018f4 f   ModemStat.obj
 0001:00000ce0       ??1CModemStatus@@UAA@XZ    00101ce0 f   ModemStat.obj
 0001:00000d68       ?Initialize@CModemStatus@@QAAXXZ 00101d68 f   ModemStat.obj
 0001:0000103c       ?PrepareRilDevSpecificInfo@CModemStatus@@QAAPAUtagDEVSPECIFICDATA@@KKAAK@Z 0010203c f   ModemStat.obj
 0001:00001440       ?RILInitializeThread@@YAIPAX@Z 00102440 f   ModemStat.obj
 0001:000014f4       ?RILRegister@CModemStatus@@QAAHXZ 001024f4 f   ModemStat.obj
 0001:00001644       ?RILDeregister@CModemStatus@@QAAHXZ 00102644 f   ModemStat.obj
 0001:000016f8       ?RilNotifyCallback@@YAXKPBXKK@Z 001026f8 f   ModemStat.obj
 0001:000030fc       ?UpdateCallTypeAndStatus@CModemStatus@@QAAKKKGAAH@Z 001040fc f   ModemStat.obj
 0001:00003ad8       ?RilResultCallback@@YAXKJPBXKK@Z 00104ad8 f   ModemStat.obj
 0001:000043c4       ?ClearErrorObjectFunc@@YAXAAUtagErrorInfo@@@Z 001053c4 f   ModemStat.obj
 0001:00004400       ?PROCESS_RESULT@@YAXKK@Z   00105400 f   ModemStat.obj
 0001:0000444c       ?PROCESS_RESULT_WITH_PAYLOAD@@YAXKPAPAEPAKK@Z 0010544c f   ModemStat.obj
 0001:00004540       ?ProcessErrorFunc@@YAHAAUtagErrorInfo@@@Z 00105540 f   ModemStat.obj
 0001:00004744       ?ExecNoParamDevSpecific@@YAHKAAUtagErrorInfo@@@Z 00105744 f   ModemStat.obj
 0001:0000491c       ?ExecNoParamDevSpecificWithResponsePayload@@YAHKPAPAEPAKAAUtagErrorInfo@@@Z 0010591c f   ModemStat.obj
 0001:00004b50       ?GetEquipmentState@@YAHAAUtagErrorInfo@@@Z 00105b50 f   ModemStat.obj
 0001:00004cf4       ?GetEquipmentInfo@@YAHPAUrilequipmentinfo_tag@@AAUtagErrorInfo@@@Z 00105cf4 f   ModemStat.obj
 0001:00004f44       GetUserIdentity            00105f44 f   ModemStat.obj
 0001:00005190       GetRilDebugInfo            00106190 f   ModemStat.obj
 0001:000055f4       GetRilEVDODebugInfo        001065f4 f   ModemStat.obj
 0001:000056ac       GetRilStatus               001066ac f   ModemStat.obj
 0001:000058b0       GetRilPAParam              001068b0 f   ModemStat.obj
 0001:00005a60       GetRilPDData               00106a60 f   ModemStat.obj
 0001:00005c40       GetRilPDDLDData            00106c40 f   ModemStat.obj
 0001:00005de4       SetEquipmentState          00106de4 f   ModemStat.obj
 0001:00006014       HangUp                     00107014 f   ModemStat.obj
 0001:00006194       Dial                       00107194 f   ModemStat.obj
 0001:00006378       DialEx                     00107378 f   ModemStat.obj
 0001:00006660       ?ModGetRegistrationStatus@@YAHAAUtagErrorInfo@@@Z 00107660 f   ModemStat.obj
 0001:00006828       ?ModGetCurrentSystemType@@YAHAAUtagErrorInfo@@@Z 00107828 f   ModemStat.obj
 0001:000069f0       ?ModGetCallList@@YAHAAUtagErrorInfo@@@Z 001079f0 f   ModemStat.obj
 0001:00006bb0       ?ModGetPacketDataStatus@@YAHAAUtagErrorInfo@@@Z 00107bb0 f   ModemStat.obj
 0001:00006c78       ModGetPreferredPrivacyMode 00107c78 f   ModemStat.obj
 0001:00006e24       ?ModGetCurrentPrivacyStatus@@YAHAAUtagErrorInfo@@@Z 00107e24 f   ModemStat.obj
 0001:00006fe4       ModGetRoamingMode          00107fe4 f   ModemStat.obj
 0001:00007188       ModSetRoamingMode          00108188 f   ModemStat.obj
 0001:00007330       ModSetPreferredPrivacyMode 00108330 f   ModemStat.obj
 0001:000074d8       ModGetLocationStatus       001084d8 f   ModemStat.obj
 0001:00007670       ModSetLocationMode         00108670 f   ModemStat.obj
 0001:000078bc       ModGetRoamStatus           001088bc f   ModemStat.obj
 0001:00007a5c       ReadNv                     00108a5c f   ModemStat.obj
 0001:00007cc8       WriteNv                    00108cc8 f   ModemStat.obj
 0001:00007f5c       ValidateSpc                00108f5c f   ModemStat.obj
 0001:00008240       SetModemPowerState         00109240 f   ModemStat.obj
 0001:000082ac       GetMDNLengthSupported      001092ac f   ModemStat.obj
 0001:0000836c       SetProvisionInfo           0010936c f   ModemStat.obj
 0001:000087d4       GetAdvancedMenuInfo        001097d4 f   ModemStat.obj
 0001:00008940       GetProvisionInfo           00109940 f   ModemStat.obj
 0001:00008cdc       SetSIPNaiPassword          00109cdc f   ModemStat.obj
 0001:00008e10       ?GetModemState@@YAHPAUtagBLModemState@@AAUtagErrorInfo@@@Z 00109e10 f   ModemStat.obj
 0001:00008ee4       SaveAkey                   00109ee4 f   ModemStat.obj
 0001:000090e4       GetVersionInfo             0010a0e4 f   ModemStat.obj
 0001:000095b4       StartDebugMode             0010a5b4 f   ModemStat.obj
 0001:00009800       StopDebugMode              0010a800 f   ModemStat.obj
 0001:00009a4c       EnableTechHdrNotifications 0010aa4c f   ModemStat.obj
 0001:00009cb8       GetCarrierIndex            0010acb8 f   ModemStat.obj
 0001:00009d30       GetCallGuardRegistry       0010ad30 f   ModemStat.obj
 0001:00009d94       SetCallGuardRegistry       0010ad94 f   ModemStat.obj
 0001:00009dec       GetActWizDisabledRegistry  0010adec f   ModemStat.obj
 0001:00009e50       SetActWizDisabledRegistry  0010ae50 f   ModemStat.obj
 0001:00009ea8       GetLogoTestReg             0010aea8 f   ModemStat.obj
 0001:00009f0c       IsConsumerProduct          0010af0c f   ModemStat.obj
 0001:00009f70       EnableCarrierLogo          0010af70 f   ModemStat.obj
 0001:00009fc8       SetAutoUpdateTime          0010afc8 f   ModemStat.obj
 0001:0000a020       SetAutoUpdateTimeUI        0010b020 f   ModemStat.obj
 0001:0000a078       GetAutoUpdateTime          0010b078 f   ModemStat.obj
 0001:0000a0dc       GetAutoUpdateTimeUI        0010b0dc f   ModemStat.obj
 0001:0000a140       ChangeCarrierIndex         0010b140 f   ModemStat.obj
 0001:0000a19c       RepairPhoneBookRegKeys     0010b19c f   ModemStat.obj
 0001:0000a1f0       GetRilTechHdrinfo          0010b1f0 f   ModemStat.obj
 0001:0000a52c       ModGetSysPrefMode          0010b52c f   ModemStat.obj
 0001:0000a560       ModSetSysPrefMode          0010b560 f   ModemStat.obj
 0001:0000a7ac       ModGetHDRHybrPrefMode      0010b7ac f   ModemStat.obj
 0001:0000a7e0       ModSetHDRHybrPrefMode      0010b7e0 f   ModemStat.obj
 0001:0000aa2c       GetIOTALog                 0010ba2c f   ModemStat.obj
 0001:0000ac90       GetIOTALogSize             0010bc90 f   ModemStat.obj
 0001:0000ae78       StartIOTA                  0010be78 f   ModemStat.obj
 0001:0000b01c       StopIOTA                   0010c01c f   ModemStat.obj
 0001:0000b1b4       EnableIOTA                 0010c1b4 f   ModemStat.obj
 0001:0000b400       IsIOTAEnabled              0010c400 f   ModemStat.obj
 0001:0000b68c       GetIOTAStatus              0010c68c f   ModemStat.obj
 0001:0000b7a0       GetDsMipList               0010c7a0 f   ModemStat.obj
 0001:0000bab8       GetDsMipProfile            0010cab8 f   ModemStat.obj
 0001:0000bdb0       SetDsMipProfile            0010cdb0 f   ModemStat.obj
 0001:0000c03c       GetByteCounter             0010d03c f   ModemStat.obj
 0001:0000c2b4       ReadPDSMPAParam            0010d2b4 f   ModemStat.obj
 0001:0000c66c       StartLBTrackSession        0010d66c f   ModemStat.obj
 0001:0000c91c       EndLBTrackSession          0010d91c f   ModemStat.obj
 0001:0000cb8c       SetPDSMPAParam             0010db8c f   ModemStat.obj
 0001:0000ce7c       ReadPDSMPADldData          0010de7c f   ModemStat.obj
 0001:0000cf20       ReadPDSMPAData             0010df20 f   ModemStat.obj
 0001:0000d108       StartPDSMLocNotifstatus    0010e108 f   ModemStat.obj
 0001:0000d13c       StartPDSMDldNotifstatus    0010e13c f   ModemStat.obj
 0001:0000d170       StopPDSMLocNotifstatus     0010e170 f   ModemStat.obj
 0001:0000d1a4       StopPDSMDldNotifstatus     0010e1a4 f   ModemStat.obj
 0001:0000d1d8       StartDMMode                0010e1d8 f   ModemStat.obj
 0001:0000d424       StopDMMode                 0010e424 f   ModemStat.obj
 0001:0000d458       GetDMMode                  0010e458 f   ModemStat.obj
 0001:0000d4e4       StartPTMode                0010e4e4 f   ModemStat.obj
 0001:0000d518       StopPTMode                 0010e518 f   ModemStat.obj
 0001:0000d54c       GetPTMode                  0010e54c f   ModemStat.obj
 0001:0000d5d8       GetCallstate               0010e5d8 f   ModemStat.obj
 0001:0000d7c0       GetProvisionState          0010e7c0 f   ModemStat.obj
 0001:0000d9b8       InitiateHostBoot           0010e9b8 f   ModemStat.obj
 0001:0000dc04       RtnReset                   0010ec04 f   ModemStat.obj
 0001:0000de58       SetHdrNaiPassword          0010ee58 f   ModemStat.obj
 0001:0000df58       GetHdrNaiPassword          0010ef58 f   ModemStat.obj
 0001:0000e18c       GetActWizUIMask            0010f18c f   ModemStat.obj
 0001:0000e218       GetNAIPWUIDisplayMode      0010f218 f   ModemStat.obj
 0001:0000e4c0       GetOMADMConfig             0010f4c0 f   ModemStat.obj
 0001:0000e54c       SendATTunnel               0010f54c f   ModemStat.obj
 0001:0000e9a4       GetGSMInfo                 0010f9a4 f   ModemStat.obj
 0001:0000ebe8       GetItemnizedUMTSInfo       0010fbe8 f   ModemStat.obj
 0001:0000ef84       GetCurrentGSMBandAndList   0010ff84 f   ModemStat.obj
 0001:0000f0a4       SelectGSMBand              001100a4 f   ModemStat.obj
 0001:0000f304       GetSIPNaiPassword          00110304 f   ModemStat.obj
 0001:0000f518       ??_ECModemStatus@@UAAPAXI@Z 00110518 f i ModemStat.obj
 0001:0000f518       ??_GCModemStatus@@UAAPAXI@Z 00110518 f i ModemStat.obj
 0001:0000f558       ?SetMessageVars@CModemStatus@@SAXXZ 00110558 f i ModemStat.obj
 0001:0000f768       ResetEvent                 00110768 f i ModemStat.obj
 0001:0000f79c       SetEvent                   0011079c f i ModemStat.obj
 0001:0000f7d0       ?WAITFORCOMMANDCOMPLETION@@YAXK@Z 001107d0 f i ModemStat.obj
 0001:0000f83c       ??0SWISYNCBLOCK@@QAA@PAVCriticalSection@@@Z 0011083c f i ModemStat.obj
 0001:0000f878       ?Lock@CriticalSection@@QAA_NXZ 00110878 f i ModemStat.obj
 0001:0000f8a8       ??1SWISYNCBLOCK@@QAA@XZ    001108a8 f i ModemStat.obj
 0001:0000f8c4       ?Unlock@CriticalSection@@QAA_NXZ 001108c4 f i ModemStat.obj
 0001:0000f8f4       ??0CriticalSection@@QAA@XZ 001108f4 f i ModemStat.obj
 0001:0000f934       ??_ECriticalSection@@UAAPAXI@Z 00110934 f i ModemStat.obj
 0001:0000f934       ??_GCriticalSection@@UAAPAXI@Z 00110934 f i ModemStat.obj
 0001:0000f974       ??1CriticalSection@@UAA@XZ 00110974 f i ModemStat.obj
 0001:0000f9a0       ??0CAtlWinModule@ATL@@QAA@XZ 001109a0 f i stdafx.obj
 0001:0000fa5c       ??0_ATL_WIN_MODULE70@ATL@@QAA@XZ 00110a5c f i stdafx.obj
 0001:0000fac0       ??0CComCriticalSection@ATL@@QAA@XZ 00110ac0 f i stdafx.obj
 0001:0000faf4       ??1CComCriticalSection@ATL@@QAA@XZ 00110af4 f i stdafx.obj
 0001:0000fb04       ??0?$CSimpleArray@GV?$CSimpleArrayEqualHelper@G@ATL@@@ATL@@QAA@XZ 00110b04 f i stdafx.obj
 0001:0000fb5c       ??1CAtlWinModule@ATL@@QAA@XZ 00110b5c f i stdafx.obj
 0001:0000fb9c       ?Term@CAtlWinModule@ATL@@QAAXXZ 00110b9c f i stdafx.obj
 0001:0000fbd0       ?GetModuleInstance@CAtlBaseModule@ATL@@QAAPAUHINSTANCE__@@XZ 00110bd0 f i stdafx.obj
 0001:0000fc04       ??1_ATL_WIN_MODULE70@ATL@@QAA@XZ 00110c04 f i stdafx.obj
 0001:0000fc50       ?AtlWinModuleTerm@ATL@@YAJPAU_ATL_WIN_MODULE70@1@PAUHINSTANCE__@@@Z 00110c50 f i stdafx.obj
 0001:0000fd50       ?Term@CComCriticalSection@ATL@@QAAJXZ 00110d50 f i stdafx.obj
 0001:0000fd7c       ?GetSize@?$CSimpleArray@GV?$CSimpleArrayEqualHelper@G@ATL@@@ATL@@QBAHXZ 00110d7c f i stdafx.obj
 0001:0000fda8       ?RemoveAll@?$CSimpleArray@GV?$CSimpleArrayEqualHelper@G@ATL@@@ATL@@QAAXXZ 00110da8 f i stdafx.obj
 0001:0000fe3c       ??A?$CSimpleArray@GV?$CSimpleArrayEqualHelper@G@ATL@@@ATL@@QAAAAGH@Z 00110e3c f i stdafx.obj
 0001:0000ff04       ?_AtlRaiseException@ATL@@YAXKK@Z 00110f04 f i stdafx.obj
 0001:0000ff28       ??1?$CSimpleArray@GV?$CSimpleArrayEqualHelper@G@ATL@@@ATL@@QAA@XZ 00110f28 f i stdafx.obj
 0001:0000ff40       ??0SW_Log@@QAA@XZ          00110f40 f   SW_Log.obj
 0001:0000ff84       ??1SW_Log@@QAA@XZ          00110f84 f   SW_Log.obj
 0001:00010154       ?Init@SW_Log@@QAAXPAUHINSTANCE__@@@Z 00111154 f   SW_Log.obj
 0001:000101b0       ?InitObject@SW_Log@@IAAXXZ 001111b0 f   SW_Log.obj
 0001:000104ac       ?GetLogFileFromReg@SW_Log@@IAAJPAGAAK@Z 001114ac f   SW_Log.obj
 0001:00010550       ?Filename@SW_Log@@QAAPBGXZ 00111550 f   SW_Log.obj
 0001:00010578       ?GetMaxLogFileReg@SW_Log@@IAAJXZ 00111578 f   SW_Log.obj
 0001:0001062c       ?GetModuleFilter@SW_Log@@IAAJPAUHINSTANCE__@@@Z 0011162c f   SW_Log.obj
 0001:00010734       ?GetCompFilterFromReg@SW_Log@@IAAJAAKK@Z 00111734 f   SW_Log.obj
 0001:00010804       ?GetRetailDebugEnableFromReg@SW_Log@@IAAJPAK@Z 00111804 f   SW_Log.obj
 0001:000108b0       ?GetFilterFromReg@SW_Log@@IAAJAAK@Z 001118b0 f   SW_Log.obj
 0001:000109d4       ?WriteLog@SW_Log@@QAAXPAGHKPBGPAPAD@Z 001119d4 f   SW_Log.obj
 0001:00011020       ?EraseLog@SW_Log@@QAAXXZ   00112020 f   SW_Log.obj
 0001:00011064       ?IsFileASerialDevice@SW_Log@@QAAHXZ 00112064 f   SW_Log.obj
 0001:000110bc       ?SetupCOMChannel@SW_Log@@QAAXPAX@Z 001120bc f   SW_Log.obj
 0001:0001127c       ?SetFilter@SW_Log@@IAAXAAK@Z 0011227c f   SW_Log.obj
 0001:000112d4       ?GetDisplayMemFromReg@SW_Log@@AAAJPAK@Z 001122d4 f   SW_Log.obj
 0001:000113e8       ?DisplayLog@SW_Log@@QAAXPBGPAPAD@Z 001123e8 f   SW_Log.obj
 0001:00011488       ?LogThreadFunc@SW_Log@@CAXPAX@Z 00112488 f   SW_Log.obj
 0001:000114b8       ?Run@SW_Log@@IAAXXZ        001124b8 f   SW_Log.obj
 0001:00011788       ?LogWndProc@SW_Log@@CAJPAUHWND__@@IIJ@Z 00112788 f   SW_Log.obj
 0001:0001184c       ?SWSerialize@SW_Log@@IAAXPAXPBGK@Z 0011284c f   SW_Log.obj
 0001:00011da4       ?MessageBoxOnSeparateThread@SW_Log@@QAAXPBG@Z 00112da4 f   SW_Log.obj
 0001:00011e1c       ?MessageBoxFunction@SW_Log@@KAIPAX@Z 00112e1c f   SW_Log.obj
 0001:00011e60       ?wcsstr@@YAPAGPAGPBG@Z     00112e60 f i SW_Log.obj
 0001:00011e94       ?Filter@SW_Log@@QBA?BKXZ   00112e94 f i SW_Log.obj
 0001:00011ebc       ?Filter@SW_Log@@QAA?BKK@Z  00112ebc f i SW_Log.obj
 0001:00011f0c       ?MaxLogFileSize@SW_Log@@IAAKXZ 00112f0c f i SW_Log.obj
 0001:00011f38       ?InitLog@@YAXPAUHINSTANCE__@@@Z 00112f38 f   SW_Log_Include.obj
 0001:00011f68       ?WriteLog@@YAXPAVSW_Log@@KPBGPAPAD@Z 00112f68 f   SW_Log_Include.obj
 0001:00011fb0       ?DisplayLog@@YAXPAVSW_Log@@PBGPAPAD@Z 00112fb0 f   SW_Log_Include.obj
 0001:00011fd0       ?WriteLog@@YAXPAVSW_Log@@KPBGZZ 00112fd0 f   SW_Log_Include.obj
 0001:00012010       ?WriteLog@@YAXPAVSW_Log@@PBGZZ 00113010 f   SW_Log_Include.obj
 0001:0001205c       ?WriteLog@@YAXKPBGZZ       0011305c f   SW_Log_Include.obj
 0001:000120a0       ?WriteLog@@YAXPBGZZ        001130a0 f   SW_Log_Include.obj
 0001:000120f0       ?LogV@@YAXPBGZZ            001130f0 f   SW_Log_Include.obj
 0001:00012134       ?LogC@@YAXPBGZZ            00113134 f   SW_Log_Include.obj
 0001:00012178       ?LogW@@YAXPBGZZ            00113178 f   SW_Log_Include.obj
 0001:000121bc       ?LogWindowText@@YAXPBGZZ   001131bc f   SW_Log_Include.obj
 0001:000121fc       ?LogStoreFileLine@@YAXPAGH@Z 001131fc f   SW_Log_Include.obj
 0001:0001222c       ?GetAvailProgramMem@@YAKXZ 0011322c f   SW_Log_Include.obj
 0001:00012268       ?GetAvailStoreMem@@YAKXZ   00113268 f   SW_Log_Include.obj
 0001:00012298       ?GetAvailMem@@YAKXZ        00113298 f   SW_Log_Include.obj
 0001:000122c4       ?GetMemUsed@@YAKXZ         001132c4 f   SW_Log_Include.obj
 0001:000122f8       ?TBD_Assert@@YA_N_NQBG1H@Z 001132f8 f   SW_Log_Include.obj
 0001:00012350       ?TBD_Output@@YAXW4TBD_CLASS_TYPE@@W4TBD_OUTPUT_LEVEL@@QBGZZ 00113350 f   SW_Log_Include.obj
 0001:000123bc       ?DisplayRawData@@YAXIPAEHPBG@Z 001133bc f   SW_Log_Include.obj
 0001:00012678       ?GetRegValue@@YAJPAUHKEY__@@PBG1AAK@Z 00113678 f   SW_Registrykey.obj
 0001:0001283c       ?GetRegValue@@YAJPAUHKEY__@@PBG1PAGPAK@Z 0011383c f   SW_Registrykey.obj
 0001:00012a18       ?GetRegValue@@YAJPAUHKEY__@@PBG1PAEPAK@Z 00113a18 f   SW_Registrykey.obj
 0001:00012bbc       ?SetRegValue@@YAJPAUHKEY__@@PBG11@Z 00113bbc f   SW_Registrykey.obj
 0001:00012cc8       ?SetRegValue@@YAJPAUHKEY__@@PBG1QAEK@Z 00113cc8 f   SW_Registrykey.obj
 0001:00012dd8       ?SetRegValue@@YAJPAUHKEY__@@PBG1K@Z 00113dd8 f   SW_Registrykey.obj
 0001:00012ee4       ?SWAI_GetRegValue@@YAJPAUHKEY__@@PBG1AAK@Z 00113ee4 f   SW_Registrykey.obj
 0001:00013144       ?SWAI_GetRegValue@@YAJPAUHKEY__@@PBG1PAGPAK@Z 00114144 f   SW_Registrykey.obj
 0001:000133f8       ?SWAI_GetRegValue@@YAJPAUHKEY__@@PBG1PAEPAK@Z 001143f8 f   SW_Registrykey.obj
 0001:00013678       ?SWAI_SetRegValue@@YAJPAUHKEY__@@PBG11@Z 00114678 f   SW_Registrykey.obj
 0001:00013808       ?SWAI_SetRegValue@@YAJPAUHKEY__@@PBG1QAEK@Z 00114808 f   SW_Registrykey.obj
 0001:0001399c       ?SWAI_SetRegValue@@YAJPAUHKEY__@@PBG1K@Z 0011499c f   SW_Registrykey.obj
 0001:00013b2c       ?CopyRegKey@@YAJPAUHKEY__@@PBG11H@Z 00114b2c f   SW_Registrykey.obj
 0001:00013f10       ?DeleteRegKey@@YAJPAUHKEY__@@PBG1H@Z 00114f10 f   SW_Registrykey.obj
 0001:000141a8       ?RenameRegKey@@YAJPAUHKEY__@@PBG11H@Z 001151a8 f   SW_Registrykey.obj
 0001:000145a0       ?DeleteSubKey@SW_RegistryKey@@IAAJPBG@Z 001155a0 f   SW_Registrykey.obj
 0001:00014608       ?RecurseDeleteKey@SW_RegistryKey@@QAAJPBG@Z 00115608 f   SW_Registrykey.obj
 0001:00014798       ??0SW_RegistryKey@@QAA@XZ  00115798 f   SW_Registrykey.obj
 0001:000147d4       ??0SW_RegistryKey@@QAA@PAUHKEY__@@@Z 001157d4 f   SW_Registrykey.obj
 0001:00014838       ??1SW_RegistryKey@@QAA@XZ  00115838 f   SW_Registrykey.obj
 0001:000148c0       ?InitObject@SW_RegistryKey@@MAAXXZ 001158c0 f   SW_Registrykey.obj
 0001:000148e8       ?CreateKey@SW_RegistryKey@@UAAJPAUHKEY__@@PBGKPAK@Z 001158e8 f   SW_Registrykey.obj
 0001:00014c10       ?CreateKey@SW_RegistryKey@@UAAJPBGKPAK@Z 00115c10 f   SW_Registrykey.obj
 0001:00014cb8       ?OpenKey@SW_RegistryKey@@UAAJPBGK@Z 00115cb8 f   SW_Registrykey.obj
 0001:00014d58       ?OpenKey@SW_RegistryKey@@UAAJPAUHKEY__@@PBGK@Z 00115d58 f   SW_Registrykey.obj
 0001:00014de4       ?CloseKey@SW_RegistryKey@@UAAJXZ 00115de4 f   SW_Registrykey.obj
 0001:00014e90       ?QueryValue@SW_RegistryKey@@UAAJPBGPAPAG@Z 00115e90 f   SW_Registrykey.obj
 0001:00015118       ?QueryValue@SW_RegistryKey@@UAAJPBGPAK@Z 00116118 f   SW_Registrykey.obj
 0001:0001523c       ?QueryValue@SW_RegistryKey@@UAAJPBGPAPAEPAK@Z 0011623c f   SW_Registrykey.obj
 0001:0001547c       ?SetValue@SW_RegistryKey@@UAAJPBG0@Z 0011647c f   SW_Registrykey.obj
 0001:00015520       ?SetValue@SW_RegistryKey@@UAAJPBGK@Z 00116520 f   SW_Registrykey.obj
 0001:00015590       ?SetValue@SW_RegistryKey@@UAAJPBGQAEK@Z 00116590 f   SW_Registrykey.obj
 0001:00015614       ?EnumKey@SW_RegistryKey@@IAAJAAKPAG@Z 00116614 f   SW_Registrykey.obj
 0001:000156b0       ?Duplicate@SW_RegistryKey@@QAAHAAV1@@Z 001166b0 f   SW_Registrykey.obj
 0001:00015ac0       ?wcschr@@YAPAGPAGG@Z       00116ac0 f i SW_Registrykey.obj
 0001:00015afc       ?GetVerInfo@@YAPAGPAUHINSTANCE__@@@Z 00116afc f   Utilities.obj
 0001:00015c88       ?GetOSVersioninfo@@YAXXZ   00116c88 f   Utilities.obj
 0001:00015d30       ?GetDataPortDetails@@YAHPAGAAK@Z 00116d30 f   Utilities.obj
 0001:00015e48       ?ChangeCarrierIndex@@YAJKK@Z 00116e48 f   Utilities.obj
 0001:000162a4       ?GetCarrierIndex@@YAKXZ    001172a4 f   Utilities.obj
 0001:00016560       ?GetAutoUpdateTimeUI@@YAKXZ 00117560 f   Utilities.obj
 0001:000165c8       ?GetAutoUpdateTime@@YAKXZ  001175c8 f   Utilities.obj
 0001:00016630       ?GetCallGuardReg@@YAKXZ    00117630 f   Utilities.obj
 0001:00016698       ?SetAutoUpdateTime@@YAXH@Z 00117698 f   Utilities.obj
 0001:000166e8       ?SetAutoUpdateTimeUI@@YAXK@Z 001176e8 f   Utilities.obj
 0001:00016738       ?SetCallGuardReg@@YAXK@Z   00117738 f   Utilities.obj
 0001:00016788       ?GetActWizDisabled@@YAKXZ  00117788 f   Utilities.obj
 0001:000167dc       ?SetActWizDisabled@@YAXK@Z 001177dc f   Utilities.obj
 0001:0001682c       ?GetMdnLen@@YAHAAK@Z       0011782c f   Utilities.obj
 0001:000168c0       ?IsConsumerProduct@@YAHXZ  001178c0 f   Utilities.obj
 0001:00016930       ?GetLogoTestReg@@YAKXZ     00117930 f   Utilities.obj
 0001:000169a8       ?EnableCarrierLogo@@YAXH@Z 001179a8 f   Utilities.obj
 0001:00016a48       ?EncodeMCC1112@@YAHPBG_N@Z 00117a48 f   Utilities.obj
 0001:00016b38       ?EncodePhoneNumber@@YA_NPAGPAK@Z 00117b38 f   Utilities.obj
 0001:00016f5c       ?DecodeMCC1112@@YAHH_N@Z   00117f5c f   Utilities.obj
 0001:000170d4       ?DecodeAreaCode@@YA_NPAGG@Z 001180d4 f   Utilities.obj
 0001:00017290       ?DecodePhoneNumber@@YA_NPAGK@Z 00118290 f   Utilities.obj
 0001:000175c8       ?SW_AtoT@@YAPAGPAGPADK@Z   001185c8 f   Utilities.obj
 0001:00017630       ?SW_TtoA@@YAPADPADPAGK@Z   00118630 f   Utilities.obj
 0001:00017690       ?GetProductFeatures@@YAHAAK@Z 00118690 f   Utilities.obj
 0001:00017708       ?RelayoutDialog@@YAHPAUHINSTANCE__@@PAUHWND__@@PBG@Z 00118708 f   Utilities.obj
 0001:00017d3c       ?InWideMode@@YAHXZ         00118d3c f   Utilities.obj
 0001:00017e0c       ?SetLimitText@@YAJPAUHWND__@@H@Z 00118e0c f   Utilities.obj
 0001:00017e50       ?GetResolution@@YAHXZ      00118e50 f   Utilities.obj
 0001:00017ee8       ?SetConnectionProfile@@YAJXZ 00118ee8 f   Utilities.obj
 0001:00018868       ?EnableLocationReg@@YAJXZ  00119868 f   Utilities.obj
 0001:000189f0       ?SetLocationResourceBaseID@@YAJK@Z 001199f0 f   Utilities.obj
 0001:00018d14       ?SetSpecialNumber@@YAJPAG@Z 00119d14 f   Utilities.obj
 0001:00018e2c       ?GetSpecialNumber@@YAJPAG@Z 00119e2c f   Utilities.obj
 0001:00018f7c       ?SetNormalCursor@@YAXXZ    00119f7c f   Utilities.obj
 0001:00018fa4       ?SetWaitCursor@@YAXXZ      00119fa4 f   Utilities.obj
 0001:00019008       ?ConvertPrefMode@@YAH_NH@Z 0011a008 f   Utilities.obj
 0001:00019190       ?BtoH@@YAED@Z              0011a190 f   Utilities.obj
 0001:00019240       ?HtoB@@YADE@Z              0011a240 f   Utilities.obj
 0001:000192b0       ?TtoTH@@YAXPAG0H@Z         0011a2b0 f   Utilities.obj
 0001:00019430       ?THtoT@@YAXPAG0H@Z         0011a430 f   Utilities.obj
 0001:000195a0       ?LocalToUTCTime@@YAHPAU_SYSTEMTIME@@0@Z 0011a5a0 f   Utilities.obj
 0001:00019650       ?DWORD2IP@@YAPBGK@Z        0011a650 f   Utilities.obj
 0001:00019734       ?IP2DWORD@@YAKPBG@Z        0011a734 f   Utilities.obj
 0001:0001999c       LockResource               0011a99c f i Utilities.obj
 0001:000199c0       memcpy                     0011a9c0 f   coredll:COREDLL.dll
 0001:000199d0       GetModuleFileNameW         0011a9d0 f   coredll:COREDLL.dll
 0001:000199e0       ??3@YAXPAX@Z               0011a9e0 f   coredll:COREDLL.dll
 0001:000199f0       GetFileVersionInfoW        0011a9f0 f   coredll:COREDLL.dll
 0001:00019a00       ??2@YAPAXI@Z               0011aa00 f   coredll:COREDLL.dll
 0001:00019a10       GetFileVersionInfoSizeW    0011aa10 f   coredll:COREDLL.dll
 0001:00019a20       wcscpy                     0011aa20 f   coredll:COREDLL.dll
 0001:00019a30       OutputDebugStringW         0011aa30 f   coredll:COREDLL.dll
 0001:00019a40       swprintf                   0011aa40 f   coredll:COREDLL.dll
 0001:00019a50       VerQueryValueW             0011aa50 f   coredll:COREDLL.dll
 0001:00019a60       wcscat                     0011aa60 f   coredll:COREDLL.dll
 0001:00019a70       CreateEventW               0011aa70 f   coredll:COREDLL.dll
 0001:00019a80       RegisterWindowMessageW     0011aa80 f   coredll:COREDLL.dll
 0001:00019a90       CloseHandle                0011aa90 f   coredll:COREDLL.dll
 0001:00019aa0       WaitForSingleObject        0011aaa0 f   coredll:COREDLL.dll
 0001:00019ab0       CreateThread               0011aab0 f   coredll:COREDLL.dll
 0001:00019ac0       EventModify                0011aac0 f   coredll:COREDLL.dll
 0001:00019ad0       PostMessageW               0011aad0 f   coredll:COREDLL.dll
 0001:00019ae0       __rt_udiv                  0011aae0 f   coredll:COREDLL.dll
 0001:00019af0       wsprintfW                  0011aaf0 f   coredll:COREDLL.dll
 0001:00019b00       EnterCriticalSection       0011ab00 f   coredll:COREDLL.dll
 0001:00019b10       LeaveCriticalSection       0011ab10 f   coredll:COREDLL.dll
 0001:00019b20       wcslen                     0011ab20 f   coredll:COREDLL.dll
 0001:00019b30       strcpy                     0011ab30 f   coredll:COREDLL.dll
 0001:00019b40       memset                     0011ab40 f   coredll:COREDLL.dll
 0001:00019b50       wcsncpy                    0011ab50 f   coredll:COREDLL.dll
 0001:00019b60       strlen                     0011ab60 f   coredll:COREDLL.dll
 0001:00019b70       InitializeCriticalSection  0011ab70 f   coredll:COREDLL.dll
 0001:00019b80       DeleteCriticalSection      0011ab80 f   coredll:COREDLL.dll
 0001:00019b90       UnregisterClassW           0011ab90 f   coredll:COREDLL.dll
 0001:00019ba0       free                       0011aba0 f   coredll:COREDLL.dll
 0001:00019bb0       RaiseException             0011abb0 f   coredll:COREDLL.dll
 0001:00019bc0       CloseMsgQueue              0011abc0 f   coredll:COREDLL.dll
 0001:00019bd0       TerminateThread            0011abd0 f   coredll:COREDLL.dll
 0001:00019be0       WriteMsgQueue              0011abe0 f   coredll:COREDLL.dll
 0001:00019bf0       CreateMsgQueue             0011abf0 f   coredll:COREDLL.dll
 0001:00019c00       Sleep                      0011ac00 f   coredll:COREDLL.dll
 0001:00019c10       ReleaseMutex               0011ac10 f   coredll:COREDLL.dll
 0001:00019c20       GetLastError               0011ac20 f   coredll:COREDLL.dll
 0001:00019c30       CreateMutexW               0011ac30 f   coredll:COREDLL.dll
 0001:00019c40       _wcslwr                    0011ac40 f   coredll:COREDLL.dll
 0001:00019c50       wcscmp                     0011ac50 f   coredll:COREDLL.dll
 0001:00019c60       GetLocalTime               0011ac60 f   coredll:COREDLL.dll
 0001:00019c70       NKDbgPrintfW               0011ac70 f   coredll:COREDLL.dll
 0001:00019c80       vswprintf                  0011ac80 f   coredll:COREDLL.dll
 0001:00019c90       DeleteFileW                0011ac90 f   coredll:COREDLL.dll
 0001:00019ca0       PurgeComm                  0011aca0 f   coredll:COREDLL.dll
 0001:00019cb0       SetCommMask                0011acb0 f   coredll:COREDLL.dll
 0001:00019cc0       SetCommTimeouts            0011acc0 f   coredll:COREDLL.dll
 0001:00019cd0       SetCommState               0011acd0 f   coredll:COREDLL.dll
 0001:00019ce0       GetCommState               0011ace0 f   coredll:COREDLL.dll
 0001:00019cf0       ReadMsgQueue               0011acf0 f   coredll:COREDLL.dll
 0001:00019d00       SetFilePointer             0011ad00 f   coredll:COREDLL.dll
 0001:00019d10       CreateFileW                0011ad10 f   coredll:COREDLL.dll
 0001:00019d20       DefWindowProcW             0011ad20 f   coredll:COREDLL.dll
 0001:00019d30       PostQuitMessage            0011ad30 f   coredll:COREDLL.dll
 0001:00019d40       FlushFileBuffers           0011ad40 f   coredll:COREDLL.dll
 0001:00019d50       WriteFile                  0011ad50 f   coredll:COREDLL.dll
 0001:00019d60       CopyFileW                  0011ad60 f   coredll:COREDLL.dll
 0001:00019d70       GetFileSize                0011ad70 f   coredll:COREDLL.dll
 0001:00019d80       MessageBoxW                0011ad80 f   coredll:COREDLL.dll
 0001:00019d90       wcsstr                     0011ad90 f   coredll:COREDLL.dll
 0001:00019da0       GlobalMemoryStatus         0011ada0 f   coredll:COREDLL.dll
 0001:00019db0       GetStoreInformation        0011adb0 f   coredll:COREDLL.dll
 0001:00019dc0       MessageBeep                0011adc0 f   coredll:COREDLL.dll
 0001:00019dd0       rand                       0011add0 f   coredll:COREDLL.dll
 0001:00019de0       RegDeleteKeyW              0011ade0 f   coredll:COREDLL.dll
 0001:00019df0       RegEnumKeyExW              0011adf0 f   coredll:COREDLL.dll
 0001:00019e00       RegCloseKey                0011ae00 f   coredll:COREDLL.dll
 0001:00019e10       RegCreateKeyExW            0011ae10 f   coredll:COREDLL.dll
 0001:00019e20       RegOpenKeyExW              0011ae20 f   coredll:COREDLL.dll
 0001:00019e30       RegQueryValueExW           0011ae30 f   coredll:COREDLL.dll
 0001:00019e40       RegSetValueExW             0011ae40 f   coredll:COREDLL.dll
 0001:00019e50       RegEnumValueW              0011ae50 f   coredll:COREDLL.dll
 0001:00019e60       wcschr                     0011ae60 f   coredll:COREDLL.dll
 0001:00019e70       GetVersionExW              0011ae70 f   coredll:COREDLL.dll
 0001:00019e80       _wcsicmp                   0011ae80 f   coredll:COREDLL.dll
 0001:00019e90       _wtol                      0011ae90 f   coredll:COREDLL.dll
 0001:00019ea0       __rt_sdiv                  0011aea0 f   coredll:COREDLL.dll
 0001:00019eb0       mbstowcs                   0011aeb0 f   coredll:COREDLL.dll
 0001:00019ec0       wcstombs                   0011aec0 f   coredll:COREDLL.dll
 0001:00019ed0       EndDeferWindowPos          0011aed0 f   coredll:COREDLL.dll
 0001:00019ee0       DeferWindowPos             0011aee0 f   coredll:COREDLL.dll
 0001:00019ef0       MapDialogRect              0011aef0 f   coredll:COREDLL.dll
 0001:00019f00       GetDlgItem                 0011af00 f   coredll:COREDLL.dll
 0001:00019f10       BeginDeferWindowPos        0011af10 f   coredll:COREDLL.dll
 0001:00019f20       LoadResource               0011af20 f   coredll:COREDLL.dll
 0001:00019f30       FindResourceW              0011af30 f   coredll:COREDLL.dll
 0001:00019f40       SetDlgItemTextW            0011af40 f   coredll:COREDLL.dll
 0001:00019f50       DeleteObject               0011af50 f   coredll:COREDLL.dll
 0001:00019f60       LoadBitmapW                0011af60 f   coredll:COREDLL.dll
 0001:00019f70       DestroyIcon                0011af70 f   coredll:COREDLL.dll
 0001:00019f80       LoadIconW                  0011af80 f   coredll:COREDLL.dll
 0001:00019f90       SendDlgItemMessageW        0011af90 f   coredll:COREDLL.dll
 0001:00019fa0       GetSystemMetrics           0011afa0 f   coredll:COREDLL.dll
 0001:00019fb0       SendMessageW               0011afb0 f   coredll:COREDLL.dll
 0001:00019fc0       FreeLibrary                0011afc0 f   coredll:COREDLL.dll
 0001:00019fd0       GetProcAddressW            0011afd0 f   coredll:COREDLL.dll
 0001:00019fe0       LoadLibraryW               0011afe0 f   coredll:COREDLL.dll
 0001:00019ff0       RegDeleteValueW            0011aff0 f   coredll:COREDLL.dll
 0001:0001a000       SetCursor                  0011b000 f   coredll:COREDLL.dll
 0001:0001a010       LoadCursorW                0011b010 f   coredll:COREDLL.dll
 0001:0001a020       FileTimeToSystemTime       0011b020 f   coredll:COREDLL.dll
 0001:0001a030       LocalFileTimeToFileTime    0011b030 f   coredll:COREDLL.dll
 0001:0001a040       SystemTimeToFileTime       0011b040 f   coredll:COREDLL.dll
 0001:0001a050       RIL_Initialize             0011b050 f   ril:ril.dll
 0001:0001a060       RIL_Deinitialize           0011b060 f   ril:ril.dll
 0001:0001a070       RIL_DevSpecific            0011b070 f   ril:ril.dll
 0001:0001a080       RIL_GetEquipmentState      0011b080 f   ril:ril.dll
 0001:0001a090       RIL_GetEquipmentInfo       0011b090 f   ril:ril.dll
 0001:0001a0a0       RIL_GetUserIdentity        0011b0a0 f   ril:ril.dll
 0001:0001a0b0       RIL_SetEquipmentState      0011b0b0 f   ril:ril.dll
 0001:0001a0c0       RIL_Hangup                 0011b0c0 f   ril:ril.dll
 0001:0001a0d0       RIL_Dial                   0011b0d0 f   ril:ril.dll
 0001:0001a0e0       RIL_GetRegistrationStatus  0011b0e0 f   ril:ril.dll
 0001:0001a0f0       RIL_GetCurrentSystemType   0011b0f0 f   ril:ril.dll
 0001:0001a100       RIL_GetCallList            0011b100 f   ril:ril.dll
 0001:0001a110       RIL_GetPreferredPrivacyMode 0011b110 f   ril:ril.dll
 0001:0001a120       RIL_GetRoamingMode         0011b120 f   ril:ril.dll
 0001:0001a130       RIL_SetRoamingMode         0011b130 f   ril:ril.dll
 0001:0001a140       RIL_SetPreferredPrivacyMode 0011b140 f   ril:ril.dll
 0001:0001a150       RIL_SendAKey               0011b150 f   ril:ril.dll
 0001:0001a160       RIL_GetPacketByteCount     0011b160 f   ril:ril.dll
 0001:0001a170       ntohl                      0011b170 f   ws2:WS2.dll
 0001:0001a180       _DllMainCRTStartup         0011b180 f   corelibc:pegdmain.obj
 0001:0001a218       __security_check_cookie    0011b218     corelibc:armsecgs.obj
 0001:0001a22c       __gsfailure                0011b22c     corelibc:armsecgs.obj
 0001:0001a270       _onexit                    0011b270 f   corelibc:onexit.obj
 0001:0001a31c       atexit                     0011b31c f   corelibc:onexit.obj
 0001:0001a33c       GetCurrentProcess          0011b33c f i corelibc:crt0dat.obj
 0001:0001a378       _cinit                     0011b378 f   corelibc:crt0dat.obj
 0001:0001a4e8       exit                       0011b4e8 f   corelibc:crt0dat.obj
 0001:0001a500       _exit                      0011b500 f   corelibc:crt0dat.obj
 0001:0001a518       _cexit                     0011b518 f   corelibc:crt0dat.obj
 0001:0001a534       _c_exit                    0011b534 f   corelibc:crt0dat.obj
 0001:0001a580       DllMain                    0011b580 f   corelibc:dllmain.obj
 0001:0001a598       __security_init_cookie     0011b598 f   corelibc:seccinit.obj
 0001:0001a5e8       ?AtlAdvise@ATL@@YAJPAUIUnknown@@0ABU_GUID@@PAK@Z 0011b5e8 f   atlsd:atlfuncs.obj
 0001:0001a7a4       ?AtlUnadvise@ATL@@YAJPAUIUnknown@@ABU_GUID@@K@Z 0011b7a4 f   atlsd:atlfuncs.obj
 0001:0001a95c       ?AtlFreeMarshalStream@ATL@@YAJPAUIStream@@@Z 0011b95c f   atlsd:atlfuncs.obj
 0001:0001aa14       ?AtlMarshalPtrInProc@ATL@@YAJPAUIUnknown@@ABU_GUID@@PAPAUIStream@@@Z 0011ba14 f   atlsd:atlfuncs.obj
 0001:0001ab58       ?AtlUnmarshalPtr@ATL@@YAJPAUIStream@@ABU_GUID@@PAPAUIUnknown@@@Z 0011bb58 f   atlsd:atlfuncs.obj
 0001:0001ac78       ?AtlComModuleGetClassObject@ATL@@YAJPAU_ATL_COM_MODULE70@1@ABU_GUID@@1PAPAX@Z 0011bc78 f   atlsd:atlfuncs.obj
 0001:0001aff0       ?AtlComModuleRegisterClassObjects@ATL@@YAJPAU_ATL_COM_MODULE70@1@KK@Z 0011bff0 f   atlsd:atlfuncs.obj
 0001:0001b110       ?AtlComModuleRevokeClassObjects@ATL@@YAJPAU_ATL_COM_MODULE70@1@@Z 0011c110 f   atlsd:atlfuncs.obj
 0001:0001b228       ?AtlWaitWithMessageLoop@ATL@@YAHPAX@Z 0011c228 f   atlsd:atlfuncs.obj
 0001:0001b3c0       ?AtlInternalQueryInterface@ATL@@YAJPAXPBU_ATL_INTMAP_ENTRY@1@ABU_GUID@@PAPAX@Z 0011c3c0 f   atlsd:atlfuncs.obj
 0001:0001b748       ?AtlGetVersion@ATL@@YAKPAX@Z 0011c748 f   atlsd:atlfuncs.obj
 0001:0001b770       ?AtlWinModuleAddCreateWndData@ATL@@YAXPAU_ATL_WIN_MODULE70@1@PAU_AtlCreateWndData@1@PAX@Z 0011c770 f   atlsd:atlfuncs.obj
 0001:0001b9ac       ?AtlWinModuleExtractCreateWndData@ATL@@YAPAXPAU_ATL_WIN_MODULE70@1@@Z 0011c9ac f   atlsd:atlfuncs.obj
 0001:0001bbf8       ?AtlWinModuleInit@ATL@@YAJPAU_ATL_WIN_MODULE70@1@@Z 0011cbf8 f   atlsd:atlfuncs.obj
 0001:0001bd48       ?AtlModuleAddTermFunc@ATL@@YAJPAU_ATL_MODULE70@1@P6AXK@ZK@Z 0011cd48 f   atlsd:atlfuncs.obj
 0001:0001bf54       ?AtlCallTermFunc@ATL@@YAXPAU_ATL_MODULE70@1@@Z 0011cf54 f   atlsd:atlfuncs.obj
 0001:0001c01c       ??1?$CComPtr@UIConnectionPointContainer@@@ATL@@QAA@XZ 0011d01c f i atlsd:atlfuncs.obj
 0001:0001c044       ??1?$CComPtr@UIConnectionPoint@@@ATL@@QAA@XZ 0011d044 f i atlsd:atlfuncs.obj
 0001:0001c06c       GetCurrentThreadId         0011d06c f i atlsd:atlfuncs.obj
 0001:0001c08c       ?IsWindowUnicode@ATL@@YAHPAUHWND__@@@Z 0011d08c f i atlsd:atlfuncs.obj
 0001:0001c0b4       ??0?$CComPtr@UIConnectionPointContainer@@@ATL@@QAA@XZ 0011d0b4 f i atlsd:atlfuncs.obj
 0001:0001c0f4       ??1?$CComPtrBase@UIConnectionPointContainer@@@ATL@@QAA@XZ 0011d0f4 f i atlsd:atlfuncs.obj
 0001:0001c13c       ??I?$CComPtrBase@UIConnectionPointContainer@@@ATL@@QAAPAPAUIConnectionPointContainer@@XZ 0011d13c f i atlsd:atlfuncs.obj
 0001:0001c1b8       ??C?$CComPtrBase@UIConnectionPointContainer@@@ATL@@QBAPAV?$_NoAddRefReleaseOnCComPtr@UIConnectionPointContainer@@@1@XZ 0011d1b8 f i atlsd:atlfuncs.obj
 0001:0001c238       ??0?$CComPtr@UIConnectionPoint@@@ATL@@QAA@XZ 0011d238 f i atlsd:atlfuncs.obj
 0001:0001c278       ??1?$CComPtrBase@UIConnectionPoint@@@ATL@@QAA@XZ 0011d278 f i atlsd:atlfuncs.obj
 0001:0001c2c0       ??I?$CComPtrBase@UIConnectionPoint@@@ATL@@QAAPAPAUIConnectionPoint@@XZ 0011d2c0 f i atlsd:atlfuncs.obj
 0001:0001c33c       ??C?$CComPtrBase@UIConnectionPoint@@@ATL@@QBAPAV?$_NoAddRefReleaseOnCComPtr@UIConnectionPoint@@@1@XZ 0011d33c f i atlsd:atlfuncs.obj
 0001:0001c3bc       ??0?$CComPtrBase@UIConnectionPointContainer@@@ATL@@IAA@XZ 0011d3bc f i atlsd:atlfuncs.obj
 0001:0001c3f0       ??0?$CComPtrBase@UIConnectionPoint@@@ATL@@IAA@XZ 0011d3f0 f i atlsd:atlfuncs.obj
 0001:0001c424       ?InlineIsEqualGUID@ATL@@YAHABU_GUID@@0@Z 0011d424 f i atlsd:atlfuncs.obj
 0001:0001c4d8       ??0CTraceFileAndLineInfo@ATL@@QAA@PBDH@Z 0011d4d8 f i atlsd:atlfuncs.obj
 0001:0001c51c       ??RCTraceFileAndLineInfo@ATL@@QBAXKIPB_WZZ 0011d51c f i atlsd:atlfuncs.obj
 0001:0001c594       ?TraceV@CTrace@ATL@@QBAXPBDHKIPB_WPAD@Z 0011d594 f i atlsd:atlfuncs.obj
 0001:0001c5f0       ??BCTraceCategory@ATL@@QBAKXZ 0011d5f0 f i atlsd:atlfuncs.obj
 0001:0001c624       ?Init@CComCriticalSection@ATL@@QAAJXZ 0011d624 f i atlsd:atlfuncs.obj
 0001:0001c6c8       ?RevokeClassObject@_ATL_OBJMAP_ENTRY30@ATL@@QAAJXZ 0011d6c8 f i atlsd:atlfuncs.obj
 0001:0001c730       ?RegisterClassObject@_ATL_OBJMAP_ENTRY30@ATL@@QAAJKK@Z 0011d730 f i atlsd:atlfuncs.obj
 0001:0001c828       ?InlineIsEqualUnknown@ATL@@YAHABU_GUID@@@Z 0011d828 f i atlsd:atlfuncs.obj
 0001:0001c8b0       ??0?$CComCritSecLock@VCComCriticalSection@ATL@@@ATL@@QAA@AAVCComCriticalSection@1@_N@Z 0011d8b0 f i atlsd:atlfuncs.obj
 0001:0001c940       ?AtlThrowImpl@ATL@@YAXJ@Z  0011d940 f i atlsd:atlfuncs.obj
 0001:0001ca50       ??1?$CComCritSecLock@VCComCriticalSection@ATL@@@ATL@@QAA@XZ 0011da50 f i atlsd:atlfuncs.obj
 0001:0001ca8c       ?Unlock@?$CComCritSecLock@VCComCriticalSection@ATL@@@ATL@@QAAXXZ 0011da8c f i atlsd:atlfuncs.obj
 0001:0001cb2c       ?Unlock@CComCriticalSection@ATL@@QAAJXZ 0011db2c f i atlsd:atlfuncs.obj
 0001:0001cb68       ?Lock@?$CComCritSecLock@VCComCriticalSection@ATL@@@ATL@@QAAJXZ 0011db68 f i atlsd:atlfuncs.obj
 0001:0001cc38       ?Lock@CComCriticalSection@ATL@@QAAJXZ 0011dc38 f i atlsd:atlfuncs.obj
 0001:0001cc74       AtlRawDllMain              0011dc74 f   atlsd:atlbase.obj
 0001:0001cd74       ?CoDisconnectObject@ATL@@YAJPAUIUnknown@@K@Z 0011dd74 f   atlsd:atlbase.obj
 0001:0001cec8       ?CoInitialize@ATL@@YAJPAX@Z 0011dec8 f   atlsd:atlbase.obj
 0001:0001cf7c       ?CoRevokeClassObject@ATL@@YAJK@Z 0011df7c f   atlsd:atlbase.obj
 0001:0001d030       ?CoRegisterClassObject@ATL@@YAJABU_GUID@@PAUIUnknown@@KKPAK@Z 0011e030 f   atlsd:atlbase.obj
 0001:0001d0f8       ?CoMarshalInterface@ATL@@YAJPAUIStream@@ABU_GUID@@PAUIUnknown@@KPAXK@Z 0011e0f8 f   atlsd:atlbase.obj
 0001:0001d1c8       ?CoUnmarshalInterface@ATL@@YAJPAUIStream@@ABU_GUID@@PAPAX@Z 0011e1c8 f   atlsd:atlbase.obj
 0001:0001d284       ?CoReleaseMarshalData@ATL@@YAJPAUIStream@@@Z 0011e284 f   atlsd:atlbase.obj
 0001:0001d338       ?OleSaveToStream@ATL@@YAJPAUIPersistStream@@PAUIStream@@@Z 0011e338 f   atlsd:atlbase.obj
 0001:0001d4f0       ?OleLoadFromStream@ATL@@YAJPAUIStream@@ABU_GUID@@PAPAX@Z 0011e4f0 f   atlsd:atlbase.obj
 0001:0001d81c       ??0CAtlBaseModule@ATL@@QAA@XZ 0011e81c f   atlsd:atlbase.obj
 0001:0001d9a8       ??1CAtlBaseModule@ATL@@QAA@XZ 0011e9a8 f   atlsd:atlbase.obj
 0001:0001d9e8       ?AddResourceInstance@CAtlBaseModule@ATL@@QAA_NPAUHINSTANCE__@@@Z 0011e9e8 f   atlsd:atlbase.obj
 0001:0001db84       ?RemoveResourceInstance@CAtlBaseModule@ATL@@QAA_NPAUHINSTANCE__@@@Z 0011eb84 f   atlsd:atlbase.obj
 0001:0001dd98       ?GetHInstanceAt@CAtlBaseModule@ATL@@QAAPAUHINSTANCE__@@H@Z 0011ed98 f   atlsd:atlbase.obj
 0001:0001dfcc       ??0_ATL_BASE_MODULE70@ATL@@QAA@XZ 0011efcc f i atlsd:atlbase.obj
 0001:0001e02c       ??1_ATL_BASE_MODULE70@ATL@@QAA@XZ 0011f02c f i atlsd:atlbase.obj
 0001:0001e070       ?_AtlGetThisModuleHandle@ATL@@YAPAUHINSTANCE__@@XZ 0011f070 f i atlsd:atlbase.obj
 0001:0001e0d0       ??0?$CSimpleArray@PAUHINSTANCE__@@V?$CSimpleArrayEqualHelper@PAUHINSTANCE__@@@ATL@@@ATL@@QAA@XZ 0011f0d0 f i atlsd:atlbase.obj
 0001:0001e124       ?GetSize@?$CSimpleArray@PAUHINSTANCE__@@V?$CSimpleArrayEqualHelper@PAUHINSTANCE__@@@ATL@@@ATL@@QBAHXZ 0011f124 f i atlsd:atlbase.obj
 0001:0001e154       ?Add@?$CSimpleArray@PAUHINSTANCE__@@V?$CSimpleArrayEqualHelper@PAUHINSTANCE__@@@ATL@@@ATL@@QAAHABQAUHINSTANCE__@@@Z 0011f154 f i atlsd:atlbase.obj
 0001:0001e2a4       ?RemoveAt@?$CSimpleArray@PAUHINSTANCE__@@V?$CSimpleArrayEqualHelper@PAUHINSTANCE__@@@ATL@@@ATL@@QAAHH@Z 0011f2a4 f i atlsd:atlbase.obj
 0001:0001e41c       ??A?$CSimpleArray@PAUHINSTANCE__@@V?$CSimpleArrayEqualHelper@PAUHINSTANCE__@@@ATL@@@ATL@@QAAAAPAUHINSTANCE__@@H@Z 0011f41c f i atlsd:atlbase.obj
 0001:0001e500       ?InternalSetAtIndex@?$CSimpleArray@PAUHINSTANCE__@@V?$CSimpleArrayEqualHelper@PAUHINSTANCE__@@@ATL@@@ATL@@QAAXHABQAUHINSTANCE__@@@Z 0011f500 f i atlsd:atlbase.obj
 0001:0001e590       ??0Wrapper@?$CSimpleArray@PAUHINSTANCE__@@V?$CSimpleArrayEqualHelper@PAUHINSTANCE__@@@ATL@@@ATL@@QAA@ABQAUHINSTANCE__@@@Z 0011f590 f i atlsd:atlbase.obj
 0001:0001e5c8       ??1?$CSimpleArray@PAUHINSTANCE__@@V?$CSimpleArrayEqualHelper@PAUHINSTANCE__@@@ATL@@@ATL@@QAA@XZ 0011f5c8 f i atlsd:atlbase.obj
 0001:0001e5f0       ??$?2PAUHINSTANCE__@@@Wrapper@?$CSimpleArray@PAUHINSTANCE__@@V?$CSimpleArrayEqualHelper@PAUHINSTANCE__@@@ATL@@@ATL@@SAPAXIPAPAUHINSTANCE__@@@Z 0011f5f0 f i atlsd:atlbase.obj
 0001:0001e618       ?RemoveAll@?$CSimpleArray@PAUHINSTANCE__@@V?$CSimpleArrayEqualHelper@PAUHINSTANCE__@@@ATL@@@ATL@@QAAXXZ 0011f618 f i atlsd:atlbase.obj
 0001:0001e6bc       ?memmove_s@Checked@ATL@@YAXPAXIPBXI@Z 0011f6bc f i atlsd:atlbase.obj
 0001:0001e710       ?AtlCrtErrorCheck@ATL@@YAHH@Z 0011f710 f i atlsd:atlbase.obj
 0001:0001e7dc       ??1?$CComPtr@UIUnknown@@@ATL@@QAA@XZ 0011f7dc f i atlsd:atlbase.obj
 0001:0001e804       ??1?$CComPtr@UIPersistStream@@@ATL@@QAA@XZ 0011f804 f i atlsd:atlbase.obj
 0001:0001e82c       ??0?$CComPtr@UIUnknown@@@ATL@@QAA@XZ 0011f82c f i atlsd:atlbase.obj
 0001:0001e86c       ??1?$CComPtrBase@UIUnknown@@@ATL@@QAA@XZ 0011f86c f i atlsd:atlbase.obj
 0001:0001e8b4       ??I?$CComPtrBase@UIUnknown@@@ATL@@QAAPAPAUIUnknown@@XZ 0011f8b4 f i atlsd:atlbase.obj
 0001:0001e930       ??C?$CComPtrBase@UIUnknown@@@ATL@@QBAPAV?$_NoAddRefReleaseOnCComPtr@UIUnknown@@@1@XZ 0011f930 f i atlsd:atlbase.obj
 0001:0001e9b0       ??0?$CComPtr@UIPersistStream@@@ATL@@QAA@XZ 0011f9b0 f i atlsd:atlbase.obj
 0001:0001e9f0       ??1?$CComPtrBase@UIPersistStream@@@ATL@@QAA@XZ 0011f9f0 f i atlsd:atlbase.obj
 0001:0001ea38       ??I?$CComPtrBase@UIPersistStream@@@ATL@@QAAPAPAUIPersistStream@@XZ 0011fa38 f i atlsd:atlbase.obj
 0001:0001eab4       ??C?$CComPtrBase@UIPersistStream@@@ATL@@QBAPAV?$_NoAddRefReleaseOnCComPtr@UIPersistStream@@@1@XZ 0011fab4 f i atlsd:atlbase.obj
 0001:0001eb34       ??0?$CComPtrBase@UIUnknown@@@ATL@@IAA@XZ 0011fb34 f i atlsd:atlbase.obj
 0001:0001eb68       ??0?$CComPtrBase@UIPersistStream@@@ATL@@IAA@XZ 0011fb68 f i atlsd:atlbase.obj
 0001:0001eb9c       ??0CTraceCategory@ATL@@QAA@PB_WI@Z 0011fb9c f i atlsd:atltrace.obj
 0001:0001ec20       ?ChangeCategory@CTrace@ATL@@QAA_NKIW4ATLTRACESTATUS@2@@Z 0011fc20 f i atlsd:atltrace.obj
 0001:0001ec90       ?RegisterCategory@CTrace@ATL@@QAAKPB_W@Z 0011fc90 f i atlsd:atltrace.obj
 0001:0001ecdc       ??0CAtlAllocator@@QAA@XZ   0011fcdc f i atlsd:Externs.obj
 0001:0001ed6c       ??0CTraceSnapshot@@QAA@XZ  0011fd6c f i atlsd:Externs.obj
 0001:0001edc8       ??0?$CSimpleArray@UCModuleInfo@CTraceSnapshot@@V?$CSimpleArrayEqualHelper@UCModuleInfo@CTraceSnapshot@@@ATL@@@ATL@@QAA@XZ 0011fdc8 f i atlsd:Externs.obj
 0001:0001ee1c       ??0?$CSimpleArray@KV?$CSimpleArrayEqualHelper@K@ATL@@@ATL@@QAA@XZ 0011fe1c f i atlsd:Externs.obj
 0001:0001efe0       GetCurrentProcessId        0011ffe0 f i atlsd:Externs.obj
 0001:0001f000       ??0CAtlException@ATL@@QAA@J@Z 00120000 f i atlsd:Externs.obj
 0001:0001f034       ??0CTrace@ATL@@AAA@P6AHHPB_WH00ZZ@Z 00120034 f i atlsd:Externs.obj
 0001:0001f0bc       ??1CAtlAllocator@@QAA@XZ   001200bc f i atlsd:Externs.obj
 0001:0001f0fc       ??1CTraceSnapshot@@QAA@XZ  001200fc f i atlsd:Externs.obj
 0001:0001f13c       ??1?$CSimpleArray@UCModuleInfo@CTraceSnapshot@@V?$CSimpleArrayEqualHelper@UCModuleInfo@CTraceSnapshot@@@ATL@@@ATL@@QAA@XZ 0012013c f i atlsd:Externs.obj
 0001:0001f164       ??1?$CSimpleArray@KV?$CSimpleArrayEqualHelper@K@ATL@@@ATL@@QAA@XZ 00120164 f i atlsd:Externs.obj
 0001:0001f18c       ?RemoveAll@?$CSimpleArray@UCModuleInfo@CTraceSnapshot@@V?$CSimpleArrayEqualHelper@UCModuleInfo@CTraceSnapshot@@@ATL@@@ATL@@QAAXXZ 0012018c f i atlsd:Externs.obj
 0001:0001f230       ?RemoveAll@?$CSimpleArray@KV?$CSimpleArrayEqualHelper@K@ATL@@@ATL@@QAAXXZ 00120230 f i atlsd:Externs.obj
 0001:0001f2d4       ??1CTrace@ATL@@AAA@XZ      001202d4 f i atlsd:Externs.obj
 0001:0001f304       ?NotifyTool@ATL@@YAXXZ     00120304 f   atlsd:AtlDebugAPI.obj
 0001:0001f37c       AtlTraceRegister           0012037c f   atlsd:AtlDebugAPI.obj
 0001:0001f478       AtlTraceUnregister         00120478 f   atlsd:AtlDebugAPI.obj
 0001:0001f4d8       AtlTraceRegisterCategoryU  001204d8 f   atlsd:AtlDebugAPI.obj
 0001:0001f564       AtlTraceModifyProcess      00120564 f   atlsd:AtlDebugAPI.obj
 0001:0001f6e4       AtlTraceModifyModule       001206e4 f   atlsd:AtlDebugAPI.obj
 0001:0001f884       AtlTraceModifyCategory     00120884 f   atlsd:AtlDebugAPI.obj
 0001:0001f9c4       AtlTraceGetProcess         001209c4 f   atlsd:AtlDebugAPI.obj
 0001:0001fb64       AtlTraceGetModule          00120b64 f   atlsd:AtlDebugAPI.obj
 0001:0001fd54       AtlTraceGetCategory        00120d54 f   atlsd:AtlDebugAPI.obj
 0001:0001fef8       AtlTraceGetUpdateEventNameU 00120ef8 f   atlsd:AtlDebugAPI.obj
 0001:0001ff4c       AtlTraceGetUpdateEventNameU_s 00120f4c f   atlsd:AtlDebugAPI.obj
 0001:0001ffa4       AtlTraceVU                 00120fa4 f   atlsd:AtlDebugAPI.obj
 0001:000202b4       AtlTraceOpenProcess        001212b4 f   atlsd:AtlDebugAPI.obj
 0001:00020310       AtlTraceCloseProcess       00121310 f   atlsd:AtlDebugAPI.obj
 0001:0002044c       AtlTraceSnapshotProcess    0012144c f   atlsd:AtlDebugAPI.obj
 0001:00020524       AtlTraceGetProcessInfo     00121524 f   atlsd:AtlDebugAPI.obj
 0001:00020854       AtlTraceGetModuleInfo      00121854 f   atlsd:AtlDebugAPI.obj
 0001:00020b48       AtlTraceGetCategoryInfo    00121b48 f   atlsd:AtlDebugAPI.obj
 0001:00021200       ?GetProcess@CAtlAllocator@@QBAPAVCAtlTraceProcess@@XZ 00122200 f i atlsd:AtlDebugAPI.obj
 0001:00021230       ?Name@CAtlTraceCategory@@QBAPB_WXZ 00122230 f i atlsd:AtlDebugAPI.obj
 0001:0002125c       ?Path@CAtlTraceModuleInfo@@QBAPB_WXZ 0012225c f i atlsd:AtlDebugAPI.obj
 0001:00021288       ?Name@CAtlTraceModuleInfo@@QBAPB_WXZ 00122288 f i atlsd:AtlDebugAPI.obj
 0001:000212b4       ?Id@CAtlTraceProcess@@QBAKXZ 001222b4 f i atlsd:AtlDebugAPI.obj
 0001:000212e8       ?CrtDbgReport@CAtlTraceModule@@QBAP6AHHPB_WH00ZZXZ 001222e8 f i atlsd:AtlDebugAPI.obj
 0001:0002131c       ?GetSize@?$CSimpleArray@UCModuleInfo@CTraceSnapshot@@V?$CSimpleArrayEqualHelper@UCModuleInfo@CTraceSnapshot@@@ATL@@@ATL@@QBAHXZ 0012231c f i atlsd:AtlDebugAPI.obj
 0001:0002134c       ??A?$CSimpleArray@UCModuleInfo@CTraceSnapshot@@V?$CSimpleArrayEqualHelper@UCModuleInfo@CTraceSnapshot@@@ATL@@@ATL@@QAAAAUCModuleInfo@CTraceSnapshot@@H@Z 0012234c f i atlsd:AtlDebugAPI.obj
 0001:00021430       ?wcscpy_s@Checked@ATL@@YAXPA_WIPB_W@Z 00122430 f i atlsd:AtlDebugAPI.obj
 0001:00021488       ?Init@CAtlAllocator@@QAA_NPB_WK@Z 00122488 f   atlsd:Allocate.obj
 0001:00021960       ?Close@CAtlAllocator@@QAAX_N@Z 00122960 f   atlsd:Allocate.obj
 0001:00021a30       ?GetModule@CAtlAllocator@@QBAPAVCAtlTraceModule@@H@Z 00122a30 f   atlsd:Allocate.obj
 0001:00021b44       ?GetCategory@CAtlAllocator@@QBAPAVCAtlTraceCategory@@H@Z 00122b44 f   atlsd:Allocate.obj
 0001:00021c8c       ?GetCategoryCount@CAtlAllocator@@QBAHH@Z 00122c8c f   atlsd:Allocate.obj
 0001:00021d64       ?GetCategoryCount@CAtlAllocator@@QBAHABVCAtlTraceModule@@@Z 00122d64 f   atlsd:Allocate.obj
 0001:00021e00       ?GetModuleCount@CAtlAllocator@@QBAHXZ 00122e00 f   atlsd:Allocate.obj
 0001:00021ea0       ?FindModule@CAtlAllocator@@QBA_NPB_WPAI@Z 00122ea0 f   atlsd:Allocate.obj
 0001:00021f94       ?AddModule@CAtlAllocator@@QAAHPAUHINSTANCE__@@@Z 00122f94 f   atlsd:Allocate.obj
 0001:000222dc       ?AddCategory@CAtlAllocator@@QAAHHPB_W@Z 001232dc f   atlsd:Allocate.obj
 0001:000226e4       ?RemoveModule@CAtlAllocator@@QAA_NH@Z 001236e4 f   atlsd:Allocate.obj
 0001:00022818       ?CleanUp@CAtlAllocator@@QAAXXZ 00123818 f   atlsd:Allocate.obj
 0001:00022844       ?TakeSnapshot@CAtlAllocator@@QAAXXZ 00123844 f   atlsd:Allocate.obj
 0001:00022b80       ?ReleaseSnapshot@CAtlAllocator@@QAAXXZ 00123b80 f   atlsd:Allocate.obj
 0001:00022d20       ?IncRef@CAtlTraceProcess@@QAAIXZ 00123d20 f i atlsd:Allocate.obj
 0001:00022d78       ?Base@CAtlTraceProcess@@QBAPAXXZ 00123d78 f i atlsd:Allocate.obj
 0001:00022dac       ?DecRef@CAtlTraceProcess@@QAAIXZ 00123dac f i atlsd:Allocate.obj
 0001:00022e04       ?ModuleCount@CAtlTraceProcess@@QBAHXZ 00123e04 f i atlsd:Allocate.obj
 0001:00022e38       ?MaxSize@CAtlTraceProcess@@QBAKXZ 00123e38 f i atlsd:Allocate.obj
 0001:00022e68       ?CategoryCount@CAtlTraceProcess@@QBAHXZ 00123e68 f i atlsd:Allocate.obj
 0001:00022e98       ?TryAllocate@CAtlTraceSettings@@QAA_NXZ 00123e98 f i atlsd:Allocate.obj
 0001:00022f1c       ?MarkValid@CAtlTraceSettings@@QAAXJ@Z 00123f1c f i atlsd:Allocate.obj
 0001:00022f98       ?IncModuleCount@CAtlTraceProcess@@QAAXI@Z 00123f98 f i atlsd:Allocate.obj
 0001:00022fd4       ?TryAddRef@CAtlTraceSettings@@QAA_NXZ 00123fd4 f i atlsd:Allocate.obj
 0001:00023064       ?Release@CAtlTraceSettings@@QAAXXZ 00124064 f i atlsd:Allocate.obj
 0001:000230c0       ?IncCategoryCount@CAtlTraceProcess@@QAAXI@Z 001240c0 f i atlsd:Allocate.obj
 0001:000230f4       ?Add@?$CSimpleArray@UCModuleInfo@CTraceSnapshot@@V?$CSimpleArrayEqualHelper@UCModuleInfo@CTraceSnapshot@@@ATL@@@ATL@@QAAHABUCModuleInfo@CTraceSnapshot@@@Z 001240f4 f i atlsd:Allocate.obj
 0001:0002324c       ?GetSize@?$CSimpleArray@KV?$CSimpleArrayEqualHelper@K@ATL@@@ATL@@QBAHXZ 0012424c f i atlsd:Allocate.obj
 0001:0002327c       ?Add@?$CSimpleArray@KV?$CSimpleArrayEqualHelper@K@ATL@@@ATL@@QAAHABK@Z 0012427c f i atlsd:Allocate.obj
 0001:000233cc       ?RemoveAt@?$CSimpleArray@KV?$CSimpleArrayEqualHelper@K@ATL@@@ATL@@QAAHH@Z 001243cc f i atlsd:Allocate.obj
 0001:00023544       ??A?$CSimpleArray@KV?$CSimpleArrayEqualHelper@K@ATL@@@ATL@@QAAAAKH@Z 00124544 f i atlsd:Allocate.obj
 0001:00023628       ?InternalSetAtIndex@?$CSimpleArray@UCModuleInfo@CTraceSnapshot@@V?$CSimpleArrayEqualHelper@UCModuleInfo@CTraceSnapshot@@@ATL@@@ATL@@QAAXHABUCModuleInfo@CTraceSnapshot@@@Z 00124628 f i atlsd:Allocate.obj
 0001:000236b8       ?InternalSetAtIndex@?$CSimpleArray@KV?$CSimpleArrayEqualHelper@K@ATL@@@ATL@@QAAXHABK@Z 001246b8 f i atlsd:Allocate.obj
 0001:00023748       ??0Wrapper@?$CSimpleArray@UCModuleInfo@CTraceSnapshot@@V?$CSimpleArrayEqualHelper@UCModuleInfo@CTraceSnapshot@@@ATL@@@ATL@@QAA@ABUCModuleInfo@CTraceSnapshot@@@Z 00124748 f i atlsd:Allocate.obj
 0001:00023780       ??0Wrapper@?$CSimpleArray@KV?$CSimpleArrayEqualHelper@K@ATL@@@ATL@@QAA@ABK@Z 00124780 f i atlsd:Allocate.obj
 0001:000237b8       ??$?2UCModuleInfo@CTraceSnapshot@@@Wrapper@?$CSimpleArray@UCModuleInfo@CTraceSnapshot@@V?$CSimpleArrayEqualHelper@UCModuleInfo@CTraceSnapshot@@@ATL@@@ATL@@SAPAXIPAUCModuleInfo@CTraceSnapshot@@@Z 001247b8 f i atlsd:Allocate.obj
 0001:000237e0       ??$?2K@Wrapper@?$CSimpleArray@KV?$CSimpleArrayEqualHelper@K@ATL@@@ATL@@SAPAXIPAK@Z 001247e0 f i atlsd:Allocate.obj
 0001:00023808       ??2@YAPAXIPAX@Z            00124808 f i atlsd:Allocate.obj
 0001:00023830       ??0CAtlTraceModuleInfo@@QAA@XZ 00124830 f   atlsd:AtlTraceModuleManager.obj
 0001:000238a4       ?Reset@CAtlTraceModuleInfo@@QAAXPAUHINSTANCE__@@@Z 001248a4 f   atlsd:AtlTraceModuleManager.obj
 0001:00023a40       ??0CAtlTraceCategory@@QAA@XZ 00124a40 f   atlsd:AtlTraceModuleManager.obj
 0001:00023aac       ?Reset@CAtlTraceCategory@@QAAXPB_WJ@Z 00124aac f   atlsd:AtlTraceModuleManager.obj
 0001:00023b2c       ??0CAtlTraceModule@@QAA@XZ 00124b2c f   atlsd:AtlTraceModuleManager.obj
 0001:00023b98       ?CrtDbgReport@CAtlTraceModule@@QAAXP6AHHPB_WH00ZZ@Z 00124b98 f   atlsd:AtlTraceModuleManager.obj
 0001:00023bec       ??0CAtlTraceProcess@@QAA@K@Z 00124bec f   atlsd:AtlTraceModuleManager.obj
 0001:00023d64       ?GetNextCookie@CAtlTraceProcess@@QAAJXZ 00124d64 f   atlsd:AtlTraceModuleManager.obj
 0001:00023dac       ??0CAtlTraceSettings@@QAA@XZ 00124dac f i atlsd:AtlTraceModuleManager.obj
 0001:00023e10       __GSHandlerCheckCommon     00124e10 f   LIBCMTD:gshandler.obj
 0001:00023e58       __GSHandlerCheck           00124e58 f   LIBCMTD:gshandler.obj
 0001:00023e88       __InternalCxxFrameHandler  00124e88 f   LIBCMTD:frame_ce.obj
 0001:00024064       __CxxFrameHandler3         00125064 f   LIBCMTD:frame_ce.obj
 0001:00024840       __FrameUnwindToState       00125840 f   LIBCMTD:frame_ce.obj
 0001:000255ec       ?_DestructExceptionObject@@YAXPAUEHExceptionRecord@@E@Z 001265ec f   LIBCMTD:frame_ce.obj
 0001:0002573c       ?_OffsetToAddress@@YAPAXHPAKK@Z 0012673c f   LIBCMTD:frame_ce.obj
 0001:000257c8       ?FindFrameInfo@@YAPAU_FrameInfo@@PAK@Z 001267c8 f   LIBCMTD:frame_ce.obj
 0001:00025850       ?FindCatchFrameInfo@@YAPAU_FrameInfo@@PAK@Z 00126850 f   LIBCMTD:frame_ce.obj
 0001:000258d4       ?_GetRangeOfTrysToCheck@@YAPBU_s_TryBlockMapEntry@@PBU_s_FuncInfo@@HHPAI1@Z 001268d4 f   LIBCMTD:frame_ce.obj
 0001:000259d4       _CrtSetReportHookT2        001269d4 f   LIBCMTD:dbgrpt.obj
 0001:00025ea0       _CrtDbgReportW             00126ea0 f   LIBCMTD:dbgrpt.obj
 0001:00025f18       _CrtDbgReportTV            00126f18 f i LIBCMTD:dbgrpt.obj
 0001:00025f74       __crtMessageWindowW        00126f74 f   LIBCMTD:dbgrpt.obj
 0001:0002664c       _invoke_watson_if_error    0012764c f i LIBCMTD:dbgrpt.obj
 0001:000266a0       __GSHandlerCheck_EH        001276a0 f   LIBCMTD:gshandlereh.obj
 0001:00026734       memmove_s                  00127734 f   LIBCMTD:memmove_s.obj
 0001:000269a8       wcscpy_s                   001279a8 f   LIBCMTD:wcscpy_s.obj
 0001:00026e1c       wcsncpy_s                  00127e1c f   LIBCMTD:wcsncpy_s.obj
 0001:0002741c       GetCRTStorage              0012841c f   LIBCMTD:corecrt.obj
 0001:0002752c       TlsAlloc                   0012852c f i LIBCMTD:corecrt.obj
 0001:00027568       TlsFree                    00128568 f i LIBCMTD:corecrt.obj
 0001:000275ac       ?FindFrameForUnwind@@YAPAKPAKPBU_s_FuncInfo@@@Z 001285ac f   LIBCMTD:mdframe_arm.obj
 0001:00027644       ?FindCatchFrame@@YAPAKPAKK@Z 00128644 f   LIBCMTD:mdframe_arm.obj
 0001:000276dc       ?AdjustFrameForCatch@@YAPAKPAKPBU_s_FuncInfo@@@Z 001286dc f   LIBCMTD:mdframe_arm.obj
 0001:0002777c       ?GetCurrentState@@YAHPAKPAU_DISPATCHER_CONTEXT@@PBU_s_FuncInfo@@@Z 0012877c f   LIBCMTD:ehstate_arm_mips.obj
 0001:00027858       _CallSettingFrame          00128858     LIBCMTD:handlers_arm.obj
 0001:0002789c       _mtinitlocks               0012889c f   LIBCMTD:mlock.obj
 0001:000279b4       _mtdeletelocks             001289b4 f   LIBCMTD:mlock.obj
 0001:00027b38       _mtinitlocknum             00128b38 f   LIBCMTD:mlock.obj
 0001:00027ca0       _lock                      00128ca0 f   LIBCMTD:mlock.obj
 0001:00027d9c       _unlock                    00128d9c f   LIBCMTD:mlock.obj
 0001:00027ddc       _lockerr_exit              00128ddc f   LIBCMTD:mlock.obj
 0001:00027e04       _CrtDbgBreak               00128e04 f   LIBCMTD:dbgrptt.obj
 0001:00027e0c       _CrtSetReportMode          00128e0c f   LIBCMTD:dbgrptt.obj
 0001:00028034       _CrtSetReportFile          00129034 f   LIBCMTD:dbgrptt.obj
 0001:000281d0       _CrtSetReportHook          001291d0 f   LIBCMTD:dbgrptt.obj
 0001:00028214       _CrtGetReportHook          00129214 f   LIBCMTD:dbgrptt.obj
 0001:0002823c       _VCrtDbgReportW            0012923c f   LIBCMTD:dbgrptt.obj
 0001:00028df4       _invalid_parameter         00129df4 f   LIBCMTD:invarginternal.obj
 0001:00028e38       __crtMessageBoxW           00129e38 f   LIBCMTD:crtmbox.obj
 0001:0002909c       _invoke_watson             0012a09c f   LIBCMTD:invarg.obj
 0001:000290d0       _initp_misc_initcrit       0012a0d0 f   LIBCMTD:initcrit.obj
 0001:000290fc       __crtInitCritSecAndSpinCount 0012a0fc f   LIBCMTD:initcrit.obj
 0001:0002922c       _amsg_exit                 0012a22c f   LIBCMTD:crt0dat.obj
 0001:00029258       __crtExitProcess           0012a258 f   LIBCMTD:crt0dat.obj
 0001:000292a0       strcpy_s                   0012a2a0 f   LIBCMTD:strcpy_s.obj
 0001:000296f4       wcscat_s                   0012a6f4 f   LIBCMTD:wcscat_s.obj
 0001:00029cd8       _itow_s                    0012acd8 f   LIBCMTD:xtows.obj
 0001:0002a364       _ltow_s                    0012b364 f   LIBCMTD:xtows.obj
 0001:0002a3e4       _ultow_s                   0012b3e4 f   LIBCMTD:xtows.obj
 0001:0002a438       _encode_pointer            0012b438 f   LIBCMTD:tidtable.obj
 0001:0002a460       _encoded_null              0012b460 f   LIBCMTD:tidtable.obj
 0001:0002a498       _decode_pointer            0012b498 f   LIBCMTD:tidtable.obj
 0001:0002a4c0       __report_gsfailure         0012b4c0 f   coredll:COREDLL.dll
 0001:0002a4d0       LocalReAlloc               0012b4d0 f   coredll:COREDLL.dll
 0001:0002a4e0       LocalAlloc                 0012b4e0 f   coredll:COREDLL.dll
 0001:0002a4f0       LocalSize                  0012b4f0 f   coredll:COREDLL.dll
 0001:0002a500       LocalFree                  0012b500 f   coredll:COREDLL.dll
 0001:0002a510       DisableThreadLibraryCalls  0012b510 f   coredll:COREDLL.dll
 0001:0002a520       __security_gen_cookie      0012b520 f   coredll:COREDLL.dll
 0001:0002a530       DispatchMessageW           0012b530 f   coredll:COREDLL.dll
 0001:0002a540       TranslateMessage           0012b540 f   coredll:COREDLL.dll
 0001:0002a550       GetMessageW                0012b550 f   coredll:COREDLL.dll
 0001:0002a560       PeekMessageW               0012b560 f   coredll:COREDLL.dll
 0001:0002a570       MsgWaitForMultipleObjectsEx 0012b570 f   coredll:COREDLL.dll
 0001:0002a580       __C_specific_handler       0012b580 f   coredll:COREDLL.dll
 0001:0002a590       GetModuleHandleW           0012b590 f   coredll:COREDLL.dll
 0001:0002a5a0       realloc                    0012b5a0 f   coredll:COREDLL.dll
 0001:0002a5b0       _snwprintf                 0012b5b0 f   coredll:COREDLL.dll
 0001:0002a5c0       __CxxThrowException        0012b5c0 f   coredll:COREDLL.dll
 0001:0002a5d0       ??_7type_info@@6B@         0012b5d0 f   coredll:COREDLL.dll
 0001:0002a5e0       OpenEventW                 0012b5e0 f   coredll:COREDLL.dll
 0001:0002a5f0       _vsnwprintf                0012b5f0 f   coredll:COREDLL.dll
 0001:0002a600       VirtualAlloc               0012b600 f   coredll:COREDLL.dll
 0001:0002a610       UnmapViewOfFile            0012b610 f   coredll:COREDLL.dll
 0001:0002a620       memcmp                     0012b620 f   coredll:COREDLL.dll
 0001:0002a630       GetSystemInfo              0012b630 f   coredll:COREDLL.dll
 0001:0002a640       MapViewOfFile              0012b640 f   coredll:COREDLL.dll
 0001:0002a650       CreateFileMappingW         0012b650 f   coredll:COREDLL.dll
 0001:0002a660       InterlockedIncrement       0012b660 f   coredll:COREDLL.dll
 0001:0002a670       InterlockedDecrement       0012b670 f   coredll:COREDLL.dll
 0001:0002a680       strcmp                     0012b680 f   coredll:COREDLL.dll
 0001:0002a690       ?terminate@std@@YAXXZ      0012b690 f   coredll:COREDLL.dll
 0001:0002a6a0       memmove                    0012b6a0 f   coredll:COREDLL.dll
 0001:0002a6b0       malloc                     0012b6b0 f   coredll:COREDLL.dll
 0001:0002a6c0       TlsSetValue                0012b6c0 f   coredll:COREDLL.dll
 0001:0002a6d0       TlsGetValue                0012b6d0 f   coredll:COREDLL.dll
 0001:0002a6e0       InterlockedCompareExchange 0012b6e0 f   coredll:COREDLL.dll
 0001:0002a6f0       TlsCall                    0012b6f0 f   coredll:COREDLL.dll
 0001:0002a700       SetLastError               0012b700 f   coredll:COREDLL.dll
 0001:0002a710       TerminateProcess           0012b710 f   coredll:COREDLL.dll
 0001:0002a720       CreateStreamOnHGlobal      0012b720 f   ole32:ole32.dll
 0001:0002a730       WriteClassStm              0012b730 f   ole32:ole32.dll
 0001:0002a740       CoCreateInstance           0012b740 f   ole32:ole32.dll
 0001:0002a750       ReadClassStm               0012b750 f   ole32:ole32.dll
 0002:00008424       ??_7SW_RegistryKey@@6B@    00135424     ModemStat.obj
 0002:00008458       ??_7CModemStatus@@6B@      00135458     ModemStat.obj
 0002:0000845c       ??_C@_1CE@ILHCKNGC@?$AAR?$AAI?$AAL?$AA_?$AAC?$AAA?$AAL?$AAL?$AA_?$AAB?$AAY?$AAT?$AAE?$AA_?$AAC?$AAT?$AAR?$AA?$AA@ 0013545c     ModemStat.obj
 0002:00008480       ??_C@_1CE@GDPLDIKM@?$AAR?$AAI?$AAL?$AA_?$AAP?$AAD?$AAS?$AAM?$AA_?$AAP?$AAA?$AA_?$AAP?$AAA?$AAR?$AAA?$AAM?$AA?$AA@ 00135480     ModemStat.obj
 0002:000084a4       ??_C@_1CM@BAFGFLAD@?$AAR?$AAI?$AAL?$AA_?$AAP?$AAD?$AAS?$AAM?$AA_?$AAP?$AAD?$AA_?$AAD?$AAL?$AAD?$AA_?$AAB?$AAE?$AAG?$AAI?$AAN?$AA?$AA@ 001354a4     ModemStat.obj
 0002:000084d0       ??_C@_1CI@IINDIONI@?$AAR?$AAI?$AAL?$AA_?$AAP?$AAD?$AAS?$AAM?$AA_?$AAP?$AAD?$AA_?$AAD?$AAL?$AAD?$AA_?$AAE?$AAN?$AAD?$AA?$AA@ 001354d0     ModemStat.obj
 0002:000084f8       ??_C@_1CK@GNNIIJCK@?$AAR?$AAI?$AAL?$AA_?$AAP?$AAD?$AAS?$AAM?$AA_?$AAP?$AAD?$AA_?$AAD?$AAL?$AAD?$AA_?$AAD?$AAO?$AAN?$AAE?$AA?$AA@ 001354f8     ModemStat.obj
 0002:00008524       ??_C@_1CK@FFHNCNLC@?$AAR?$AAI?$AAL?$AA_?$AAP?$AAD?$AAS?$AAM?$AA_?$AAP?$AAD?$AA_?$AAD?$AAL?$AAD?$AA_?$AAD?$AAA?$AAT?$AAA?$AA?$AA@ 00135524     ModemStat.obj
 0002:00008550       ??_C@_1DG@ENNLKGLF@?$AAR?$AAI?$AAL?$AA_?$AAP?$AAD?$AAS?$AAM?$AA_?$AAP?$AAD?$AA_?$AAU?$AAP?$AAD?$AAA?$AAT?$AAE?$AA_?$AAF?$AAA?$AAI?$AAL?$AAU?$AAR?$AAE?$AA?$AA@ 00135550     ModemStat.obj
 0002:00008588       ??_C@_1CE@DKNHCEGP@?$AAR?$AAI?$AAL?$AA_?$AAP?$AAD?$AAS?$AAM?$AA_?$AAP?$AAD?$AA_?$AAB?$AAE?$AAG?$AAI?$AAN?$AA?$AA@ 00135588     ModemStat.obj
 0002:000085ac       ??_C@_1CA@IJMMNJBM@?$AAR?$AAI?$AAL?$AA_?$AAP?$AAD?$AAS?$AAM?$AA_?$AAP?$AAD?$AA_?$AAE?$AAN?$AAD?$AA?$AA@ 001355ac     ModemStat.obj
 0002:000085cc       ??_C@_1CC@DHEBFOCI@?$AAR?$AAI?$AAL?$AA_?$AAP?$AAD?$AAS?$AAM?$AA_?$AAP?$AAD?$AA_?$AAD?$AAO?$AAN?$AAE?$AA?$AA@ 001355cc     ModemStat.obj
 0002:000085f0       ??_C@_1CC@POEPKLA@?$AAR?$AAI?$AAL?$AA_?$AAP?$AAD?$AAS?$AAM?$AA_?$AAP?$AAD?$AA_?$AAD?$AAA?$AAT?$AAA?$AA?$AA@ 001355f0     ModemStat.obj
 0002:00008614       ??_C@_1CC@BEOCDLIL@?$AAR?$AAI?$AAL?$AA_?$AAI?$AAO?$AAT?$AAA?$AA_?$AAW?$AAA?$AAP?$AA_?$AAU?$AAR?$AAI?$AA?$AA@ 00135614     ModemStat.obj
 0002:00008638       ??_C@_1DA@MPHILDIE@?$AAR?$AAI?$AAL?$AA_?$AAI?$AAO?$AAT?$AAA?$AA_?$AAS?$AAT?$AAA?$AAT?$AAU?$AAS?$AA_?$AAC?$AAH?$AAA?$AAN?$AAG?$AAE?$AAD?$AA?$AA@ 00135638     ModemStat.obj
 0002:00008668       ??_C@_1CG@HIPGCNFB@?$AAR?$AAI?$AAL?$AA_?$AAT?$AAE?$AAC?$AAH?$AAH?$AAD?$AAR?$AA_?$AAN?$AAO?$AAT?$AAI?$AAF?$AAY?$AA?$AA@ 00135668     ModemStat.obj
 0002:00008690       ??_C@_1BO@NKICKCPO@?$AAR?$AAI?$AAL?$AA_?$AAD?$AAB?$AAG?$AA_?$AAN?$AAO?$AAT?$AAI?$AAF?$AAY?$AA?$AA@ 00135690     ModemStat.obj
 0002:000086b0       ??_C@_1CG@POBHOMMK@?$AAR?$AAI?$AAL?$AA_?$AAS?$AAT?$AAA?$AAT?$AAU?$AAS?$AA_?$AAC?$AAH?$AAA?$AAN?$AAG?$AAE?$AAD?$AA?$AA@ 001356b0     ModemStat.obj
 0002:000086d8       ??_C@_1CI@DNMBCABB@?$AAE?$AAR?$AAR?$AA_?$AAR?$AAI?$AAL?$AA_?$AAA?$AAP?$AAI?$AA_?$AAT?$AAI?$AAM?$AAE?$AAO?$AAU?$AAT?$AA?$AA@ 001356d8     ModemStat.obj
 0002:00008700       ??_7CriticalSection@@6B@   00135700     ModemStat.obj
 0002:00008914       ?_Min@?$AtlLimits@H@ATL@@2HB 00135914     stdafx.obj
 0002:00008918       ?_Max@?$AtlLimits@H@ATL@@2HB 00135918     stdafx.obj
 0002:0000891c       ?_Min@?$AtlLimits@I@ATL@@2IB 0013591c     stdafx.obj
 0002:00008920       ?_Max@?$AtlLimits@I@ATL@@2IB 00135920     stdafx.obj
 0002:00008924       ?_Min@?$AtlLimits@J@ATL@@2JB 00135924     stdafx.obj
 0002:00008928       ?_Max@?$AtlLimits@J@ATL@@2JB 00135928     stdafx.obj
 0002:0000892c       ?_Min@?$AtlLimits@K@ATL@@2KB 0013592c     stdafx.obj
 0002:00008930       ?_Max@?$AtlLimits@K@ATL@@2KB 00135930     stdafx.obj
 0002:00008938       ?_Min@?$AtlLimits@_J@ATL@@2_JB 00135938     stdafx.obj
 0002:00008940       ?_Max@?$AtlLimits@_J@ATL@@2_JB 00135940     stdafx.obj
 0002:00008948       ?_Min@?$AtlLimits@_K@ATL@@2_KB 00135948     stdafx.obj
 0002:00008950       ?_Max@?$AtlLimits@_K@ATL@@2_KB 00135950     stdafx.obj
 0002:00008958       ?VT@?$CVarTypeInfo@D@ATL@@2GB 00135958     stdafx.obj
 0002:0000895c       ?pmField@?$CVarTypeInfo@D@ATL@@2QQtagVARIANT@@DQ3@ 0013595c     stdafx.obj
 0002:00008960       ?VT@?$CVarTypeInfo@E@ATL@@2GB 00135960     stdafx.obj
 0002:00008964       ?pmField@?$CVarTypeInfo@E@ATL@@2QQtagVARIANT@@EQ3@ 00135964     stdafx.obj
 0002:00008968       ?VT@?$CVarTypeInfo@PAD@ATL@@2GB 00135968     stdafx.obj
 0002:0000896c       ?pmField@?$CVarTypeInfo@PAD@ATL@@2QQtagVARIANT@@PADQ3@ 0013596c     stdafx.obj
 0002:00008970       ?VT@?$CVarTypeInfo@PAE@ATL@@2GB 00135970     stdafx.obj
 0002:00008974       ?pmField@?$CVarTypeInfo@PAE@ATL@@2QQtagVARIANT@@PAEQ3@ 00135974     stdafx.obj
 0002:00008978       ?VT@?$CVarTypeInfo@F@ATL@@2GB 00135978     stdafx.obj
 0002:0000897c       ?pmField@?$CVarTypeInfo@F@ATL@@2QQtagVARIANT@@FQ3@ 0013597c     stdafx.obj
 0002:00008980       ?VT@?$CVarTypeInfo@PAF@ATL@@2GB 00135980     stdafx.obj
 0002:00008984       ?pmField@?$CVarTypeInfo@PAF@ATL@@2QQtagVARIANT@@PAFQ3@ 00135984     stdafx.obj
 0002:00008988       ?VT@?$CVarTypeInfo@G@ATL@@2GB 00135988     stdafx.obj
 0002:0000898c       ?pmField@?$CVarTypeInfo@G@ATL@@2QQtagVARIANT@@GQ3@ 0013598c     stdafx.obj
 0002:00008990       ?VT@?$CVarTypeInfo@H@ATL@@2GB 00135990     stdafx.obj
 0002:00008994       ?pmField@?$CVarTypeInfo@H@ATL@@2QQtagVARIANT@@HQ3@ 00135994     stdafx.obj
 0002:00008998       ?VT@?$CVarTypeInfo@PAH@ATL@@2GB 00135998     stdafx.obj
 0002:0000899c       ?pmField@?$CVarTypeInfo@PAH@ATL@@2QQtagVARIANT@@PAHQ3@ 0013599c     stdafx.obj
 0002:000089a0       ?VT@?$CVarTypeInfo@I@ATL@@2GB 001359a0     stdafx.obj
 0002:000089a4       ?pmField@?$CVarTypeInfo@I@ATL@@2QQtagVARIANT@@IQ3@ 001359a4     stdafx.obj
 0002:000089a8       ?VT@?$CVarTypeInfo@PAI@ATL@@2GB 001359a8     stdafx.obj
 0002:000089ac       ?pmField@?$CVarTypeInfo@PAI@ATL@@2QQtagVARIANT@@PAIQ3@ 001359ac     stdafx.obj
 0002:000089b0       ?VT@?$CVarTypeInfo@J@ATL@@2GB 001359b0     stdafx.obj
 0002:000089b4       ?pmField@?$CVarTypeInfo@J@ATL@@2QQtagVARIANT@@JQ3@ 001359b4     stdafx.obj
 0002:000089b8       ?VT@?$CVarTypeInfo@PAJ@ATL@@2GB 001359b8     stdafx.obj
 0002:000089bc       ?pmField@?$CVarTypeInfo@PAJ@ATL@@2QQtagVARIANT@@PAJQ3@ 001359bc     stdafx.obj
 0002:000089c0       ?VT@?$CVarTypeInfo@K@ATL@@2GB 001359c0     stdafx.obj
 0002:000089c4       ?pmField@?$CVarTypeInfo@K@ATL@@2QQtagVARIANT@@KQ3@ 001359c4     stdafx.obj
 0002:000089c8       ?VT@?$CVarTypeInfo@PAK@ATL@@2GB 001359c8     stdafx.obj
 0002:000089cc       ?pmField@?$CVarTypeInfo@PAK@ATL@@2QQtagVARIANT@@PAKQ3@ 001359cc     stdafx.obj
 0002:000089d0       ?VT@?$CVarTypeInfo@M@ATL@@2GB 001359d0     stdafx.obj
 0002:000089d4       ?pmField@?$CVarTypeInfo@M@ATL@@2QQtagVARIANT@@MQ3@ 001359d4     stdafx.obj
 0002:000089d8       ?VT@?$CVarTypeInfo@PAM@ATL@@2GB 001359d8     stdafx.obj
 0002:000089dc       ?pmField@?$CVarTypeInfo@PAM@ATL@@2QQtagVARIANT@@PAMQ3@ 001359dc     stdafx.obj
 0002:000089e0       ?VT@?$CVarTypeInfo@N@ATL@@2GB 001359e0     stdafx.obj
 0002:000089e4       ?pmField@?$CVarTypeInfo@N@ATL@@2QQtagVARIANT@@NQ3@ 001359e4     stdafx.obj
 0002:000089e8       ?VT@?$CVarTypeInfo@PAN@ATL@@2GB 001359e8     stdafx.obj
 0002:000089ec       ?pmField@?$CVarTypeInfo@PAN@ATL@@2QQtagVARIANT@@PANQ3@ 001359ec     stdafx.obj
 0002:000089f0       ?VT@?$CVarTypeInfo@UtagVARIANT@@@ATL@@2GB 001359f0     stdafx.obj
 0002:000089f4       ?VT@?$CVarTypeInfo@PAG@ATL@@2GB 001359f4     stdafx.obj
 0002:000089f8       ?pmField@?$CVarTypeInfo@PAG@ATL@@2QQtagVARIANT@@PAGQ3@ 001359f8     stdafx.obj
 0002:000089fc       ?VT@?$CVarTypeInfo@PAPAG@ATL@@2GB 001359fc     stdafx.obj
 0002:00008a00       ?pmField@?$CVarTypeInfo@PAPAG@ATL@@2QQtagVARIANT@@PAPAGQ3@ 00135a00     stdafx.obj
 0002:00008a04       ?VT@?$CVarTypeInfo@PAUIUnknown@@@ATL@@2GB 00135a04     stdafx.obj
 0002:00008a08       ?pmField@?$CVarTypeInfo@PAUIUnknown@@@ATL@@2QQtagVARIANT@@PAUIUnknown@@Q3@ 00135a08     stdafx.obj
 0002:00008a0c       ?VT@?$CVarTypeInfo@PAPAUIUnknown@@@ATL@@2GB 00135a0c     stdafx.obj
 0002:00008a10       ?pmField@?$CVarTypeInfo@PAPAUIUnknown@@@ATL@@2QQtagVARIANT@@PAPAUIUnknown@@Q3@ 00135a10     stdafx.obj
 0002:00008a14       ?VT@?$CVarTypeInfo@PAUIDispatch@@@ATL@@2GB 00135a14     stdafx.obj
 0002:00008a18       ?pmField@?$CVarTypeInfo@PAUIDispatch@@@ATL@@2QQtagVARIANT@@PAUIDispatch@@Q3@ 00135a18     stdafx.obj
 0002:00008a1c       ?VT@?$CVarTypeInfo@PAPAUIDispatch@@@ATL@@2GB 00135a1c     stdafx.obj
 0002:00008a20       ?pmField@?$CVarTypeInfo@PAPAUIDispatch@@@ATL@@2QQtagVARIANT@@PAPAUIDispatch@@Q3@ 00135a20     stdafx.obj
 0002:00008a24       ?VT@?$CVarTypeInfo@TtagCY@@@ATL@@2GB 00135a24     stdafx.obj
 0002:00008a28       ?pmField@?$CVarTypeInfo@TtagCY@@@ATL@@2QQtagVARIANT@@TtagCY@@Q3@ 00135a28     stdafx.obj
 0002:00008a2c       ?VT@?$CVarTypeInfo@PATtagCY@@@ATL@@2GB 00135a2c     stdafx.obj
 0002:00008a30       ?pmField@?$CVarTypeInfo@PATtagCY@@@ATL@@2QQtagVARIANT@@PATtagCY@@Q3@ 00135a30     stdafx.obj
 0002:00008a34       LIBID_ATLLib               00135a34     stdafx.obj
 0002:00008a44       CLSID_Registrar            00135a44     stdafx.obj
 0002:00008a54       IID_IRegistrar             00135a54     stdafx.obj
 0002:00008a64       IID_IAxWinHostWindow       00135a64     stdafx.obj
 0002:00008a74       IID_IAxWinAmbientDispatch  00135a74     stdafx.obj
 0002:00008a84       IID_IInternalConnection    00135a84     stdafx.obj
 0002:00008a94       IID_IDocHostUIHandlerDispatch 00135a94     stdafx.obj
 0002:00008aa4       IID_IAxWinHostWindowLic    00135aa4     stdafx.obj
 0002:00008ab4       IID_IAxWinAmbientDispatchEx 00135ab4     stdafx.obj
 0002:00008ac4       ?MAX_VALUE@CRegParser@ATL@@1HB 00135ac4     stdafx.obj
 0002:00008ac8       ?MAX_TYPE@CRegParser@ATL@@1HB 00135ac8     stdafx.obj
 0002:00008acc       ?rgszNeverDelete@CRegParser@ATL@@1QBQBGB 00135acc     stdafx.obj
 0002:00008afc       ?cbNeverDelete@CRegParser@ATL@@1HB 00135afc     stdafx.obj
 0002:00008b00       ??_C@_1JE@NABCONDI@?$AAC?$AA?3?$AA?2?$AAP?$AAr?$AAo?$AAg?$AAr?$AAa?$AAm?$AA?5?$AAF?$AAi?$AAl?$AAe?$AAs?$AA?2?$AAM?$AAi?$AAc?$AAr?$AAo?$AAs?$AAo?$AAf?$AAt?$AA?5?$AAV?$AAi?$AAs?$AAu?$AAa@ 00135b00     stdafx.obj
 0002:00008b94       ??_C@_13COJANIEC@?$AA0?$AA?$AA@ 00135b94     stdafx.obj
 0002:00008c50       ??_C@_1JM@HGDAICHJ@?$AAC?$AA?3?$AA?2?$AAP?$AAr?$AAo?$AAg?$AAr?$AAa?$AAm?$AA?5?$AAF?$AAi?$AAl?$AAe?$AAs?$AA?2?$AAM?$AAi?$AAc?$AAr?$AAo?$AAs?$AAo?$AAf?$AAt?$AA?5?$AAV?$AAi?$AAs?$AAu?$AAa@ 00135c50     stdafx.obj
 0002:00008cf0       ??_C@_1EA@JHMKKLFC@?$AAn?$AAI?$AAn?$AAd?$AAe?$AAx?$AA?5?$AA?$DO?$AA?$DN?$AA?5?$AA0?$AA?5?$AA?$CG?$AA?$CG?$AA?5?$AAn?$AAI?$AAn?$AAd?$AAe?$AAx?$AA?5?$AA?$DM?$AA?5?$AAm?$AA_?$AAn?$AAS?$AAi?$AAz?$AAe?$AA?$AA@ 00135cf0     stdafx.obj
 0002:00010db4       _GUID_b196b284_bab4_101a_b69c_00aa00341d07 0013ddb4     atlsd:atlfuncs.obj
 0002:00010dc4       _GUID_00000000_0000_0000_c000_000000000046 0013ddc4     atlsd:atlfuncs.obj
 0002:00010dd8       ??_C@_1HA@FENMNPLO@?$AAf?$AA?3?$AA?2?$AAd?$AAd?$AA?2?$AAv?$AAc?$AAt?$AAo?$AAo?$AAl?$AAs?$AA?2?$AAv?$AAc?$AA7?$AAl?$AAi?$AAb?$AAs?$AAc?$AAe?$AA?2?$AAs?$AAh?$AAi?$AAp?$AA?2?$AAa?$AAt?$AAl@ 0013ddd8     atlsd:atlfuncs.obj
 0002:00010e48       ??_C@_19LMDLLIGP@?$AAp?$AA?$DN?$AA?$DN?$AA0?$AA?$AA@ 0013de48     atlsd:atlfuncs.obj
 0002:00010e54       ??_C@_19JHCPJMAL@?$AAp?$AA?$CB?$AA?$DN?$AA0?$AA?$AA@ 0013de54     atlsd:atlfuncs.obj
 0002:00010e60       ??_C@_1HA@LPPEBACM@?$AAf?$AA?3?$AA?2?$AAd?$AAd?$AA?2?$AAv?$AAc?$AAt?$AAo?$AAo?$AAl?$AAs?$AA?2?$AAv?$AAc?$AA7?$AAl?$AAi?$AAb?$AAs?$AAc?$AAe?$AA?2?$AAs?$AAh?$AAi?$AAp?$AA?2?$AAa?$AAt?$AAl@ 0013de60     atlsd:atlfuncs.obj
 0002:00010ed0       ??_C@_1M@HLGKFCJM@?$AAf?$AAa?$AAl?$AAs?$AAe?$AA?$AA@ 0013ded0     atlsd:atlfuncs.obj
 0002:00010edc       ??_C@_1CK@DFMKPFAK@?$AAA?$AAt?$AAl?$AAT?$AAh?$AAr?$AAo?$AAw?$AA?3?$AA?5?$AAh?$AAr?$AA?5?$AA?$DN?$AA?5?$AA0?$AAx?$AA?$CF?$AAx?$AA?6?$AA?$AA@ 0013dedc     atlsd:atlfuncs.obj
 0002:00010f08       ??_C@_0DI@MHBOGIL@f?3?2dd?2vctools?2vc7libsce?2ship?2atl@ 0013df08     atlsd:atlfuncs.obj
 0002:00010f40       ??_C@_1GM@IDLEHDFG@?$AAf?$AA?3?$AA?2?$AAd?$AAd?$AA?2?$AAv?$AAc?$AAt?$AAo?$AAo?$AAl?$AAs?$AA?2?$AAv?$AAc?$AA7?$AAl?$AAi?$AAb?$AAs?$AAc?$AAe?$AA?2?$AAs?$AAh?$AAi?$AAp?$AA?2?$AAa?$AAt?$AAl@ 0013df40     atlsd:atlfuncs.obj
 0002:00010fac       ??_C@_1BE@NPGJNKLA@?$AAm?$AA_?$AAb?$AAL?$AAo?$AAc?$AAk?$AAe?$AAd?$AA?$AA@ 0013dfac     atlsd:atlfuncs.obj
 0002:00010fc0       ??_C@_1BG@OHCCAGNO@?$AA?$CB?$AAm?$AA_?$AAb?$AAL?$AAo?$AAc?$AAk?$AAe?$AAd?$AA?$AA@ 0013dfc0     atlsd:atlfuncs.obj
 0002:00010fd8       ??_C@_1HE@LMFAHKHJ@?$AAf?$AA?3?$AA?2?$AAd?$AAd?$AA?2?$AAv?$AAc?$AAt?$AAo?$AAo?$AAl?$AAs?$AA?2?$AAv?$AAc?$AA7?$AAl?$AAi?$AAb?$AAs?$AAc?$AAe?$AA?2?$AAs?$AAh?$AAi?$AAp?$AA?2?$AAa?$AAt?$AAl@ 0013dfd8     atlsd:atlfuncs.obj
 0002:000111c0       GUID_ATLVer30              0013e1c0     atlsd:atlbase.obj
 0002:000111d0       GUID_ATLVer70              0013e1d0     atlsd:atlbase.obj
 0002:00014480       ??_C@_1JC@IHNNLNKC@?$AAf?$AA?3?$AA?2?$AAd?$AAd?$AA?2?$AAv?$AAc?$AAt?$AAo?$AAo?$AAl?$AAs?$AA?2?$AAv?$AAc?$AA7?$AAl?$AAi?$AAb?$AAs?$AAc?$AAe?$AA?2?$AAs?$AAh?$AAi?$AAp?$AA?2?$AAa?$AAt?$AAl@ 00141480     atlsd:Allocate.obj
 0002:00014514       ??_C@_1BK@GFEAMNLJ@?$AAn?$AAC?$AAo?$AAo?$AAk?$AAi?$AAe?$AA?5?$AA?$CB?$AA?$DN?$AA?5?$AA0?$AA?$AA@ 00141514     atlsd:Allocate.obj
 0002:00014914       ??_C@_17LGKOMLJ@?$AA?4?$AA?4?$AA?4?$AA?$AA@ 00141914     LIBCMTD:dbgrpt.obj
 0002:0001491c       ??_C@_1CC@CGHMNGDG@?$AAA?$AAs?$AAs?$AAe?$AAr?$AAt?$AAi?$AAo?$AAn?$AA?5?$AAF?$AAa?$AAi?$AAl?$AAe?$AAd?$AA?$AA@ 0014191c     LIBCMTD:dbgrpt.obj
 0002:00014940       ??_C@_1M@ILHOPKA@?$AAE?$AAr?$AAr?$AAo?$AAr?$AA?$AA@ 00141940     LIBCMTD:dbgrpt.obj
 0002:0001494c       ??_C@_1BA@GLMCNLEM@?$AAW?$AAa?$AAr?$AAn?$AAi?$AAn?$AAg?$AA?$AA@ 0014194c     LIBCMTD:dbgrpt.obj
 0002:00014960       ??_C@_1FI@PHIAFFHM@?$AA?$CI?$AA?$CC?$AAT?$AAh?$AAe?$AA?5?$AAh?$AAo?$AAo?$AAk?$AA?5?$AAf?$AAu?$AAn?$AAc?$AAt?$AAi?$AAo?$AAn?$AA?5?$AAi?$AAs?$AA?5?$AAn?$AAo?$AAt?$AA?5?$AAi?$AAn?$AA?5?$AAt?$AAh@ 00141960     LIBCMTD:dbgrpt.obj
 0002:000149b8       ??_C@_1CG@JBJEFOCM@?$AAp?$AAf?$AAn?$AAN?$AAe?$AAw?$AAH?$AAo?$AAo?$AAk?$AA?5?$AA?$CB?$AA?$DN?$AA?5?$AAN?$AAU?$AAL?$AAL?$AA?$AA@ 001419b8     LIBCMTD:dbgrpt.obj
 0002:000149e0       ??_C@_1CI@OOAHIOG@?$AA_?$AAC?$AAr?$AAt?$AAS?$AAe?$AAt?$AAR?$AAe?$AAp?$AAo?$AAr?$AAt?$AAH?$AAo?$AAo?$AAk?$AAT?$AA2?$AA?$AA@ 001419e0     LIBCMTD:dbgrpt.obj
 0002:00014a08       ??_C@_1FC@DDJKODKC@?$AAf?$AA?3?$AA?2?$AAs?$AAp?$AA?2?$AAv?$AAc?$AAt?$AAo?$AAo?$AAl?$AAs?$AA?2?$AAc?$AAr?$AAt?$AAc?$AAe?$AA?2?$AAc?$AAr?$AAt?$AAw?$AA3?$AA2?$AA?2?$AAm?$AAi?$AAs?$AAc?$AA?2@ 00141a08     LIBCMTD:dbgrpt.obj
 0002:00014a60       ??_C@_1HI@OFEHGPPC@?$AAm?$AAo?$AAd?$AAe?$AA?5?$AA?$DN?$AA?$DN?$AA?5?$AA_?$AAC?$AAR?$AAT?$AA_?$AAR?$AAP?$AAT?$AAH?$AAO?$AAO?$AAK?$AA_?$AAI?$AAN?$AAS?$AAT?$AAA?$AAL?$AAL?$AA?5?$AA?$HM?$AA?$HM?$AA?5@ 00141a60     LIBCMTD:dbgrpt.obj
 0002:00014ad8       ??_C@_1EG@PEOEAKBB@?$AAM?$AAi?$AAc?$AAr?$AAo?$AAs?$AAo?$AAf?$AAt?$AA?5?$AAV?$AAi?$AAs?$AAu?$AAa?$AAl?$AA?5?$AAC?$AA?$CL?$AA?$CL?$AA?5?$AAD?$AAe?$AAb?$AAu?$AAg?$AA?5?$AAL?$AAi?$AAb?$AAr?$AAa@ 00141ad8     LIBCMTD:dbgrpt.obj
 0002:00014b20       ??_C@_1JI@EACPGHID@?$AAw?$AAc?$AAs?$AAc?$AAp?$AAy?$AA_?$AAs?$AA?$CI?$AAs?$AAz?$AAO?$AAu?$AAt?$AAM?$AAe?$AAs?$AAs?$AAa?$AAg?$AAe?$AA?0?$AA?5?$AA4?$AA0?$AA9?$AA6?$AA?0?$AA?5?$AAL?$AA?$CC?$AA_@ 00141b20     LIBCMTD:dbgrpt.obj
 0002:00014bb8       ??_C@_1FG@BBOLDHGF@?$AA_?$AAC?$AAr?$AAt?$AAD?$AAb?$AAg?$AAR?$AAe?$AAp?$AAo?$AAr?$AAt?$AA?3?$AA?5?$AAS?$AAt?$AAr?$AAi?$AAn?$AAg?$AA?5?$AAt?$AAo?$AAo?$AA?5?$AAl?$AAo?$AAn?$AAg?$AA?5?$AAo@ 00141bb8     LIBCMTD:dbgrpt.obj
 0002:00014c10       ??_C@_1KG@MFHGLLO@?$AAD?$AAe?$AAb?$AAu?$AAg?$AA?5?$AA?$CF?$AAs?$AA?$CB?$AA?6?$AA?6?$AAP?$AAr?$AAo?$AAg?$AAr?$AAa?$AAm?$AA?3?$AA?5?$AA?$CF?$AAs?$AA?$CF?$AAs?$AA?$CF?$AAs?$AA?$CF?$AAs?$AA?$CF?$AAs?$AA?$CF?$AAs@ 00141c10     LIBCMTD:dbgrpt.obj
 0002:00014cb8       ??_C@_1BE@CGCJKGHI@?$AA?6?$AAM?$AAo?$AAd?$AAu?$AAl?$AAe?$AA?3?$AA?5?$AA?$AA@ 00141cb8     LIBCMTD:dbgrpt.obj
 0002:00014ccc       ??_C@_1BA@LNHECFIM@?$AA?6?$AAF?$AAi?$AAl?$AAe?$AA?3?$AA?5?$AA?$AA@ 00141ccc     LIBCMTD:dbgrpt.obj
 0002:00014cdc       ??_C@_1BA@GLLGCPCK@?$AA?6?$AAL?$AAi?$AAn?$AAe?$AA?3?$AA?5?$AA?$AA@ 00141cdc     LIBCMTD:dbgrpt.obj
 0002:00014cec       ??_C@_13LBAGMAIH@?$AA?6?$AA?$AA@ 00141cec     LIBCMTD:dbgrpt.obj
 0002:00014cf0       ??_C@_1BK@PEDCIPMA@?$AAE?$AAx?$AAp?$AAr?$AAe?$AAs?$AAs?$AAi?$AAo?$AAn?$AA?3?$AA?5?$AA?$AA@ 00141cf0     LIBCMTD:dbgrpt.obj
 0002:00014d0c       ??_C@_11LOCGONAA@?$AA?$AA@ 00141d0c     LIBCMTD:dbgrpt.obj
 0002:00014d10       ??_C@_1JM@GKDPCMEA@?$AAw?$AAc?$AAs?$AAn?$AAc?$AAp?$AAy?$AA_?$AAs?$AA?$CI?$AAs?$AAz?$AAS?$AAh?$AAo?$AAr?$AAt?$AAP?$AAr?$AAo?$AAg?$AAN?$AAa?$AAm?$AAe?$AA?0?$AA?5?$AA2?$AA6?$AA0?$AA?5?$AA?9@ 00141d10     LIBCMTD:dbgrpt.obj
 0002:00014db0       ??_C@_1GI@DEDNNLCI@?$AAw?$AAc?$AAs?$AAc?$AAp?$AAy?$AA_?$AAs?$AA?$CI?$AAs?$AAz?$AAE?$AAx?$AAe?$AAN?$AAa?$AAm?$AAe?$AA?0?$AA?5?$AA2?$AA6?$AA0?$AA?0?$AA?5?$AAL?$AA?$CC?$AA?$DM?$AAp?$AAr?$AAo?$AAg@ 00141db0     LIBCMTD:dbgrpt.obj
 0002:00014e18       ??_C@_1CI@PGJIFDEK@?$AA_?$AA_?$AAc?$AAr?$AAt?$AAM?$AAe?$AAs?$AAs?$AAa?$AAg?$AAe?$AAW?$AAi?$AAn?$AAd?$AAo?$AAw?$AAW?$AA?$AA@ 00141e18     LIBCMTD:dbgrpt.obj
 0002:00014e40       ??_C@_1CO@EAEJAADC@?$AA?$DM?$AAp?$AAr?$AAo?$AAg?$AAr?$AAa?$AAm?$AA?5?$AAn?$AAa?$AAm?$AAe?$AA?5?$AAu?$AAn?$AAk?$AAn?$AAo?$AAw?$AAn?$AA?$DO?$AA?$AA@ 00141e40     LIBCMTD:dbgrpt.obj
 0002:00014e70       ??_C@_1CK@DDKKOLAN@?$AAs?$AAi?$AAz?$AAe?$AAI?$AAn?$AAB?$AAy?$AAt?$AAe?$AAs?$AA?5?$AA?$DO?$AA?$DN?$AA?5?$AAc?$AAo?$AAu?$AAn?$AAt?$AA?$AA@ 00141e70     LIBCMTD:memmove_s.obj
 0002:00014e9c       ??_C@_1BI@DCHLDCPP@?$AAs?$AAr?$AAc?$AA?5?$AA?$CB?$AA?$DN?$AA?5?$AAN?$AAU?$AAL?$AAL?$AA?$AA@ 00141e9c     LIBCMTD:memmove_s.obj
 0002:00014eb4       ??_C@_1BE@NMKKBGPA@?$AAm?$AAe?$AAm?$AAm?$AAo?$AAv?$AAe?$AA_?$AAs?$AA?$AA@ 00141eb4     LIBCMTD:memmove_s.obj
 0002:00014ec8       ??_C@_1FM@JMDLOEFB@?$AAf?$AA?3?$AA?2?$AAs?$AAp?$AA?2?$AAv?$AAc?$AAt?$AAo?$AAo?$AAl?$AAs?$AA?2?$AAc?$AAr?$AAt?$AAc?$AAe?$AA?2?$AAc?$AAr?$AAt?$AAw?$AA3?$AA2?$AA?2?$AAs?$AAt?$AAr?$AAi?$AAn@ 00141ec8     LIBCMTD:memmove_s.obj
 0002:00014f24       ??_C@_1BI@GKKCBDMD@?$AAd?$AAs?$AAt?$AA?5?$AA?$CB?$AA?$DN?$AA?5?$AAN?$AAU?$AAL?$AAL?$AA?$AA@ 00141f24     LIBCMTD:memmove_s.obj
 0002:00014f3c       ??_C@_1DM@MADKGDLO@?$AA?$CI?$AAL?$AA?$CC?$AAB?$AAu?$AAf?$AAf?$AAe?$AAr?$AA?5?$AAi?$AAs?$AA?5?$AAt?$AAo?$AAo?$AA?5?$AAs?$AAm?$AAa?$AAl?$AAl?$AA?$CC?$AA?5?$AA?$CG?$AA?$CG?$AA?5?$AA0?$AA?$CJ?$AA?$AA@ 00141f3c     LIBCMTD:wcscpy_s.obj
 0002:00014f78       ??_C@_1CI@HCPHDDLE@?$AAB?$AAu?$AAf?$AAf?$AAe?$AAr?$AA?5?$AAi?$AAs?$AA?5?$AAt?$AAo?$AAo?$AA?5?$AAs?$AAm?$AAa?$AAl?$AAl?$AA?$AA@ 00141f78     LIBCMTD:wcscpy_s.obj
 0002:00014fa0       ??_C@_1CG@OFBJMIGJ@?$AA?$CI?$AA?$CI?$AA?$CI?$AA_?$AAS?$AAr?$AAc?$AA?$CJ?$AA?$CJ?$AA?$CJ?$AA?5?$AA?$CB?$AA?$DN?$AA?5?$AAN?$AAU?$AAL?$AAL?$AA?$AA@ 00141fa0     LIBCMTD:wcscpy_s.obj
 0002:00014fc8       ??_C@_1BC@KIONAFPO@?$AAw?$AAc?$AAs?$AAc?$AAp?$AAy?$AA_?$AAs?$AA?$AA@ 00141fc8     LIBCMTD:wcscpy_s.obj
 0002:00014fe0       ??_C@_1FE@IPADLOPJ@?$AAf?$AA?3?$AA?2?$AAs?$AAp?$AA?2?$AAv?$AAc?$AAt?$AAo?$AAo?$AAl?$AAs?$AA?2?$AAc?$AAr?$AAt?$AAc?$AAe?$AA?2?$AAc?$AAr?$AAt?$AAw?$AA3?$AA2?$AA?2?$AAh?$AA?2?$AAt?$AAc?$AAs@ 00141fe0     LIBCMTD:wcscpy_s.obj
 0002:00015038       ??_C@_1FC@PFMLEHKI@?$AA?$CI?$AA?$CI?$AA_?$AAD?$AAs?$AAt?$AA?$CJ?$AA?$CJ?$AA?5?$AA?$CB?$AA?$DN?$AA?5?$AAN?$AAU?$AAL?$AAL?$AA?5?$AA?$CG?$AA?$CG?$AA?5?$AA?$CI?$AA?$CI?$AA_?$AAS?$AAi?$AAz?$AAe?$AAI?$AAn?$AAW?$AAo?$AAr@ 00142038     LIBCMTD:wcscpy_s.obj
 0002:0001508c       ??_C@_1BE@PMMBFFCC@?$AAw?$AAc?$AAs?$AAn?$AAc?$AAp?$AAy?$AA_?$AAs?$AA?$AA@ 0014208c     LIBCMTD:wcsncpy_s.obj
 0002:000150a0       ??_C@_1FG@OHHBDIEA@?$AAf?$AA?3?$AA?2?$AAs?$AAp?$AA?2?$AAv?$AAc?$AAt?$AAo?$AAo?$AAl?$AAs?$AA?2?$AAc?$AAr?$AAt?$AAc?$AAe?$AA?2?$AAc?$AAr?$AAt?$AAw?$AA3?$AA2?$AA?2?$AAh?$AA?2?$AAt?$AAc?$AAs@ 001420a0     LIBCMTD:wcsncpy_s.obj
 0002:000150f8       ??_C@_0BJ@IPHDMCNM@fatal?5error?5in?5_lock?5?$CD0?6?$AA@ 001420f8     LIBCMTD:mlock.obj
 0002:00015118       ??_C@_1NK@LOFHIHFC@?$AAf?$AAM?$AAo?$AAd?$AAe?$AA?5?$AA?$DN?$AA?$DN?$AA?5?$AA_?$AAC?$AAR?$AAT?$AAD?$AAB?$AAG?$AA_?$AAR?$AAE?$AAP?$AAO?$AAR?$AAT?$AA_?$AAM?$AAO?$AAD?$AAE?$AA?5?$AA?$HM?$AA?$HM?$AA?5@ 00142118     LIBCMTD:dbgrptt.obj
 0002:000151f4       ??_C@_1CE@FIHIECNJ@?$AA_?$AAC?$AAr?$AAt?$AAS?$AAe?$AAt?$AAR?$AAe?$AAp?$AAo?$AAr?$AAt?$AAM?$AAo?$AAd?$AAe?$AA?$AA@ 001421f4     LIBCMTD:dbgrptt.obj
 0002:00015218       ??_C@_1FE@PLIBPAGC@?$AAf?$AA?3?$AA?2?$AAs?$AAp?$AA?2?$AAv?$AAc?$AAt?$AAo?$AAo?$AAl?$AAs?$AA?2?$AAc?$AAr?$AAt?$AAc?$AAe?$AA?2?$AAc?$AAr?$AAt?$AAw?$AA3?$AA2?$AA?2?$AAm?$AAi?$AAs?$AAc?$AA?2@ 00142218     LIBCMTD:dbgrptt.obj
 0002:00015270       ??_C@_1FA@IFFFOLDJ@?$AAn?$AAR?$AAp?$AAt?$AAT?$AAy?$AAp?$AAe?$AA?5?$AA?$DO?$AA?$DN?$AA?5?$AA0?$AA?5?$AA?$CG?$AA?$CG?$AA?5?$AAn?$AAR?$AAp?$AAt?$AAT?$AAy?$AAp?$AAe?$AA?5?$AA?$DM?$AA?5?$AA_?$AAC?$AAR?$AAT@ 00142270     LIBCMTD:dbgrptt.obj
 0002:000152c0       ??_C@_1CE@IKKEDCME@?$AA_?$AAC?$AAr?$AAt?$AAS?$AAe?$AAt?$AAR?$AAe?$AAp?$AAo?$AAr?$AAt?$AAF?$AAi?$AAl?$AAe?$AA?$AA@ 001422c0     LIBCMTD:dbgrptt.obj
 0002:000152e8       ??_C@_1MA@LBAMNNOB@?$AAs?$AAt?$AAr?$AAc?$AAp?$AAy?$AA_?$AAs?$AA?$CI?$AAs?$AAz?$AAO?$AAu?$AAt?$AAM?$AAe?$AAs?$AAs?$AAa?$AAg?$AAe?$AA2?$AA?0?$AA?5?$AA4?$AA0?$AA9?$AA6?$AA?0?$AA?5?$AA?$CC?$AA_@ 001422e8     LIBCMTD:dbgrptt.obj
 0002:000153a8       ??_C@_0DP@GNPEPHJD@_CrtDbgReport?3?5String?5too?5long?5o@ 001423a8     LIBCMTD:dbgrptt.obj
 0002:000153e8       ??_C@_1FI@DBAIJPJE@?$AAw?$AAc?$AAs?$AAc?$AAp?$AAy?$AA_?$AAs?$AA?$CI?$AAs?$AAz?$AAO?$AAu?$AAt?$AAM?$AAe?$AAs?$AAs?$AAa?$AAg?$AAe?$AA?0?$AA?5?$AA4?$AA0?$AA9?$AA6?$AA?0?$AA?5?$AAs?$AAz?$AAL@ 001423e8     LIBCMTD:dbgrptt.obj
 0002:00015440       ??_C@_1BI@JIDBEPIG@?$AA?$CF?$AAs?$AA?$CI?$AA?$CF?$AAd?$AA?$CJ?$AA?5?$AA?3?$AA?5?$AA?$CF?$AAs?$AA?$AA@ 00142440     LIBCMTD:dbgrptt.obj
 0002:00015458       ??_C@_1EK@PHCBEDKB@?$AAw?$AAc?$AAs?$AAc?$AAa?$AAt?$AA_?$AAs?$AA?$CI?$AAs?$AAz?$AAL?$AAi?$AAn?$AAe?$AAM?$AAe?$AAs?$AAs?$AAa?$AAg?$AAe?$AA?0?$AA?5?$AA4?$AA0?$AA9?$AA6?$AA?0?$AA?5?$AAL?$AA?$CC@ 00142458     LIBCMTD:dbgrptt.obj
 0002:000154a8       ??_C@_1EK@NMDFGHMF@?$AAw?$AAc?$AAs?$AAc?$AAa?$AAt?$AA_?$AAs?$AA?$CI?$AAs?$AAz?$AAL?$AAi?$AAn?$AAe?$AAM?$AAe?$AAs?$AAs?$AAa?$AAg?$AAe?$AA?0?$AA?5?$AA4?$AA0?$AA9?$AA6?$AA?0?$AA?5?$AAL?$AA?$CC@ 001424a8     LIBCMTD:dbgrptt.obj
 0002:000154f4       ??_C@_13CMNBPIDO@?$AA?$AN?$AA?$AA@ 001424f4     LIBCMTD:dbgrptt.obj
 0002:000154f8       ??_C@_1FK@HPADHBBD@?$AAw?$AAc?$AAs?$AAc?$AAa?$AAt?$AA_?$AAs?$AA?$CI?$AAs?$AAz?$AAL?$AAi?$AAn?$AAe?$AAM?$AAe?$AAs?$AAs?$AAa?$AAg?$AAe?$AA?0?$AA?5?$AA4?$AA0?$AA9?$AA6?$AA?0?$AA?5?$AAs?$AAz@ 001424f8     LIBCMTD:dbgrptt.obj
 0002:00015558       ??_C@_1KO@DGAHENCH@?$AAw?$AAc?$AAs?$AAc?$AAp?$AAy?$AA_?$AAs?$AA?$CI?$AAs?$AAz?$AAL?$AAi?$AAn?$AAe?$AAM?$AAe?$AAs?$AAs?$AAa?$AAg?$AAe?$AA?0?$AA?5?$AA4?$AA0?$AA9?$AA6?$AA?0?$AA?5?$AAs?$AAz@ 00142558     LIBCMTD:dbgrptt.obj
 0002:00015608       ??_C@_1CE@OJBNHDMO@?$AAA?$AAs?$AAs?$AAe?$AAr?$AAt?$AAi?$AAo?$AAn?$AA?5?$AAf?$AAa?$AAi?$AAl?$AAe?$AAd?$AA?$CB?$AA?$AA@ 00142608     LIBCMTD:dbgrptt.obj
 0002:0001562c       ??_C@_1CG@FFFGGODN@?$AAA?$AAs?$AAs?$AAe?$AAr?$AAt?$AAi?$AAo?$AAn?$AA?5?$AAf?$AAa?$AAi?$AAl?$AAe?$AAd?$AA?3?$AA?5?$AA?$AA@ 0014262c     LIBCMTD:dbgrptt.obj
 0002:00015658       ??_C@_1JK@KHFABAEO@?$AAw?$AAc?$AAs?$AAc?$AAp?$AAy?$AA_?$AAs?$AA?$CI?$AAs?$AAz?$AAU?$AAs?$AAe?$AAr?$AAM?$AAe?$AAs?$AAs?$AAa?$AAg?$AAe?$AA?0?$AA?5?$AA4?$AA0?$AA9?$AA6?$AA?0?$AA?5?$AAL?$AA?$CC@ 00142658     LIBCMTD:dbgrptt.obj
 0002:000156f4       ??_C@_1BA@ELMMDCFC@?$AA?0?$AA?5?$AAL?$AAi?$AAn?$AAe?$AA?5?$AA?$AA@ 001426f4     LIBCMTD:dbgrptt.obj
 0002:00015704       ??_C@_1BO@OCHMLCAG@?$AA?$DM?$AAf?$AAi?$AAl?$AAe?$AA?5?$AAu?$AAn?$AAk?$AAn?$AAo?$AAw?$AAn?$AA?$DO?$AA?$AA@ 00142704     LIBCMTD:dbgrptt.obj
 0002:00015728       ??_C@_1EM@MJFLEDMB@?$AAS?$AAe?$AAc?$AAo?$AAn?$AAd?$AA?5?$AAC?$AAh?$AAa?$AAn?$AAc?$AAe?$AA?5?$AAA?$AAs?$AAs?$AAe?$AAr?$AAt?$AAi?$AAo?$AAn?$AA?5?$AAF?$AAa?$AAi?$AAl?$AAe?$AAd?$AA?3?$AA?5@ 00142728     LIBCMTD:dbgrptt.obj
 0002:00015778       ??_C@_1FA@CNLLOMHI@?$AA_?$AAi?$AAt?$AAo?$AAw?$AA_?$AAs?$AA?$CI?$AAn?$AAL?$AAi?$AAn?$AAe?$AA?0?$AA?5?$AAs?$AAz?$AAL?$AAi?$AAn?$AAe?$AAM?$AAe?$AAs?$AAs?$AAa?$AAg?$AAe?$AA?0?$AA?5?$AA4?$AA0@ 00142778     LIBCMTD:dbgrptt.obj
 0002:000157c8       ??_C@_1CA@HPALHDOD@?$AA_?$AAV?$AAC?$AAr?$AAt?$AAD?$AAb?$AAg?$AAR?$AAe?$AAp?$AAo?$AAr?$AAt?$AAW?$AA?$AA@ 001427c8     LIBCMTD:dbgrptt.obj
 0002:000157e8       ??_C@_1CG@MKBKDNCP@?$AAG?$AAe?$AAt?$AAL?$AAa?$AAs?$AAt?$AAA?$AAc?$AAt?$AAi?$AAv?$AAe?$AAP?$AAo?$AAp?$AAu?$AAp?$AA?$AA@ 001427e8     LIBCMTD:crtmbox.obj
 0002:00015810       ??_C@_1CA@HNKPMKAN@?$AAG?$AAe?$AAt?$AAA?$AAc?$AAt?$AAi?$AAv?$AAe?$AAW?$AAi?$AAn?$AAd?$AAo?$AAw?$AA?$AA@ 00142810     LIBCMTD:crtmbox.obj
 0002:00015830       ??_C@_1BI@OGPGOOGK@?$AAM?$AAe?$AAs?$AAs?$AAa?$AAg?$AAe?$AAB?$AAo?$AAx?$AAW?$AA?$AA@ 00142830     LIBCMTD:crtmbox.obj
 0002:00015848       ??_C@_1BI@IENOMFML@?$AAC?$AAO?$AAR?$AAE?$AAD?$AAL?$AAL?$AA?4?$AAD?$AAL?$AAL?$AA?$AA@ 00142848     LIBCMTD:crtmbox.obj
 0002:00015860       ??_C@_1BC@CFJEPFGF@?$AAs?$AAt?$AAr?$AAc?$AAp?$AAy?$AA_?$AAs?$AA?$AA@ 00142860     LIBCMTD:strcpy_s.obj
 0002:00015878       ??_C@_1FC@NCPEPIBI@?$AA?$CI?$AA?$CI?$AA_?$AAD?$AAs?$AAt?$AA?$CJ?$AA?$CJ?$AA?5?$AA?$CB?$AA?$DN?$AA?5?$AAN?$AAU?$AAL?$AAL?$AA?5?$AA?$CG?$AA?$CG?$AA?5?$AA?$CI?$AA?$CI?$AA_?$AAS?$AAi?$AAz?$AAe?$AAI?$AAn?$AAB?$AAy?$AAt@ 00142878     LIBCMTD:strcpy_s.obj
 0002:000158d0       ??_C@_1FA@MJKDNFFB@?$AA?$CI?$AAL?$AA?$CC?$AAS?$AAt?$AAr?$AAi?$AAn?$AAg?$AA?5?$AAi?$AAs?$AA?5?$AAn?$AAo?$AAt?$AA?5?$AAn?$AAu?$AAl?$AAl?$AA?5?$AAt?$AAe?$AAr?$AAm?$AAi?$AAn?$AAa?$AAt?$AAe?$AAd@ 001428d0     LIBCMTD:wcscat_s.obj
 0002:00015920       ??_C@_1DM@FHLMIEG@?$AAS?$AAt?$AAr?$AAi?$AAn?$AAg?$AA?5?$AAi?$AAs?$AA?5?$AAn?$AAo?$AAt?$AA?5?$AAn?$AAu?$AAl?$AAl?$AA?5?$AAt?$AAe?$AAr?$AAm?$AAi?$AAn?$AAa?$AAt?$AAe?$AAd?$AA?$AA@ 00142920     LIBCMTD:wcscat_s.obj
 0002:0001595c       ??_C@_1BC@PLIEPKPJ@?$AAw?$AAc?$AAs?$AAc?$AAa?$AAt?$AA_?$AAs?$AA?$AA@ 0014295c     LIBCMTD:wcscat_s.obj
 0002:00015970       ??_C@_1FE@EHLIBGFJ@?$AAf?$AA?3?$AA?2?$AAs?$AAp?$AA?2?$AAv?$AAc?$AAt?$AAo?$AAo?$AAl?$AAs?$AA?2?$AAc?$AAr?$AAt?$AAc?$AAe?$AA?2?$AAc?$AAr?$AAt?$AAw?$AA3?$AA2?$AA?2?$AAh?$AA?2?$AAt?$AAc?$AAs@ 00142970     LIBCMTD:wcscat_s.obj
 0002:000159c4       ??_C@_1CM@HABGDNLJ@?$AAl?$AAe?$AAn?$AAg?$AAt?$AAh?$AA?5?$AA?$DM?$AA?5?$AAs?$AAi?$AAz?$AAe?$AAI?$AAn?$AAT?$AAC?$AAh?$AAa?$AAr?$AAs?$AA?$AA@ 001429c4     LIBCMTD:xtows.obj
 0002:000159f0       ??_C@_1DE@PCJGDBBD@?$AA2?$AA?5?$AA?$DM?$AA?$DN?$AA?5?$AAr?$AAa?$AAd?$AAi?$AAx?$AA?5?$AA?$CG?$AA?$CG?$AA?5?$AAr?$AAa?$AAd?$AAi?$AAx?$AA?5?$AA?$DM?$AA?$DN?$AA?5?$AA3?$AA6?$AA?$AA@ 001429f0     LIBCMTD:xtows.obj
 0002:00015a28       ??_C@_1FA@MKGGAGEI@?$AAs?$AAi?$AAz?$AAe?$AAI?$AAn?$AAT?$AAC?$AAh?$AAa?$AAr?$AAs?$AA?5?$AA?$DO?$AA?5?$AA?$CI?$AAs?$AAi?$AAz?$AAe?$AA_?$AAt?$AA?$CJ?$AA?$CI?$AAi?$AAs?$AA_?$AAn?$AAe?$AAg?$AA?5?$AA?$DP@ 00142a28     LIBCMTD:xtows.obj
 0002:00015a78       ??_C@_1CC@JNJFIMGE@?$AAs?$AAi?$AAz?$AAe?$AAI?$AAn?$AAT?$AAC?$AAh?$AAa?$AAr?$AAs?$AA?5?$AA?$DO?$AA?5?$AA0?$AA?$AA@ 00142a78     LIBCMTD:xtows.obj
 0002:00015a9c       ??_C@_1O@NCBFODOE@?$AAx?$AAt?$AAo?$AAw?$AA_?$AAs?$AA?$AA@ 00142a9c     LIBCMTD:xtows.obj
 0002:00015ab0       ??_C@_1FE@LAGNOOBA@?$AAf?$AA?3?$AA?2?$AAs?$AAp?$AA?2?$AAv?$AAc?$AAt?$AAo?$AAo?$AAl?$AAs?$AA?2?$AAc?$AAr?$AAt?$AAc?$AAe?$AA?2?$AAc?$AAr?$AAt?$AAw?$AA3?$AA2?$AA?2?$AAc?$AAo?$AAn?$AAv?$AAe@ 00142ab0     LIBCMTD:xtows.obj
 0002:00015b04       ??_C@_1BI@ICGGMGLK@?$AAb?$AAu?$AAf?$AA?5?$AA?$CB?$AA?$DN?$AA?5?$AAN?$AAU?$AAL?$AAL?$AA?$AA@ 00142b04     LIBCMTD:xtows.obj
 0002:00015b1c       IID_IPersistStream         00142b1c     uuid:objidl_i_guid12.obj
 0002:00015cec       _TI1?AVCAtlException@ATL@@ 00142cec     atlsd:Externs.obj
 0002:00015cfc       _CTA1?AVCAtlException@ATL@@ 00142cfc     atlsd:Externs.obj
 0002:00015d04       _CT??_R0?AVCAtlException@ATL@@@84 00142d04     atlsd:Externs.obj
 0002:00015d20       __pobjMapEntryFirst        00142d20     stdafx.obj
 0002:00015d24       __pobjMapEntryLast         00142d24     stdafx.obj
 0002:00015d28       __IMPORT_DESCRIPTOR_COREDLL 00142d28     coredll:COREDLL.dll
 0002:00015d3c       __IMPORT_DESCRIPTOR_ril    00142d3c     ril:ril.dll
 0002:00015d50       __IMPORT_DESCRIPTOR_WS2    00142d50     ws2:WS2.dll
 0002:00015d64       __IMPORT_DESCRIPTOR_ole32  00142d64     ole32:ole32.dll
 0002:00015d78       __NULL_IMPORT_DESCRIPTOR   00142d78     coredll:COREDLL.dll
 0003:00000000       __imp_memcpy               00145000     coredll:COREDLL.dll
 0003:00000004       __imp_GetModuleFileNameW   00145004     coredll:COREDLL.dll
 0003:00000008       __imp_??3@YAXPAX@Z         00145008     coredll:COREDLL.dll
 0003:0000000c       __imp_GetFileVersionInfoW  0014500c     coredll:COREDLL.dll
 0003:00000010       __imp_??2@YAPAXI@Z         00145010     coredll:COREDLL.dll
 0003:00000014       __imp_GetFileVersionInfoSizeW 00145014     coredll:COREDLL.dll
 0003:00000018       __imp_wcscpy               00145018     coredll:COREDLL.dll
 0003:0000001c       __imp_OutputDebugStringW   0014501c     coredll:COREDLL.dll
 0003:00000020       __imp_swprintf             00145020     coredll:COREDLL.dll
 0003:00000024       __imp_VerQueryValueW       00145024     coredll:COREDLL.dll
 0003:00000028       __imp_wcscat               00145028     coredll:COREDLL.dll
 0003:0000002c       __imp_CreateEventW         0014502c     coredll:COREDLL.dll
 0003:00000030       __imp_RegisterWindowMessageW 00145030     coredll:COREDLL.dll
 0003:00000034       __imp_CloseHandle          00145034     coredll:COREDLL.dll
 0003:00000038       __imp_WaitForSingleObject  00145038     coredll:COREDLL.dll
 0003:0000003c       __imp_CreateThread         0014503c     coredll:COREDLL.dll
 0003:00000040       __imp_EventModify          00145040     coredll:COREDLL.dll
 0003:00000044       __imp_PostMessageW         00145044     coredll:COREDLL.dll
 0003:00000048       __imp___rt_udiv            00145048     coredll:COREDLL.dll
 0003:0000004c       __imp_wsprintfW            0014504c     coredll:COREDLL.dll
 0003:00000050       __imp_EnterCriticalSection 00145050     coredll:COREDLL.dll
 0003:00000054       __imp_LeaveCriticalSection 00145054     coredll:COREDLL.dll
 0003:00000058       __imp_wcslen               00145058     coredll:COREDLL.dll
 0003:0000005c       __imp_strcpy               0014505c     coredll:COREDLL.dll
 0003:00000060       __imp_memset               00145060     coredll:COREDLL.dll
 0003:00000064       __imp_wcsncpy              00145064     coredll:COREDLL.dll
 0003:00000068       __imp_strlen               00145068     coredll:COREDLL.dll
 0003:0000006c       __imp_InitializeCriticalSection 0014506c     coredll:COREDLL.dll
 0003:00000070       __imp_DeleteCriticalSection 00145070     coredll:COREDLL.dll
 0003:00000074       __imp_UnregisterClassW     00145074     coredll:COREDLL.dll
 0003:00000078       __imp_free                 00145078     coredll:COREDLL.dll
 0003:0000007c       __imp_RaiseException       0014507c     coredll:COREDLL.dll
 0003:00000080       __imp_CloseMsgQueue        00145080     coredll:COREDLL.dll
 0003:00000084       __imp_TerminateThread      00145084     coredll:COREDLL.dll
 0003:00000088       __imp_WriteMsgQueue        00145088     coredll:COREDLL.dll
 0003:0000008c       __imp_CreateMsgQueue       0014508c     coredll:COREDLL.dll
 0003:00000090       __imp_Sleep                00145090     coredll:COREDLL.dll
 0003:00000094       __imp_ReleaseMutex         00145094     coredll:COREDLL.dll
 0003:00000098       __imp_GetLastError         00145098     coredll:COREDLL.dll
 0003:0000009c       __imp_CreateMutexW         0014509c     coredll:COREDLL.dll
 0003:000000a0       __imp__wcslwr              001450a0     coredll:COREDLL.dll
 0003:000000a4       __imp_wcscmp               001450a4     coredll:COREDLL.dll
 0003:000000a8       __imp_GetLocalTime         001450a8     coredll:COREDLL.dll
 0003:000000ac       __imp_NKDbgPrintfW         001450ac     coredll:COREDLL.dll
 0003:000000b0       __imp_vswprintf            001450b0     coredll:COREDLL.dll
 0003:000000b4       __imp_DeleteFileW          001450b4     coredll:COREDLL.dll
 0003:000000b8       __imp_PurgeComm            001450b8     coredll:COREDLL.dll
 0003:000000bc       __imp_SetCommMask          001450bc     coredll:COREDLL.dll
 0003:000000c0       __imp_SetCommTimeouts      001450c0     coredll:COREDLL.dll
 0003:000000c4       __imp_SetCommState         001450c4     coredll:COREDLL.dll
 0003:000000c8       __imp_GetCommState         001450c8     coredll:COREDLL.dll
 0003:000000cc       __imp_ReadMsgQueue         001450cc     coredll:COREDLL.dll
 0003:000000d0       __imp_SetFilePointer       001450d0     coredll:COREDLL.dll
 0003:000000d4       __imp_CreateFileW          001450d4     coredll:COREDLL.dll
 0003:000000d8       __imp_DefWindowProcW       001450d8     coredll:COREDLL.dll
 0003:000000dc       __imp_PostQuitMessage      001450dc     coredll:COREDLL.dll
 0003:000000e0       __imp_FlushFileBuffers     001450e0     coredll:COREDLL.dll
 0003:000000e4       __imp_WriteFile            001450e4     coredll:COREDLL.dll
 0003:000000e8       __imp_CopyFileW            001450e8     coredll:COREDLL.dll
 0003:000000ec       __imp_GetFileSize          001450ec     coredll:COREDLL.dll
 0003:000000f0       __imp_MessageBoxW          001450f0     coredll:COREDLL.dll
 0003:000000f4       __imp_wcsstr               001450f4     coredll:COREDLL.dll
 0003:000000f8       __imp_GlobalMemoryStatus   001450f8     coredll:COREDLL.dll
 0003:000000fc       __imp_GetStoreInformation  001450fc     coredll:COREDLL.dll
 0003:00000100       __imp_MessageBeep          00145100     coredll:COREDLL.dll
 0003:00000104       __imp_rand                 00145104     coredll:COREDLL.dll
 0003:00000108       __imp_RegDeleteKeyW        00145108     coredll:COREDLL.dll
 0003:0000010c       __imp_RegEnumKeyExW        0014510c     coredll:COREDLL.dll
 0003:00000110       __imp_RegCloseKey          00145110     coredll:COREDLL.dll
 0003:00000114       __imp_RegCreateKeyExW      00145114     coredll:COREDLL.dll
 0003:00000118       __imp_RegOpenKeyExW        00145118     coredll:COREDLL.dll
 0003:0000011c       __imp_RegQueryValueExW     0014511c     coredll:COREDLL.dll
 0003:00000120       __imp_RegSetValueExW       00145120     coredll:COREDLL.dll
 0003:00000124       __imp_RegEnumValueW        00145124     coredll:COREDLL.dll
 0003:00000128       __imp_wcschr               00145128     coredll:COREDLL.dll
 0003:0000012c       __imp_GetVersionExW        0014512c     coredll:COREDLL.dll
 0003:00000130       __imp__wcsicmp             00145130     coredll:COREDLL.dll
 0003:00000134       __imp__wtol                00145134     coredll:COREDLL.dll
 0003:00000138       __imp___rt_sdiv            00145138     coredll:COREDLL.dll
 0003:0000013c       __imp_mbstowcs             0014513c     coredll:COREDLL.dll
 0003:00000140       __imp_wcstombs             00145140     coredll:COREDLL.dll
 0003:00000144       __imp_EndDeferWindowPos    00145144     coredll:COREDLL.dll
 0003:00000148       __imp_DeferWindowPos       00145148     coredll:COREDLL.dll
 0003:0000014c       __imp_MapDialogRect        0014514c     coredll:COREDLL.dll
 0003:00000150       __imp_GetDlgItem           00145150     coredll:COREDLL.dll
 0003:00000154       __imp_BeginDeferWindowPos  00145154     coredll:COREDLL.dll
 0003:00000158       __imp_LoadResource         00145158     coredll:COREDLL.dll
 0003:0000015c       __imp_FindResourceW        0014515c     coredll:COREDLL.dll
 0003:00000160       __imp_SetDlgItemTextW      00145160     coredll:COREDLL.dll
 0003:00000164       __imp_DeleteObject         00145164     coredll:COREDLL.dll
 0003:00000168       __imp_LoadBitmapW          00145168     coredll:COREDLL.dll
 0003:0000016c       __imp_DestroyIcon          0014516c     coredll:COREDLL.dll
 0003:00000170       __imp_LoadIconW            00145170     coredll:COREDLL.dll
 0003:00000174       __imp_SendDlgItemMessageW  00145174     coredll:COREDLL.dll
 0003:00000178       __imp_GetSystemMetrics     00145178     coredll:COREDLL.dll
 0003:0000017c       __imp_SendMessageW         0014517c     coredll:COREDLL.dll
 0003:00000180       __imp_FreeLibrary          00145180     coredll:COREDLL.dll
 0003:00000184       __imp_GetProcAddressW      00145184     coredll:COREDLL.dll
 0003:00000188       __imp_LoadLibraryW         00145188     coredll:COREDLL.dll
 0003:0000018c       __imp_RegDeleteValueW      0014518c     coredll:COREDLL.dll
 0003:00000190       __imp_SetCursor            00145190     coredll:COREDLL.dll
 0003:00000194       __imp_LoadCursorW          00145194     coredll:COREDLL.dll
 0003:00000198       __imp_FileTimeToSystemTime 00145198     coredll:COREDLL.dll
 0003:0000019c       __imp_LocalFileTimeToFileTime 0014519c     coredll:COREDLL.dll
 0003:000001a0       __imp_SystemTimeToFileTime 001451a0     coredll:COREDLL.dll
 0003:000001a4       __imp_TerminateProcess     001451a4     coredll:COREDLL.dll
 0003:000001a8       __imp_SetLastError         001451a8     coredll:COREDLL.dll
 0003:000001ac       __imp_TlsCall              001451ac     coredll:COREDLL.dll
 0003:000001b0       __imp_InterlockedCompareExchange 001451b0     coredll:COREDLL.dll
 0003:000001b4       __imp_TlsGetValue          001451b4     coredll:COREDLL.dll
 0003:000001b8       __imp_TlsSetValue          001451b8     coredll:COREDLL.dll
 0003:000001bc       __imp_malloc               001451bc     coredll:COREDLL.dll
 0003:000001c0       __imp_memmove              001451c0     coredll:COREDLL.dll
 0003:000001c4       __imp_?terminate@std@@YAXXZ 001451c4     coredll:COREDLL.dll
 0003:000001c8       __imp_strcmp               001451c8     coredll:COREDLL.dll
 0003:000001cc       __imp_InterlockedDecrement 001451cc     coredll:COREDLL.dll
 0003:000001d0       __imp_InterlockedIncrement 001451d0     coredll:COREDLL.dll
 0003:000001d4       __imp_CreateFileMappingW   001451d4     coredll:COREDLL.dll
 0003:000001d8       __imp_MapViewOfFile        001451d8     coredll:COREDLL.dll
 0003:000001dc       __imp_GetSystemInfo        001451dc     coredll:COREDLL.dll
 0003:000001e0       __imp_memcmp               001451e0     coredll:COREDLL.dll
 0003:000001e4       __imp_UnmapViewOfFile      001451e4     coredll:COREDLL.dll
 0003:000001e8       __imp_VirtualAlloc         001451e8     coredll:COREDLL.dll
 0003:000001ec       __imp__vsnwprintf          001451ec     coredll:COREDLL.dll
 0003:000001f0       __imp_OpenEventW           001451f0     coredll:COREDLL.dll
 0003:000001f4       __imp_??_7type_info@@6B@   001451f4     coredll:COREDLL.dll
 0003:000001f8       __imp___report_gsfailure   001451f8     coredll:COREDLL.dll
 0003:000001fc       __imp_LocalReAlloc         001451fc     coredll:COREDLL.dll
 0003:00000200       __imp_LocalAlloc           00145200     coredll:COREDLL.dll
 0003:00000204       __imp_LocalSize            00145204     coredll:COREDLL.dll
 0003:00000208       __imp_LocalFree            00145208     coredll:COREDLL.dll
 0003:0000020c       __imp_DisableThreadLibraryCalls 0014520c     coredll:COREDLL.dll
 0003:00000210       __imp___security_gen_cookie 00145210     coredll:COREDLL.dll
 0003:00000214       __imp_DispatchMessageW     00145214     coredll:COREDLL.dll
 0003:00000218       __imp_TranslateMessage     00145218     coredll:COREDLL.dll
 0003:0000021c       __imp_GetMessageW          0014521c     coredll:COREDLL.dll
 0003:00000220       __imp_PeekMessageW         00145220     coredll:COREDLL.dll
 0003:00000224       __imp_MsgWaitForMultipleObjectsEx 00145224     coredll:COREDLL.dll
 0003:00000228       __imp___C_specific_handler 00145228     coredll:COREDLL.dll
 0003:0000022c       __imp_GetModuleHandleW     0014522c     coredll:COREDLL.dll
 0003:00000230       __imp_realloc              00145230     coredll:COREDLL.dll
 0003:00000234       __imp__snwprintf           00145234     coredll:COREDLL.dll
 0003:00000238       __imp___CxxThrowException  00145238     coredll:COREDLL.dll
 0003:0000023c       \177COREDLL_NULL_THUNK_DATA 0014523c     coredll:COREDLL.dll
 0003:00000240       __imp_ntohl                00145240     ws2:WS2.dll
 0003:00000244       \177WS2_NULL_THUNK_DATA    00145244     ws2:WS2.dll
 0003:00000248       __imp_ReadClassStm         00145248     ole32:ole32.dll
 0003:0000024c       __imp_CoCreateInstance     0014524c     ole32:ole32.dll
 0003:00000250       __imp_WriteClassStm        00145250     ole32:ole32.dll
 0003:00000254       __imp_CreateStreamOnHGlobal 00145254     ole32:ole32.dll
 0003:00000258       \177ole32_NULL_THUNK_DATA  00145258     ole32:ole32.dll
 0003:0000025c       __imp_RIL_GetRoamingMode   0014525c     ril:ril.dll
 0003:00000260       __imp_RIL_GetPreferredPrivacyMode 00145260     ril:ril.dll
 0003:00000264       __imp_RIL_GetCallList      00145264     ril:ril.dll
 0003:00000268       __imp_RIL_GetCurrentSystemType 00145268     ril:ril.dll
 0003:0000026c       __imp_RIL_GetRegistrationStatus 0014526c     ril:ril.dll
 0003:00000270       __imp_RIL_Dial             00145270     ril:ril.dll
 0003:00000274       __imp_RIL_SetRoamingMode   00145274     ril:ril.dll
 0003:00000278       __imp_RIL_SetEquipmentState 00145278     ril:ril.dll
 0003:0000027c       __imp_RIL_GetUserIdentity  0014527c     ril:ril.dll
 0003:00000280       __imp_RIL_GetEquipmentInfo 00145280     ril:ril.dll
 0003:00000284       __imp_RIL_GetEquipmentState 00145284     ril:ril.dll
 0003:00000288       __imp_RIL_DevSpecific      00145288     ril:ril.dll
 0003:0000028c       __imp_RIL_Deinitialize     0014528c     ril:ril.dll
 0003:00000290       __imp_RIL_Initialize       00145290     ril:ril.dll
 0003:00000294       __imp_RIL_SetPreferredPrivacyMode 00145294     ril:ril.dll
 0003:00000298       __imp_RIL_SendAKey         00145298     ril:ril.dll
 0003:0000029c       __imp_RIL_GetPacketByteCount 0014529c     ril:ril.dll
 0003:000002a0       __imp_RIL_Hangup           001452a0     ril:ril.dll
 0003:000002a4       \177ril_NULL_THUNK_DATA    001452a4     ril:ril.dll
 0003:000002a8       __xc_a                     001452a8     corelibc:crt0init.obj
 0003:0000032c       __xc_z                     0014532c     corelibc:crt0init.obj
 0003:00000330       __xi_a                     00145330     corelibc:crt0init.obj
 0003:00000334       __xi_z                     00145334     corelibc:crt0init.obj
 0003:00000338       __xp_a                     00145338     corelibc:crt0init.obj
 0003:0000033c       __xp_z                     0014533c     corelibc:crt0init.obj
 0003:00000340       __xt_a                     00145340     corelibc:crt0init.obj
 0003:00000344       __xt_z                     00145344     corelibc:crt0init.obj
 0003:00000350       ?g_hLogOpenedBy1stApp@@3PAXA 00145350     SW_Log.obj
 0003:00000358       ?g_wszSetupSWIProxy@@3PBGB 00145358     Utilities.obj
 0003:0000035c       ?g_wszSetupGSMXml@@3PBGB   0014535c     Utilities.obj
 0003:00000360       ?g_wszSetupPCSXml@@3PBGB   00145360     Utilities.obj
 0003:00000364       ?g_wszSetupVZWXml@@3PBGB   00145364     Utilities.obj
 0003:00000368       ?g_wszRemoveGSMNetworkXml@@3PBGB 00145368     Utilities.obj
 0003:0000036c       ?g_wszRemoveGSMEntriesXml@@3PBGB 0014536c     Utilities.obj
 0003:00000370       ?g_wszRemovePCSNetworkXml@@3PBGB 00145370     Utilities.obj
 0003:00000374       ?g_wszRemovePCSEntriesXml@@3PBGB 00145374     Utilities.obj
 0003:00000378       ?g_wszRemoveVZWNetworkXml@@3PBGB 00145378     Utilities.obj
 0003:0000037c       ?g_wszRemoveVZWEntriesXml@@3PBGB 0014537c     Utilities.obj
 0003:00000380       __security_cookie_complement 00145380     corelibc:seccook.obj
 0003:00000384       __security_cookie          00145384     corelibc:seccook.obj
 0003:00000388       ?rcDefault@CWindow@ATL@@2UtagRECT@@A 00145388     atlsd:atlfuncs.obj
 0003:00000398       _pRawDllMain               00145398     atlsd:atlbase.obj
 0003:0000039c       ?g_pszUpdateEventName@@3PB_WB 0014539c     atlsd:Externs.obj
 0003:000003a0       ?g_pszAllocFileMapName@@3PB_WB 001453a0     atlsd:Externs.obj
 0003:000003a4       ?g_pszKernelObjFmt@@3PB_WB 001453a4     atlsd:Externs.obj
 0003:000003a8       ??_R0?AVCAtlException@ATL@@@8 001453a8     atlsd:Externs.obj
 0003:00000500       _crtAssertBusy             00145500     LIBCMTD:dbgrptt.obj
 0003:00000504       _CrtDbgMode                00145504     LIBCMTD:dbgrptt.obj
 0003:00000510       _CrtDbgFile                00145510     LIBCMTD:dbgrptt.obj
 0003:0000051c       _aexit_rtn                 0014551c     LIBCMTD:crt0dat.obj
 0003:00000520       ?RIL_STATUS_CHANGED@CModemStatus@@2IA 00145520     ModemStat.obj
 0003:00000524       ?RIL_DBG_NOTIFY@CModemStatus@@2IA 00145524     ModemStat.obj
 0003:00000528       ?RIL_TECHHDR_NOTIFY@CModemStatus@@2IA 00145528     ModemStat.obj
 0003:0000052c       ?RIL_IOTA_STATUS_CHANGED@CModemStatus@@2IA 0014552c     ModemStat.obj
 0003:00000530       ?RIL_IOTA_WAP_URI@CModemStatus@@2IA 00145530     ModemStat.obj
 0003:00000534       ?RIL_PDSM_PD_DATA@CModemStatus@@2IA 00145534     ModemStat.obj
 0003:00000538       ?RIL_PDSM_PD_DONE@CModemStatus@@2IA 00145538     ModemStat.obj
 0003:0000053c       ?RIL_PDSM_PD_END@CModemStatus@@2IA 0014553c     ModemStat.obj
 0003:00000540       ?RIL_PDSM_PD_BEGIN@CModemStatus@@2IA 00145540     ModemStat.obj
 0003:00000544       ?RIL_PDSM_PD_UPDATE_FAILURE@CModemStatus@@2IA 00145544     ModemStat.obj
 0003:00000548       ?RIL_PDSM_PD_DLD_DATA@CModemStatus@@2IA 00145548     ModemStat.obj
 0003:0000054c       ?RIL_PDSM_PD_DLD_DONE@CModemStatus@@2IA 0014554c     ModemStat.obj
 0003:00000550       ?RIL_PDSM_PD_DLD_END@CModemStatus@@2IA 00145550     ModemStat.obj
 0003:00000554       ?RIL_PDSM_PD_DLD_BEGIN@CModemStatus@@2IA 00145554     ModemStat.obj
 0003:00000558       ?RIL_PDSM_PA_PARAM@CModemStatus@@2IA 00145558     ModemStat.obj
 0003:0000055c       ?RIL_CALL_BYTE_CTR@CModemStatus@@2IA 0014555c     ModemStat.obj
 0003:00000560       ?gCommandCS@@3VCriticalSection@@A 00145560     ModemStat.obj
 0003:00000578       ?g_objModemStatus@@3VCModemStatus@@A 00145578     ModemStat.obj
 0003:00000b1c       ?m_bInitFailed@CAtlBaseModule@ATL@@2_NA 00145b1c     stdafx.obj
 0003:00000b20       ?_pPerfRegFunc@ATL@@3P6AJPAUHINSTANCE__@@@ZA 00145b20     stdafx.obj
 0003:00000b24       ?_pPerfUnRegFunc@ATL@@3P6AJXZA 00145b24     stdafx.obj
 0003:00000b28       ?_pAtlModule@ATL@@3PAVCAtlModule@1@A 00145b28     stdafx.obj
 0003:00000b2c       ?m_libid@CAtlModule@ATL@@2U_GUID@@A 00145b2c     stdafx.obj
 0003:00000b3c       ?_pModule@ATL@@3PAVCComModule@1@A 00145b3c     stdafx.obj
 0003:00000b40       ?_AtlWinModule@ATL@@3VCAtlWinModule@1@A 00145b40     stdafx.obj
 0003:00000b68       ?m_msgBoxText@SW_Log@@0PAGA 00145b68     SW_Log.obj
 0003:00001d78       ?g_MaxReachCount@@3KA      00146d78     SW_Log.obj
 0003:00001d80       ?g_Log@@3VSW_Log@@A        00146d80     SW_Log.obj
 0003:00001fc8       ?szOneLine@@3PAGA          00146fc8     SW_Log_Include.obj
 0003:000027c8       ?g_nLine@@3HA              001477c8     SW_Log_Include.obj
 0003:000027d0       ?g_szFile@@3PAGA           001477d0     SW_Log_Include.obj
 0003:000029d8       ?theSWIDisplayRawDataCR@@3VCriticalSection@@A 001479d8     SW_Log_Include.obj
 0003:000029f0       ?strFormatVer@@3PAGA       001479f0     Utilities.obj
 0003:00002bf8       ?g_dwOSMajVer@@3KA         00147bf8     Utilities.obj
 0003:00002e00       ?_pAtlRawDllMain@@3P6AHPAXK0@ZA 00147e00     atlsd:atlbase.obj
 0003:00002e04       ?_AtlModuleInstance@ATL@@3PAUHINSTANCE__@@A 00147e04     atlsd:atlbase.obj
 0003:00002e08       ?_AtlBaseModule@ATL@@3VCAtlBaseModule@1@A 00147e08     atlsd:atlbase.obj
 0003:00002e8c       ?atlTraceGeneral@ATL@@3VCTraceCategory@1@A 00147e8c     atlsd:atltrace.obj
 0003:00002e90       ?atlTraceCOM@ATL@@3VCTraceCategory@1@A 00147e90     atlsd:atltrace.obj
 0003:00002e94       ?atlTraceQI@ATL@@3VCTraceCategory@1@A 00147e94     atlsd:atltrace.obj
 0003:00002e98       ?atlTraceRegistrar@ATL@@3VCTraceCategory@1@A 00147e98     atlsd:atltrace.obj
 0003:00002e9c       ?atlTraceRefcount@ATL@@3VCTraceCategory@1@A 00147e9c     atlsd:atltrace.obj
 0003:00002ea0       ?atlTraceWindowing@ATL@@3VCTraceCategory@1@A 00147ea0     atlsd:atltrace.obj
 0003:00002ea4       ?atlTraceControls@ATL@@3VCTraceCategory@1@A 00147ea4     atlsd:atltrace.obj
 0003:00002ea8       ?atlTraceHosting@ATL@@3VCTraceCategory@1@A 00147ea8     atlsd:atltrace.obj
 0003:00002eac       ?atlTraceNotImpl@ATL@@3VCTraceCategory@1@A 00147eac     atlsd:atltrace.obj
 0003:00002eb0       ?atlTraceAllocation@ATL@@3VCTraceCategory@1@A 00147eb0     atlsd:atltrace.obj
 0003:00002eb4       ?atlTraceException@ATL@@3VCTraceCategory@1@A 00147eb4     atlsd:atltrace.obj
 0003:00002eb8       ?atlTraceTime@ATL@@3VCTraceCategory@1@A 00147eb8     atlsd:atltrace.obj
 0003:00002ebc       ?atlTraceCache@ATL@@3VCTraceCategory@1@A 00147ebc     atlsd:atltrace.obj
 0003:00002ec0       ?atlTraceStencil@ATL@@3VCTraceCategory@1@A 00147ec0     atlsd:atltrace.obj
 0003:00002ec4       ?atlTraceString@ATL@@3VCTraceCategory@1@A 00147ec4     atlsd:atltrace.obj
 0003:00002ec8       ?atlTraceMap@ATL@@3VCTraceCategory@1@A 00147ec8     atlsd:atltrace.obj
 0003:00002ecc       ?atlTraceUtil@ATL@@3VCTraceCategory@1@A 00147ecc     atlsd:atltrace.obj
 0003:00002ed0       ?atlTraceSync@ATL@@3VCTraceCategory@1@A 00147ed0     atlsd:atltrace.obj
 0003:00002ed4       ?atlTraceUser@ATL@@3VCTraceCategory@1@A 00147ed4     atlsd:atltrace.obj
 0003:00002ed8       ?atlTraceUser2@ATL@@3VCTraceCategory@1@A 00147ed8     atlsd:atltrace.obj
 0003:00002edc       ?atlTraceUser3@ATL@@3VCTraceCategory@1@A 00147edc     atlsd:atltrace.obj
 0003:00002ee0       ?atlTraceUser4@ATL@@3VCTraceCategory@1@A 00147ee0     atlsd:atltrace.obj
 0003:00002ee4       ?g_Allocator@@3VCAtlAllocator@@A 00147ee4     atlsd:Externs.obj
 0003:00002f18       ?s_trace@CTrace@ATL@@2V12@A 00147f18     atlsd:Externs.obj
 0003:00003068       __onexitend                00148068     <common>
 0003:0000306c       __onexitbegin              0014806c     <common>
 0003:00003070       _exitflag                  00148070     <common>
 0003:00003074       _pfnReportHook             00148074     <common>
 0003:00003078       _pReportHookListW          00148078     <common>
 0003:0000307c       _pReportHookList           0014807c     <common>

 entry point at        0001:0001a180

 Static symbols

 0001:000048ec       __unwind$35581             001058ec f   ModemStat.obj
 0001:00004b1c       __unwind$35638             00105b1c f   ModemStat.obj
 0001:00004cc4       __unwind$35663             00105cc4 f   ModemStat.obj
 0001:00004f14       __unwind$35688             00105f14 f   ModemStat.obj
 0001:000067f0       __unwind$35861             001077f0 f   ModemStat.obj
 0001:000069b8       __unwind$35887             001079b8 f   ModemStat.obj
 0001:00006b80       __unwind$35913             00107b80 f   ModemStat.obj
 0001:00006fb4       __unwind$35965             00107fb4 f   ModemStat.obj
 0001:00008ec0       __unwind$36191             00109ec0 f   ModemStat.obj
 0001:0000faa4       __unwind$47810             00110aa4 f i stdafx.obj
 0001:0000fb84       __unwind$47862             00110b84 f i stdafx.obj
 0001:0000fc34       __unwind$47897             00110c34 f i stdafx.obj
 0001:00012604       __unwind$46807             00113604 f   SW_Log_Include.obj
 0001:00012800       __unwind$47264             00113800 f   SW_Registrykey.obj
 0001:000129f8       __unwind$47297             001139f8 f   SW_Registrykey.obj
 0001:00012b9c       __unwind$47318             00113b9c f   SW_Registrykey.obj
 0001:00012ca0       __unwind$47337             00113ca0 f   SW_Registrykey.obj
 0001:00012db0       __unwind$47357             00113db0 f   SW_Registrykey.obj
 0001:00012ebc       __unwind$47377             00113ebc f   SW_Registrykey.obj
 0001:00013100       __unwind$47398             00114100 f   SW_Registrykey.obj
 0001:000133b8       __unwind$47428             001143b8 f   SW_Registrykey.obj
 0001:00013640       __unwind$47457             00114640 f   SW_Registrykey.obj
 0001:000137c8       __unwind$47484             001147c8 f   SW_Registrykey.obj
 0001:0001395c       __unwind$47510             0011495c f   SW_Registrykey.obj
 0001:00013aec       __unwind$47536             00114aec f   SW_Registrykey.obj
 0001:00013e84       __unwind$47564             00114e84 f   SW_Registrykey.obj
 0001:00013ea4       __unwind$47565             00114ea4 f   SW_Registrykey.obj
 0001:00013ecc       __unwind$47566             00114ecc f   SW_Registrykey.obj
 0001:00014154       __unwind$47614             00115154 f   SW_Registrykey.obj
 0001:0001416c       __unwind$47615             0011516c f   SW_Registrykey.obj
 0001:0001451c       __unwind$47652             0011551c f   SW_Registrykey.obj
 0001:00014544       __unwind$47653             00115544 f   SW_Registrykey.obj
 0001:0001456c       __unwind$47654             0011556c f   SW_Registrykey.obj
 0001:00014774       __unwind$47711             00115774 f   SW_Registrykey.obj
 0001:00015a7c       __unwind$47950             00116a7c f   SW_Registrykey.obj
 0001:00015a9c       __unwind$47951             00116a9c f   SW_Registrykey.obj
 0001:00015c48       __unwind$54019             00116c48 f   Utilities.obj
 0001:00017a68       ?FixupDialogItem@@YAXPAUHINSTANCE__@@PAUHWND__@@PAUDLGITEMTEMPLATE@@PAG3@Z 00118a68 f   Utilities.obj
 0001:00017d90       ?WalkDialogData@@YAPAEPAE@Z 00118d90 f   Utilities.obj
 0001:0001a344       _initterm                  0011b344 f   corelibc:crt0dat.obj
 0001:0001a3e4       doexit                     0011b3e4 f   corelibc:crt0dat.obj
 0001:0001ce2c       ?_ATLLoadOle32API@ATL@@YAP6AHXZPB_W@Z 0011de2c f   atlsd:atlbase.obj
 0001:0001ee70       ?Init@@YA_NXZ              0011fe70 f   atlsd:Externs.obj
 0001:00020eb8       ?ShouldTraceOutput@ATL@@YA_NKKIPAPBVCAtlTraceCategory@@PAP6AHHPB_WH11ZZ@Z 00121eb8 f   atlsd:AtlDebugAPI.obj
 0001:000240e0       ?FindHandler@@YAEPAUEHExceptionRecord@@PAKPAU_CONTEXT@@PAU_DISPATCHER_CONTEXT@@PBU_s_FuncInfo@@H@Z 001250e0 f   LIBCMTD:frame_ce.obj
 0001:000246d4       ?TypeMatch@@YAHPBU_s_HandlerType@@PBU_s_CatchableType@@PBU_s_ThrowInfo@@@Z 001256d4 f   LIBCMTD:frame_ce.obj
 0001:00024a98       ?FrameUnwindFilter@@YAHPAU_EXCEPTION_POINTERS@@@Z 00125a98 f   LIBCMTD:frame_ce.obj
 0001:00024b24       ?CallCatchBlock@@YAPAXPAUEHExceptionRecord@@PAKPAU_CONTEXT@@PBU_s_FuncInfo@@PAXHK@Z 00125b24 f   LIBCMTD:frame_ce.obj
 0001:000250c0       ?CanThisExceptionObjectBeDestructed@@YAEPAUEHExceptionRecord@@E@Z 001260c0 f   LIBCMTD:frame_ce.obj
 0001:0002534c       ?BuildCatchObject@@YAXPAUEHExceptionRecord@@PAKPBU_s_HandlerType@@PBU_s_CatchableType@@@Z 0012634c f   LIBCMTD:frame_ce.obj
 0001:0002569c       ?AdjustPointer@@YAPAXPAXABUPMD@@@Z 0012669c f   LIBCMTD:frame_ce.obj
 0001:000291f0       __crtInitCritSecNoSpinCount 0012a1f0 f   LIBCMTD:initcrit.obj
 0001:00029d88       xtow_s                     0012ad88 f   LIBCMTD:xtows.obj
 0001:0002a760       ??__EgCommandCS@@YAXXZ     0012b760 f   ModemStat.obj
 0001:0002a780       ??__Eg_objModemStatus@@YAXXZ 0012b780 f   ModemStat.obj
 0001:0002a7a0       ??__E_AtlWinModule@ATL@@YAXXZ 0012b7a0 f   stdafx.obj
 0001:0002a7c0       ??__Eg_Log@@YAXXZ          0012b7c0 f   SW_Log.obj
 0001:0002a7e0       ??__EtheSWIDisplayRawDataCR@@YAXXZ 0012b7e0 f   SW_Log_Include.obj
 0001:0002a800       ??__E_AtlWinModule@ATL@@YAXXZ 0012b800 f   atlsd:atlfuncs.obj
 0001:0002a83c       ??__E_AtlBaseModule@ATL@@YAXXZ 0012b83c f   atlsd:atlbase.obj
 0001:0002a878       ??__E_AtlWinModule@ATL@@YAXXZ 0012b878 f   atlsd:atlbase.obj
 0001:0002a8b4       ??__EatlTraceGeneral@ATL@@YAXXZ 0012b8b4 f   atlsd:atltrace.obj
 0001:0002a8e4       ??__EatlTraceCOM@ATL@@YAXXZ 0012b8e4 f   atlsd:atltrace.obj
 0001:0002a914       ??__EatlTraceQI@ATL@@YAXXZ 0012b914 f   atlsd:atltrace.obj
 0001:0002a944       ??__EatlTraceRegistrar@ATL@@YAXXZ 0012b944 f   atlsd:atltrace.obj
 0001:0002a974       ??__EatlTraceRefcount@ATL@@YAXXZ 0012b974 f   atlsd:atltrace.obj
 0001:0002a9a4       ??__EatlTraceWindowing@ATL@@YAXXZ 0012b9a4 f   atlsd:atltrace.obj
 0001:0002a9d4       ??__EatlTraceControls@ATL@@YAXXZ 0012b9d4 f   atlsd:atltrace.obj
 0001:0002aa04       ??__EatlTraceHosting@ATL@@YAXXZ 0012ba04 f   atlsd:atltrace.obj
 0001:0002aa34       ??__EatlTraceNotImpl@ATL@@YAXXZ 0012ba34 f   atlsd:atltrace.obj
 0001:0002aa64       ??__EatlTraceAllocation@ATL@@YAXXZ 0012ba64 f   atlsd:atltrace.obj
 0001:0002aa94       ??__EatlTraceException@ATL@@YAXXZ 0012ba94 f   atlsd:atltrace.obj
 0001:0002aac4       ??__EatlTraceTime@ATL@@YAXXZ 0012bac4 f   atlsd:atltrace.obj
 0001:0002aaf4       ??__EatlTraceCache@ATL@@YAXXZ 0012baf4 f   atlsd:atltrace.obj
 0001:0002ab24       ??__EatlTraceStencil@ATL@@YAXXZ 0012bb24 f   atlsd:atltrace.obj
 0001:0002ab54       ??__EatlTraceString@ATL@@YAXXZ 0012bb54 f   atlsd:atltrace.obj
 0001:0002ab84       ??__EatlTraceMap@ATL@@YAXXZ 0012bb84 f   atlsd:atltrace.obj
 0001:0002abb4       ??__EatlTraceUtil@ATL@@YAXXZ 0012bbb4 f   atlsd:atltrace.obj
 0001:0002abe4       ??__EatlTraceSync@ATL@@YAXXZ 0012bbe4 f   atlsd:atltrace.obj
 0001:0002ac14       ??__EatlTraceUser@ATL@@YAXXZ 0012bc14 f   atlsd:atltrace.obj
 0001:0002ac44       ??__EatlTraceUser2@ATL@@YAXXZ 0012bc44 f   atlsd:atltrace.obj
 0001:0002ac74       ??__EatlTraceUser3@ATL@@YAXXZ 0012bc74 f   atlsd:atltrace.obj
 0001:0002aca4       ??__EatlTraceUser4@ATL@@YAXXZ 0012bca4 f   atlsd:atltrace.obj
 0001:0002acd4       ??__E_AtlWinModule@ATL@@YAXXZ 0012bcd4 f   atlsd:atltrace.obj
 0001:0002ad10       ??__Eg_Allocator@@YAXXZ    0012bd10 f   atlsd:Externs.obj
 0001:0002ad4c       ??__Eg_bInitialized@@YAXXZ 0012bd4c f   atlsd:Externs.obj
 0001:0002ad84       ??__E?s_trace@CTrace@ATL@@2V12@A@@YAXXZ 0012bd84 f   atlsd:Externs.obj
 0001:0002adc8       ??__E_AtlWinModule@ATL@@YAXXZ 0012bdc8 f   atlsd:Externs.obj
 0001:0002ae04       ??__E_AtlWinModule@ATL@@YAXXZ 0012be04 f   atlsd:AtlDebugAPI.obj
 0001:0002ae40       ??__E_AtlWinModule@ATL@@YAXXZ 0012be40 f   atlsd:Allocate.obj
 0001:0002ae7c       ??__E_AtlWinModule@ATL@@YAXXZ 0012be7c f   atlsd:AtlTraceModuleManager.obj
 0001:0002aeb8       ??__FgCommandCS@@YAXXZ     0012beb8 f   ModemStat.obj
 0001:0002aecc       ??__Fg_objModemStatus@@YAXXZ 0012becc f   ModemStat.obj
 0001:0002aee0       ??__F_AtlWinModule@ATL@@YAXXZ 0012bee0 f   stdafx.obj
 0001:0002aef4       ??__Fg_Log@@YAXXZ          0012bef4 f   SW_Log.obj
 0001:0002af08       ??__FtheSWIDisplayRawDataCR@@YAXXZ 0012bf08 f   SW_Log_Include.obj
 0001:0002af1c       ??__F_AtlWinModule@ATL@@YAXXZ 0012bf1c f   atlsd:atlfuncs.obj
 0001:0002af40       ??__F_AtlBaseModule@ATL@@YAXXZ 0012bf40 f   atlsd:atlbase.obj
 0001:0002af64       ??__F_AtlWinModule@ATL@@YAXXZ 0012bf64 f   atlsd:atlbase.obj
 0001:0002af88       ??__F_AtlWinModule@ATL@@YAXXZ 0012bf88 f   atlsd:atltrace.obj
 0001:0002afac       ??__Fg_Allocator@@YAXXZ    0012bfac f   atlsd:Externs.obj
 0001:0002afd0       ??__F?s_trace@CTrace@ATL@@2V12@A@@YAXXZ 0012bfd0 f   atlsd:Externs.obj
 0001:0002aff4       ??__F_AtlWinModule@ATL@@YAXXZ 0012bff4 f   atlsd:Externs.obj
 0001:0002b018       ??__F_AtlWinModule@ATL@@YAXXZ 0012c018 f   atlsd:AtlDebugAPI.obj
 0001:0002b03c       ??__F_AtlWinModule@ATL@@YAXXZ 0012c03c f   atlsd:Allocate.obj
 0001:0002b060       ??__F_AtlWinModule@ATL@@YAXXZ 0012c060 f   atlsd:AtlTraceModuleManager.obj

 Exports

  ordinal    name

        1    ??0CVerInfo@@QAA@PAG@Z (public: __cdecl CVerInfo::CVerInfo(unsigned short *))
        2    ??0CVerInfo@@QAA@PAUHINSTANCE__@@@Z (public: __cdecl CVerInfo::CVerInfo(struct HINSTANCE__ *))
        3    ??0CVerInfo@@QAA@XZ (public: __cdecl CVerInfo::CVerInfo(void))
        4    ??0SW_RegistryKey@@QAA@ABV0@@Z (public: __cdecl SW_RegistryKey::SW_RegistryKey(class SW_RegistryKey const &))
        5    ??0SW_RegistryKey@@QAA@PAUHKEY__@@@Z (public: __cdecl SW_RegistryKey::SW_RegistryKey(struct HKEY__ *))
        6    ??0SW_RegistryKey@@QAA@XZ (public: __cdecl SW_RegistryKey::SW_RegistryKey(void))
        7    ??1CVerInfo@@QAA@XZ (public: __cdecl CVerInfo::~CVerInfo(void))
        8    ??1SW_RegistryKey@@QAA@XZ (public: __cdecl SW_RegistryKey::~SW_RegistryKey(void))
        9    ??4CVerInfo@@QAAAAV0@ABV0@@Z (public: class CVerInfo & __cdecl CVerInfo::operator=(class CVerInfo const &))
       10    ??4SW_RegistryKey@@QAAAAV0@ABV0@@Z (public: class SW_RegistryKey & __cdecl SW_RegistryKey::operator=(class SW_RegistryKey const &))
       11    ??_7SW_RegistryKey@@6B@ (const SW_RegistryKey::`vftable')
       12    ?Buffer@SW_RegistryKey@@IAAXPAX@Z (protected: void __cdecl SW_RegistryKey::Buffer(void *))
       13    ?Buffer@SW_RegistryKey@@IBAPAXXZ (protected: void * __cdecl SW_RegistryKey::Buffer(void)const )
       14    ?ChangeCarrierIndex@@YAJKK@Z (long __cdecl ChangeCarrierIndex(unsigned long,unsigned long))
       15    ?CloseKey@SW_RegistryKey@@UAAJXZ (public: virtual long __cdecl SW_RegistryKey::CloseKey(void))
       16    ?ConvertPrefMode@@YAH_NH@Z (int __cdecl ConvertPrefMode(bool,int))
       17    ?CopyRegKey@@YAJPAUHKEY__@@PBG11H@Z (long __cdecl CopyRegKey(struct HKEY__ *,unsigned short const *,unsigned short const *,unsigned short const *,int))
       18    ?CreateKey@SW_RegistryKey@@UAAJPAUHKEY__@@PBGKPAK@Z (public: virtual long __cdecl SW_RegistryKey::CreateKey(struct HKEY__ *,unsigned short const *,unsigned long,unsigned long *))
       19    ?CreateKey@SW_RegistryKey@@UAAJPBGKPAK@Z (public: virtual long __cdecl SW_RegistryKey::CreateKey(unsigned short const *,unsigned long,unsigned long *))
       20    ?DWORD2IP@@YAPBGK@Z (unsigned short const * __cdecl DWORD2IP(unsigned long))
       21    ?DecodeAreaCode@@YA_NPAGG@Z (bool __cdecl DecodeAreaCode(unsigned short *,unsigned short))
       22    ?DecodeMCC1112@@YAHH_N@Z (int __cdecl DecodeMCC1112(int,bool))
       23    ?DecodePhoneNumber@@YA_NPAGK@Z (bool __cdecl DecodePhoneNumber(unsigned short *,unsigned long))
       24    ?DeleteRegKey@@YAJPAUHKEY__@@PBG1H@Z (long __cdecl DeleteRegKey(struct HKEY__ *,unsigned short const *,unsigned short const *,int))
       25    ?DeleteSubKey@SW_RegistryKey@@IAAJPBG@Z (protected: long __cdecl SW_RegistryKey::DeleteSubKey(unsigned short const *))
       26    ?DisplayRawData@@YAXIPAEHPBG@Z (void __cdecl DisplayRawData(unsigned int,unsigned char *,int,unsigned short const *))
       27    ?Duplicate@SW_RegistryKey@@QAAHAAV1@@Z (public: int __cdecl SW_RegistryKey::Duplicate(class SW_RegistryKey &))
       28    ?EnableCarrierLogo@@YAXH@Z (void __cdecl EnableCarrierLogo(int))
       29    ?EncodeMCC1112@@YAHPBG_N@Z (int __cdecl EncodeMCC1112(unsigned short const *,bool))
       30    ?EncodePhoneNumber@@YA_NPAGPAK@Z (bool __cdecl EncodePhoneNumber(unsigned short *,unsigned long *))
       31    ?EnumKey@SW_RegistryKey@@IAAJAAKPAG@Z (protected: long __cdecl SW_RegistryKey::EnumKey(unsigned long &,unsigned short *))
       32    ?GetActWizDisabled@@YAKXZ (unsigned long __cdecl GetActWizDisabled(void))
       33    ?GetAutoUpdateTime@@YAKXZ (unsigned long __cdecl GetAutoUpdateTime(void))
       34    ?GetAutoUpdateTimeUI@@YAKXZ (unsigned long __cdecl GetAutoUpdateTimeUI(void))
       35    ?GetAvailMem@@YAKXZ (unsigned long __cdecl GetAvailMem(void))
       36    ?GetAvailProgramMem@@YAKXZ (unsigned long __cdecl GetAvailProgramMem(void))
       37    ?GetAvailStoreMem@@YAKXZ (unsigned long __cdecl GetAvailStoreMem(void))
       38    ?GetCallGuardReg@@YAKXZ (unsigned long __cdecl GetCallGuardReg(void))
       39    ?GetCarrierIndex@@YAKXZ (unsigned long __cdecl GetCarrierIndex(void))
       40    ?GetDataPortDetails@@YAHPAGAAK@Z (int __cdecl GetDataPortDetails(unsigned short *,unsigned long &))
       41    ?GetFileVersionStr@CVerInfo@@QAAPAGXZ (public: unsigned short * __cdecl CVerInfo::GetFileVersionStr(void))
       42    ?GetLogoTestReg@@YAKXZ (unsigned long __cdecl GetLogoTestReg(void))
       43    ?GetMdnLen@@YAHAAK@Z (int __cdecl GetMdnLen(unsigned long &))
       44    ?GetMemUsed@@YAKXZ (unsigned long __cdecl GetMemUsed(void))
       45    ?GetProductFeatures@@YAHAAK@Z (int __cdecl GetProductFeatures(unsigned long &))
       46    ?GetProductNameStr@CVerInfo@@QAAPAGXZ (public: unsigned short * __cdecl CVerInfo::GetProductNameStr(void))
       47    ?GetProductVersionStr@CVerInfo@@QAAPAGXZ (public: unsigned short * __cdecl CVerInfo::GetProductVersionStr(void))
       48    ?GetRegValue@@YAJPAUHKEY__@@PBG1AAK@Z (long __cdecl GetRegValue(struct HKEY__ *,unsigned short const *,unsigned short const *,unsigned long &))
       49    ?GetRegValue@@YAJPAUHKEY__@@PBG1PAEPAK@Z (long __cdecl GetRegValue(struct HKEY__ *,unsigned short const *,unsigned short const *,unsigned char *,unsigned long *))
       50    ?GetRegValue@@YAJPAUHKEY__@@PBG1PAGPAK@Z (long __cdecl GetRegValue(struct HKEY__ *,unsigned short const *,unsigned short const *,unsigned short *,unsigned long *))
       51    ?GetResolution@@YAHXZ (int __cdecl GetResolution(void))
       52    ?GetSpecialNumber@@YAJPAG@Z (long __cdecl GetSpecialNumber(unsigned short *))
       53    ?GetVerInfo@@YAPAGPAUHINSTANCE__@@@Z (unsigned short * __cdecl GetVerInfo(struct HINSTANCE__ *))
       54    ?GetVerResourceStr@CVerInfo@@QAAPAGPAG@Z (public: unsigned short * __cdecl CVerInfo::GetVerResourceStr(unsigned short *))
       55    ?GetVerResourceString@CVerInfo@@AAAPAGPAG@Z (private: unsigned short * __cdecl CVerInfo::GetVerResourceString(unsigned short *))
       56    ?HKey@SW_RegistryKey@@IAAQAUHKEY__@@QAU2@@Z (protected: struct HKEY__ * __cdecl SW_RegistryKey::HKey(struct HKEY__ * const))
       57    ?HKey@SW_RegistryKey@@IBAQAUHKEY__@@XZ (protected: struct HKEY__ * __cdecl SW_RegistryKey::HKey(void)const )
       58    ?IP2DWORD@@YAKPBG@Z (unsigned long __cdecl IP2DWORD(unsigned short const *))
       59    ?InWideMode@@YAHXZ (int __cdecl InWideMode(void))
       60    ?Init@CVerInfo@@AAAHPAG@Z (private: int __cdecl CVerInfo::Init(unsigned short *))
       61    ?InitLog@@YAXPAUHINSTANCE__@@@Z (void __cdecl InitLog(struct HINSTANCE__ *))
       62    ?InitObject@SW_RegistryKey@@MAAXXZ (protected: virtual void __cdecl SW_RegistryKey::InitObject(void))
       63    ?InitVerInfoStruct@CVerInfo@@AAAHPAG@Z (private: int __cdecl CVerInfo::InitVerInfoStruct(unsigned short *))
       64    ?IsConsumerProduct@@YAHXZ (int __cdecl IsConsumerProduct(void))
       65    ?IsOpen@SW_RegistryKey@@UAAHXZ (public: virtual int __cdecl SW_RegistryKey::IsOpen(void))
       66    ?LocalToUTCTime@@YAHPAU_SYSTEMTIME@@0@Z (int __cdecl LocalToUTCTime(struct _SYSTEMTIME *,struct _SYSTEMTIME *))
       67    ?LogC@@YAXPBGZZ (void __cdecl LogC(unsigned short const *,...))
       68    ?LogStoreFileLine@@YAXPAGH@Z (void __cdecl LogStoreFileLine(unsigned short *,int))
       69    ?LogV@@YAXPBGZZ (void __cdecl LogV(unsigned short const *,...))
       70    ?LogW@@YAXPBGZZ (void __cdecl LogW(unsigned short const *,...))
       71    ?LogWindowText@@YAXPBGZZ (void __cdecl LogWindowText(unsigned short const *,...))
       72    ?OpenKey@SW_RegistryKey@@UAAJPAUHKEY__@@PBGK@Z (public: virtual long __cdecl SW_RegistryKey::OpenKey(struct HKEY__ *,unsigned short const *,unsigned long))
       73    ?OpenKey@SW_RegistryKey@@UAAJPBGK@Z (public: virtual long __cdecl SW_RegistryKey::OpenKey(unsigned short const *,unsigned long))
       74    ?QueryValue@SW_RegistryKey@@UAAJPBGPAK@Z (public: virtual long __cdecl SW_RegistryKey::QueryValue(unsigned short const *,unsigned long *))
       75    ?QueryValue@SW_RegistryKey@@UAAJPBGPAPAEPAK@Z (public: virtual long __cdecl SW_RegistryKey::QueryValue(unsigned short const *,unsigned char * *,unsigned long *))
       76    ?QueryValue@SW_RegistryKey@@UAAJPBGPAPAG@Z (public: virtual long __cdecl SW_RegistryKey::QueryValue(unsigned short const *,unsigned short * *))
       77    ?RecurseDeleteKey@SW_RegistryKey@@QAAJPBG@Z (public: long __cdecl SW_RegistryKey::RecurseDeleteKey(unsigned short const *))
       78    ?RelayoutDialog@@YAHPAUHINSTANCE__@@PAUHWND__@@PBG@Z (int __cdecl RelayoutDialog(struct HINSTANCE__ *,struct HWND__ *,unsigned short const *))
       79    ?RenameRegKey@@YAJPAUHKEY__@@PBG11H@Z (long __cdecl RenameRegKey(struct HKEY__ *,unsigned short const *,unsigned short const *,unsigned short const *,int))
       80    ?SWAI_GetRegValue@@YAJPAUHKEY__@@PBG1AAK@Z (long __cdecl SWAI_GetRegValue(struct HKEY__ *,unsigned short const *,unsigned short const *,unsigned long &))
       81    ?SWAI_GetRegValue@@YAJPAUHKEY__@@PBG1PAEPAK@Z (long __cdecl SWAI_GetRegValue(struct HKEY__ *,unsigned short const *,unsigned short const *,unsigned char *,unsigned long *))
       82    ?SWAI_GetRegValue@@YAJPAUHKEY__@@PBG1PAGPAK@Z (long __cdecl SWAI_GetRegValue(struct HKEY__ *,unsigned short const *,unsigned short const *,unsigned short *,unsigned long *))
       83    ?SWAI_SetRegValue@@YAJPAUHKEY__@@PBG11@Z (long __cdecl SWAI_SetRegValue(struct HKEY__ *,unsigned short const *,unsigned short const *,unsigned short const *))
       84    ?SWAI_SetRegValue@@YAJPAUHKEY__@@PBG1K@Z (long __cdecl SWAI_SetRegValue(struct HKEY__ *,unsigned short const *,unsigned short const *,unsigned long))
       85    ?SWAI_SetRegValue@@YAJPAUHKEY__@@PBG1QAEK@Z (long __cdecl SWAI_SetRegValue(struct HKEY__ *,unsigned short const *,unsigned short const *,unsigned char * const,unsigned long))
       86    ?SW_AtoT@@YAPAGPAGPADK@Z (unsigned short * __cdecl SW_AtoT(unsigned short *,char *,unsigned long))
       87    ?SW_TtoA@@YAPADPADPAGK@Z (char * __cdecl SW_TtoA(char *,unsigned short *,unsigned long))
       88    ?SetActWizDisabled@@YAXK@Z (void __cdecl SetActWizDisabled(unsigned long))
       89    ?SetAutoUpdateTime@@YAXH@Z (void __cdecl SetAutoUpdateTime(int))
       90    ?SetAutoUpdateTimeUI@@YAXK@Z (void __cdecl SetAutoUpdateTimeUI(unsigned long))
       91    ?SetCallGuardReg@@YAXK@Z (void __cdecl SetCallGuardReg(unsigned long))
       92    ?SetConnectionProfile@@YAJXZ (long __cdecl SetConnectionProfile(void))
       93    ?SetFileVersionStr@CVerInfo@@AAAXXZ (private: void __cdecl CVerInfo::SetFileVersionStr(void))
       94    ?SetLimitText@@YAJPAUHWND__@@H@Z (long __cdecl SetLimitText(struct HWND__ *,int))
       95    ?SetNormalCursor@@YAXXZ (void __cdecl SetNormalCursor(void))
       96    ?SetProductNameStr@CVerInfo@@AAAXXZ (private: void __cdecl CVerInfo::SetProductNameStr(void))
       97    ?SetProductVersionStr@CVerInfo@@AAAXXZ (private: void __cdecl CVerInfo::SetProductVersionStr(void))
       98    ?SetRegValue@@YAJPAUHKEY__@@PBG11@Z (long __cdecl SetRegValue(struct HKEY__ *,unsigned short const *,unsigned short const *,unsigned short const *))
       99    ?SetRegValue@@YAJPAUHKEY__@@PBG1K@Z (long __cdecl SetRegValue(struct HKEY__ *,unsigned short const *,unsigned short const *,unsigned long))
      100    ?SetRegValue@@YAJPAUHKEY__@@PBG1QAEK@Z (long __cdecl SetRegValue(struct HKEY__ *,unsigned short const *,unsigned short const *,unsigned char * const,unsigned long))
      101    ?SetSpecialNumber@@YAJPAG@Z (long __cdecl SetSpecialNumber(unsigned short *))
      102    ?SetValue@SW_RegistryKey@@UAAJPBG0@Z (public: virtual long __cdecl SW_RegistryKey::SetValue(unsigned short const *,unsigned short const *))
      103    ?SetValue@SW_RegistryKey@@UAAJPBGK@Z (public: virtual long __cdecl SW_RegistryKey::SetValue(unsigned short const *,unsigned long))
      104    ?SetValue@SW_RegistryKey@@UAAJPBGQAEK@Z (public: virtual long __cdecl SW_RegistryKey::SetValue(unsigned short const *,unsigned char * const,unsigned long))
      105    ?SetWaitCursor@@YAXXZ (void __cdecl SetWaitCursor(void))
      106    ?TBD_Assert@@YA_N_NQBG1H@Z (bool __cdecl TBD_Assert(bool,unsigned short const * const,unsigned short const * const,int))
      107    ?TBD_Output@@YAXW4TBD_CLASS_TYPE@@W4TBD_OUTPUT_LEVEL@@QBGZZ (void __cdecl TBD_Output(enum TBD_CLASS_TYPE,enum TBD_OUTPUT_LEVEL,unsigned short const * const,...))
      108    ?THtoT@@YAXPAG0H@Z (void __cdecl THtoT(unsigned short *,unsigned short *,int))
      109    ?TtoTH@@YAXPAG0H@Z (void __cdecl TtoTH(unsigned short *,unsigned short *,int))
      110    ?WriteLog@@YAXKPBGZZ (void __cdecl WriteLog(unsigned long,unsigned short const *,...))
      111    ?WriteLog@@YAXPAVSW_Log@@KPBGPAPAD@Z (void __cdecl WriteLog(class SW_Log *,unsigned long,unsigned short const *,char * *))
      112    ?WriteLog@@YAXPAVSW_Log@@KPBGZZ (void __cdecl WriteLog(class SW_Log *,unsigned long,unsigned short const *,...))
      113    ?WriteLog@@YAXPAVSW_Log@@PBGZZ (void __cdecl WriteLog(class SW_Log *,unsigned short const *,...))
      114    ?WriteLog@@YAXPBGZZ (void __cdecl WriteLog(unsigned short const *,...))
      115    ChangeCarrierIndex
      116    Dial
      117    DialEx
      118    EnableCarrierLogo
      119    EnableIOTA
      120    EnableTechHdrNotifications
      121    EndLBTrackSession
      122    GetActWizDisabledRegistry
      123    GetActWizUIMask
      124    GetAdvancedMenuInfo
      125    GetAutoUpdateTime
      126    GetAutoUpdateTimeUI
      127    GetByteCounter
      128    GetCallGuardRegistry
      129    GetCallstate
      130    GetCarrierIndex
      131    GetCurrentGSMBandAndList
      132    GetDMMode
      133    GetDsMipList
      134    GetDsMipProfile
      135    GetGSMInfo
      136    GetHdrNaiPassword
      137    GetIOTALog
      138    GetIOTALogSize
      139    GetIOTAStatus
      140    GetItemnizedUMTSInfo
      141    GetLogoTestReg
      142    GetMDNLengthSupported
      143    GetNAIPWUIDisplayMode
      144    GetOMADMConfig
      145    GetPTMode
      146    GetProvisionInfo
      147    GetProvisionState
      148    GetRilDebugInfo
      149    GetRilEVDODebugInfo
      150    GetRilPAParam
      151    GetRilPDDLDData
      152    GetRilPDData
      153    GetRilStatus
      154    GetRilTechHdrinfo
      155    GetSIPNaiPassword
      156    GetUserIdentity
      157    GetVersionInfo
      158    HangUp
      159    InitiateHostBoot
      160    IsConsumerProduct
      161    IsIOTAEnabled
      162    ModGetHDRHybrPrefMode
      163    ModGetLocationStatus
      164    ModGetPreferredPrivacyMode
      165    ModGetRoamStatus
      166    ModGetRoamingMode
      167    ModGetSysPrefMode
      168    ModSetHDRHybrPrefMode
      169    ModSetLocationMode
      170    ModSetPreferredPrivacyMode
      171    ModSetRoamingMode
      172    ModSetSysPrefMode
      173    ReadNv
      174    ReadPDSMPAData
      175    ReadPDSMPADldData
      176    ReadPDSMPAParam
      177    RepairPhoneBookRegKeys
      178    RtnReset
      179    SaveAkey
      180    SelectGSMBand
      181    SendATTunnel
      182    SetActWizDisabledRegistry
      183    SetAutoUpdateTime
      184    SetAutoUpdateTimeUI
      185    SetCallGuardRegistry
      186    SetDsMipProfile
      187    SetEquipmentState
      188    SetHdrNaiPassword
      189    SetModemPowerState
      190    SetPDSMPAParam
      191    SetProvisionInfo
      192    SetSIPNaiPassword
      193    StartDMMode
      194    StartDebugMode
      195    StartIOTA
      196    StartLBTrackSession
      197    StartPDSMDldNotifstatus
      198    StartPDSMLocNotifstatus
      199    StartPTMode
      200    StopDMMode
      201    StopDebugMode
      202    StopIOTA
      203    StopPDSMDldNotifstatus
      204    StopPDSMLocNotifstatus
      205    StopPTMode
      206    ValidateSpc
      207    WriteNv
